:020000022000DC
:1060000000000420DDA30200B98402005D990200B3
:10601000B9840200B9840200B984020000000000C3
:10602000000000000000000000000000B984020031
:10603000B984020000000000B9840200B9840200A3
:1060400089A20200B98402002DA8020031A4020036
:1060500041A40200B984020085970200B9840200BD
:10606000B98402000DA802001DA80200ADA3020021
:10607000B9840200B9840200B9840200B984020024
:1060800055A80200BDA30200B9840200B984020031
:10609000B9840200B984020069A50200B984020033
:1060A000B9840200B9840200B9840200B9840200F4
:1060B000B9840200B9840200000000000000000062
:1060C000B9840200B9840200B984020051A402001C
:1060D000CDA30200B9840200B98402004DA80200D9
:1060E0003DA8020089A30200B9840200D9A40200DD
:0860F00000000000B984020069
:1070000040F8044B40F8045B40F8046B40F8047B04
:1070100040F8048B40F8049B40F804AB40F804BBF4
:1070200040F804CB40F804DB6846704781F000412B
:1070300002E000BF83F0004330B54FEA41044FEA5D
:10704000430594EA050F08BF90EA020F1FBF54EAF8
:10705000000C55EA020C7FEA645C7FEA655C00F094
:10706000E2804FEA5454D4EB5555B8BF6D420CDD65
:107070002C4480EA020281EA030382EA000083EAE8
:10708000010180EA020281EA0303362D88BF30BD88
:1070900011F0004F4FEA01314FF4801C4CEA1131DE
:1070A00002D0404261EB410113F0004F4FEA03333D
:1070B0004CEA133302D0524263EB430394EA050FC8
:1070C00000F0A780A4F10104D5F1200E0DDB02FA37
:1070D0000EFC22FA05F2801841F1000103FA0EF2CB
:1070E000801843FA05F359410EE0A5F120050EF191
:1070F000200E012A03FA0EFC28BF4CF0020C43FAC2
:1071000005F3C01851EBE37101F0004507D54FF0CE
:10711000000EDCF1000C7EEB00006EEB0101B1F51E
:10712000801F1BD3B1F5001F0CD349085FEA300064
:107130004FEA3C0C04F101044FEA445212F5800F6F
:1071400080F09A80BCF1004F08BF5FEA500C50F10C
:10715000000041EB045141EA050130BD5FEA4C0CEF
:10716000404141EB0101013C28BFB1F5801FE9D24C
:1071700091F0000F04BF01460020B1FA81F308BF6F
:107180002033A3F10B03B3F120020CDA0C3208DD3B
:1071900002F1140CC2F10C0201FA0CF021FA02F116
:1071A0000CE002F11402D8BFC2F1200C01FA02F186
:1071B00020FA0CFCDCBF41EA0C019040E41AA2BFAB
:1071C00001EB0451294330BD6FEA04041F3C1CDA73
:1071D0000C340EDC04F11404C4F1200220FA04F093
:1071E00001FA02F340EA030021FA04F345EA03013D
:1071F00030BDC4F10C04C4F1200220FA02F001FAFF
:1072000004F340EA0300294630BD21FA04F0294680
:1072100030BD94F0000F83F4801306BF81F4801119
:107220000134013D4EE77FEA645C18BF7FEA655C8C
:1072300029D094EA050F08BF90EA020F05D054EA5E
:10724000000C04BF1946104630BD91EA030F1EBF63
:107250000021002030BD5FEA545C05D14000494167
:1072600028BF41F0004130BD14F580043CBF01F55A
:10727000801130BD01F0004545F0FE4141F4700140
:107280004FF0000030BD7FEA645C1ABF194610461B
:107290007FEA655C1CBF0B46024650EA013406BF1C
:1072A00052EA033591EA030F41F4002130BD00BFDB
:1072B00090F0000F04BF0021704730B54FF4806498
:1072C00004F132044FF000054FF0000150E700BF19
:1072D00090F0000F04BF0021704730B54FF4806478
:1072E00004F1320410F0004548BF40424FF0000165
:1072F0003EE700BF42004FEAE2014FEA31014FEAA8
:1073000002701FBF12F07F4393F07F4F81F06051F6
:10731000704732F07F4208BF704793F07F4F04BF41
:1073200041F40021704730B54FF4607401F000451E
:1073300021F000411CE700BF50EA010208BF70477E
:1073400030B54FF000050AE050EA010208BF70476F
:1073500030B511F0004502D5404261EB41014FF4D8
:10736000806404F132045FEA915C3FF4D8AE4FF0E0
:1073700003025FEADC0C18BF03325FEADC0C18BFC3
:10738000033202EBDC02C2F1200300FA03FC20FA14
:1073900002F001FA03FE40EA0E0021FA02F1144461
:1073A000BDE600BF4FEA4102B2F1E04324BFB3F5AE
:1073B000001CDCF1FE5C0DD901F0004C4FEAC0026C
:1073C0004CEA5070B2F1004F40EB830008BF20F050
:1073D0000100704711F0804F21D113F13872BCBF0A
:1073E00001F00040704741F480114FEA5252C2F15F
:1073F0001802C2F1200C10FA0CF320FA02F018BFA8
:1074000040F001004FEAC1234FEAD32303FA0CFCFA
:1074100040EA0C0023FA02F34FEA4303CCE77FEA89
:10742000625307D150EA01331EBF4FF0FE4040F4D3
:107430004000704701F0004040F0FE4040F4000082
:10744000704700BF80F0004002E000BF81F00041C3
:1074500042001FBF5FEA410392EA030F7FEA226CFA
:107460007FEA236C6AD04FEA1262D2EB1363C1BF8A
:10747000D218414048404140B8BF5B42192B88BFF9
:10748000704710F0004F40F4000020F07F4018BF1C
:10749000404211F0004F41F4000121F07F4118BF3C
:1074A000494292EA030F3FD0A2F1010241FA03FCE4
:1074B00010EB0C00C3F1200301FA03F100F00043CC
:1074C00002D5494260EB4000B0F5000F13D3B0F194
:1074D000807F06D340084FEA310102F10102FE2A03
:1074E00051D2B1F1004F40EBC25008BF20F0010073
:1074F00040EA03007047490040EB0000013A28BF12
:10750000B0F5000FEDD2B0FA80FCACF1080CB2EB94
:107510000C0200FA0CF0AABF00EBC2505242184312
:10752000BCBFD0401843704792F0000F81F40001B7
:1075300006BF80F400000132013BB5E74FEA41038A
:107540007FEA226C18BF7FEA236C21D092EA030FF6
:1075500004D092F0000F08BF0846704790EA010F70
:107560001CBF0020704712F07F4F04D1400028BF9D
:1075700040F00040704712F100723CBF00F500007F
:10758000704700F0004343F0FE4040F400007047B5
:107590007FEA226216BF08467FEA23630146420261
:1075A00006BF5FEA412390EA010F40F48000704774
:1075B0004FF0000304E000BF10F0004348BF40421A
:1075C0005FEA000C08BF704743F0964301464FF056
:1075D00000001CE050EA010208BF70474FF00003B2
:1075E0000AE000BF50EA010208BF704711F00043F3
:1075F00002D5404261EB41015FEA010C02BF8446C3
:107600000146002043F0B64308BFA3F18053A3F521
:107610000003BCFA8CF2083AA3EBC25310DB01FA68
:1076200002FC634400FA02FCC2F12002BCF1004FEC
:1076300020FA02F243EB020008BF20F0010070477D
:1076400002F1200201FA02FCC2F1200250EA4C00D1
:1076500021FA02F243EB020008BF20EADC70704717
:107660007BB972B90029BEBF00204FF0004106E08F
:1076700008BF00281CBF6FF000414FF0FF3000F042
:1076800081B9ADF1080C6DE904CE002909DB002BAE
:107690001ADB05F0F5FDDDF804E0DDE9022304B0B6
:1076A0007047404261EB4101002B1BDB05F0E8FD18
:1076B000DDF804E0DDE9022304B0404261EB410162
:1076C000524263EB43037047524263EB430305F0BE
:1076D000D7FDDDF804E0DDE9022304B0404261EBB0
:1076E00041017047524263EB430305F0C9FDDDF8E9
:1076F00004E0DDE9022304B0524263EB4303704728
:1077000053B94AB9002908BF00281CBF4FF0FF3108
:107710004FF0FF3000F036B9ADF1080C6DE904CE42
:1077200005F0AEFDDDF804E0DDE9022304B07047AA
:1077300070B54FF0FF0C4CF4E06C1CEA11541DBF07
:107740001CEA135594EA0C0F95EA0C0F00F0DEF8D2
:107750002C4481EA030621EA4C5123EA4C5350EAB7
:10776000013518BF52EA033541F4801143F4801308
:1077700038D0A0FB02CE4FF00005E1FB02E506F099
:107780000042E0FB03E54FF00006E1FB03569CF0EE
:10779000000F18BF4EF0010EA4F1FF04B6F5007FF4
:1077A00064F5407404D25FEA4E0E6D4146EB060666
:1077B00042EAC62141EA55514FEAC52040EA5E50EF
:1077C0004FEACE2EB4F1FD0C88BFBCF5E06F1ED899
:1077D000BEF1004F08BF5FEA500E50F1000041EBD0
:1077E000045170BD06F0004646EA010140EA02007D
:1077F00081EA0301B4EB5C04C2BFD4EB0C0541EA9F
:10780000045170BD41F480114FF0000E013C00F3B3
:10781000AB8014F1360FDEBF002001F0004170BDD7
:10782000C4F10004203C35DA0C341BDC04F11404F0
:10783000C4F1200500FA05F320FA04F001FA05F27C
:1078400040EA020001F0004221F0004110EBD37049
:1078500021FA04F642EB06015EEA430E08BF20EA75
:10786000D37070BDC4F10C04C4F1200500FA04F318
:1078700020FA05F001FA04F240EA020001F00041AA
:1078800010EBD37041F100015EEA430E08BF20EA1D
:10789000D37070BDC4F1200500FA05F24EEA020E65
:1078A00020FA04F301FA05F243EA020321FA04F094
:1078B00001F0004121FA04F220EA020000EBD3704B
:1078C0005EEA430E08BF20EAD37070BD94F0000F4B
:1078D0000FD101F00046400041EB010111F4801F7F
:1078E00008BF013CF7D041EA060195F0000F18BF30
:1078F000704703F00046520043EB030313F4801F6C
:1079000008BF013DF7D043EA0603704794EA0C0F25
:107910000CEA135518BF95EA0C0F0CD050EA41063B
:1079200018BF52EA4306D1D181EA030101F00041B8
:107930004FF0000070BD50EA410606BF10461946E0
:1079400052EA430619D094EA0C0F02D150EA0136EC
:1079500013D195EA0C0F05D152EA03361CBF10462D
:1079600019460AD181EA030101F0004141F0FE41CC
:1079700041F470014FF0000070BD41F0FE4141F450
:10798000780170BD704700BF4A0011D212F5001295
:1079900011D20DD56FF47873B3EB62520ED44FEA67
:1079A000C12343F0004343EA505323FA02F07047E7
:1079B0004FF00000704750EA013002D14FF0FF3025
:1079C00070474FF0000070479FED197B70B51A4C5F
:1079D00084ED007B41B30023DFF868E0101F1D46F3
:1079E0009C4602E0013399420FD050F8042F9607CD
:1079F000F8D116687645F5D1BCF1000F15D10133E9
:107A0000994215464FF0010CEFD1BCF1000F0BD09D
:107A100095ED017ADFED097A67EE277A17EE900A85
:107A200004F016FAC4E9000170BD054879F010FBB6
:107A300000000000000000000012012000007A4455
:107A4000D4890B0014C70B0090F8743043F0007316
:107A500003F17E43033B102B05D8DFF83CC05CF8F4
:107A600023309A4213D310B59FED097BA0B00C468A
:107A7000043004A98DED047B019264F00BFD019AA2
:107A800003AB214604A864F029FD20B010BD704767
:107A90000000000000000000EC2D0C0000000000C1
:107AA00010B584B004469DF820E09DF828C00393EB
:107AB00008469DF81C1084F8371000216EF307016A
:107AC0006CF30F21BDF818C084F832C0CCF1080C5B
:107AD00084F836C09DF82CC09FED0F7B6CF31741E6
:107AE000E163002121609DF8241084F8331084EDB7
:107AF000027B1146CDE9010271F094FC0198029AD3
:107B00000399A0852046E28504B0BDE810402DF021
:107B10007BBE00BFAFF3008000000000000000004B
:107B200000B59FED0D7B89B00923016802904FF0ED
:107B30000A0C039302A800238DED007BCDF810C042
:107B4000CDF814D08DF8183046F01CF800980038A5
:107B500018BF012009B000BD0000000000000000B7
:107B600010B5144686B017A3D3E90023FFF778FDBC
:107B700003A9019074F0FCFD9DF80F309DF80E20D4
:107B800001980F491B0443EA42539DF8102043EA31
:107B9000C2239DF8112043EA42139DF8122043EAC4
:107BA0005203BDF80C2020F00100A2F2BC72A0FB31
:107BB000010143EA4263236006B010BDAFF30080C9
:107BC00000CA9A3B00CA9A3B000000000000000077
:107BD0002DE9F04F87B000AF00240E46904607F124
:107BE0000801012282463C7266F09CFB97F908006E
:107BF000397AA04234DA01F0E003E02B30D0A02B38
:107C000036D001F0F003902B00F0A581802B00F01E
:107C1000AB81A1F1C0031F2B00F29A81DFE813F0C2
:107C200094019801960192015800580058008B0069
:107C30008B008B004401C800E600F30028015701C7
:107C4000680176018401020113011A012101360144
:107C50003D0141004100410097009700A400A400AD
:107C6000400040F0010318461C37BD46BDE8F08FC8
:107C700001F01F02D31D03F038036C46ADEB030D7A
:107C80006B463AB169465046C7E9003266F04AFB96
:107C9000D7E900321846114649F06AF90346A5466D
:107CA000E1E72731C9B2504666F000FC04460146C0
:107CB00007F108007DF04CFF24B139692246504697
:107CC00066F030FB07F1080049F09CF90346CAE76B
:107CD0003C31C9B2504666F0E9FB04468046014695
:107CE00007F108007DF034FFFCB139697960B8F51F
:107CF000807F444628BF4FF480740AF10C03DAE910
:107D000000062246B0470346DAF80C0079680028DE
:107D100040F04A81002B00F04C819C4200F24681E9
:107D2000B8EB040321449846E0D107F1080048F07D
:107D3000D9FD034697E73931C9B2504666F0B6FB24
:107D400032460146504679F0E9F903468BE7253182
:107D5000C9B2504666F0AAFB434601463246504639
:107D600079F0A8F903467EE72331C9B2504666F0A0
:107D70009DFB0446834648F043FE0346002C3FF437
:107D800072AF00244246314650467B60FFF720FF29
:107D90004246814631465046FFF71AFF01340246FB
:107DA0004946786846F0D0F9A3457B68EAD15AE79E
:107DB0009FED837B0822B918504687ED027B66F061
:107DC000B1FAD7E9023210BA19BAFFF7EBFA07EEA7
:107DD000900AF4EE677AF1EE10FA76D6034623F0B5
:107DE000030343F00203A3F1FF433CE70023012216
:107DF00007F1080150463B7266F094FA3B7A5B004B
:107E000043F001032FE70023022207F10801504647
:107E10003B8166F087FA3B895BBA9BB25B0043F01B
:107E2000010320E79FED667B0822B918504687EDD5
:107E3000027B66F077FAD7E9021009BA00BA48F077
:107E400071FF03460FE732460121504679F066F98B
:107E5000034608E732460221504679F05FF90346AF
:107E600001E732460421504679F058F90346FAE614
:107E70000023042207F108015046BB6066F052FA65
:107E8000B86800BA48F08AFF0346ECE6324608219B
:107E9000504679F043F90346E5E632461021504654
:107EA00079F03CF90346DEE60023042207F10801DD
:107EB0005046BB6066F036FABB681BBA07EE903AD4
:107EC000F4EE677AF1EE10FA89D73F4BCBE69FEDDF
:107ED0003C7B0822B918504687ED027B66F022FAF7
:107EE000D7E9021009BA00BA48F07AFF0346BAE6A9
:107EF0000023012207F1080150463B7266F012FA96
:107F000097F908305B0043F00103ACE6002302223E
:107F100007F1080150463B8166F004FA3B89DBBA61
:107F20005B0043F001039EE60023042207F10801F1
:107F30005046BB6066F0F6F9B86800BA48F088FEB3
:107F4000034690E63E238EE60E238CE61E238AE649
:107F50001E4879F07DF84346324601F00F01504645
:107F600079F0A8F803467EE601F00F05284648F0B0
:107F700047FDAB460346002D3FF475AE4246314601
:107F800050467B60FFF724FE42468146314650460C
:107F9000FFF71EFE013402464946786846F0D4F8E1
:107FA000A3457B68EAD15EE678F0EEFF084879F0F9
:107FB0004FF80848194684F060FB00BFAFF300801B
:107FC000000000000000000002004000648C0B0074
:107FD000C0750B0074530B00D2B32DE9F0436FF062
:107FE0000E0885B00646174601F10F04A8EB0108FC
:107FF00054F80F0C54F80B1C54F8072C54F8033C9D
:10800000EC46ACE80F003146A4F10F0001F0AAFCE9
:10801000A4F1100306F1EF0213F8011F12F8010F8B
:10802000A34281EA00011970F6D1EC46BCE80F00CA
:10803000103408EB040C6745C6F8F000C6F8F410DD
:10804000C6F8F820C6F8FC30D2D805B0BDE8F083F9
:10805000704700BF2DE9F041044682B36FF00E0572
:10806000164601F10F0700F1F0086D1A08F1FF3113
:10807000A7F11003A7F10F0813F8012F11F801CF92
:10808000BB4282EA0C021A70F6D1214640461037F4
:1080900000F018F9EB199E42E8D8D8F80010D8F88B
:1080A0000420D8F80830D8F80C00C4F8FC00C4F854
:1080B000F010C4F8F420C4F8F830BDE8F08100F105
:1080C000F008EAE7002A44D070B54C1E84B006469A
:1080D00015194FF0100C01E00CF1010CBCF1100F60
:1080E0000BD00DEB0C0214F8013F1278AC4283EA7E
:1080F00002032370F0D104B070BDD6F8F000D6F8BA
:10810000F410D6F8F820D6F8FC30EC46ACE80F00B6
:108110003146684600F0D6F80F2206F5807111F856
:10812000013DFF2B0FD03244013382F8F03014F8B8
:10813000013F9DF80020AC4283EA02032370DAD0AD
:108140004FF0010CCDE70023013A0B70531CE6D130
:10815000EDE7704703460846194601F003BC00BF2F
:1081600003460846194600F0ADB800BF182A2DE9AD
:10817000F04F0546C0F800217ED0202A76D0102A84
:108180007ED1834640F20A43A5F80431AC46002074
:108190000B788CF800304B788CF801308B788CF8A9
:1081A0000230CB788CF8033095F8053101309842D5
:1081B0001A4601F104010CF1040CE9D395F80411FD
:1081C0000131B3EB810F55D20BEB8201501E11F838
:1081D00002EC1BF8204011F803CC11F8010C2B4FD6
:1081E000DFF8AC802DE017F80CA018F8099017F80C
:1081F0000EC017F800E0385D8AEA0904A2EB030913
:108200000BEB89031BF8299084EA09040C7093F89E
:10821000019004318CEA090C01F803CC93F8029028
:108220008EEA090E01F802ECDB78584001F8010CE7
:1082300095F8043101320133B2EB830F1AD295F86D
:108240000531B2FBF3F903FB192ABAF1000FCAD0CA
:10825000D5F80061202ED1D1BAF1040FCED13C5D0A
:1082600017F80CC017F80EE0385CC7E7834640F6F5
:108270000E0389E7BDE8F08F834640F20C6383E785
:1082800000239B46A0F804311A469DE7CC2C0C0035
:10829000C02B0C0000B583B0CDE90030FFF766FFBE
:1082A000009B0198D3F800C059689A68DB68C0F851
:1082B000FC30C0F8F0C0C0F8F410C0F8F82003B0EB
:1082C00000BD00BF2DE9F04FD1F80031103B102B5D
:1082D00085B08946864600F2E980754A22FA03F3A2
:1082E00013F0010F14BF0D4600250EF104063446AD
:1082F00000270EEB070379191A7811F8010B424099
:1083000003F8012B9C42F7D10437102F04F1040429
:10831000EFD10EF11008674FCDF804804FF0010C3B
:108320000EF11402AB46CA467146002311F8230031
:10833000385C01F823000133042BF7D101318E4260
:10834000F3D19EF805409EF809109EF801309EF882
:108350000D509EF802008EF801408EF805109EF830
:108360000A409EF806108EF809508EF80D309EF8DF
:108370000E509EF803308EF802408EF80A009EF8E8
:108380000F409EF80B008EF80E109EF807108EF826
:1083900006508EF803408EF80F008EF80B108EF802
:1083A00007309AF8043163456AD0CDE902CB7046B4
:1083B000047845788178C37884EA05094FEAD918AA
:1083C0004D404FEAD51C08EB480859405C4008EB8B
:1083D000C8080CEB4C0C00230CEBCC0C68F3070327
:1083E0006CF30F234FEAD11C0CEB4C0C0CEBCC0CB8
:1083F00089EA010B6CF317434FEA49094FF0000C6F
:108400006D0069F3070C490065F30F2C61F3174CFD
:108410000021E5096BF3070164006BF30F2105EB05
:10842000450564F31F6C6BF31741046805EBC50544
:108430006BF31F6165F31F6383EA0C0361404B40DC
:1084400040F8043B019B8342B2D1DDE902CB3446C4
:108450004FEA0C15231F0BEB0500197810F8018B60
:1084600081EA080103F8011B9C42F6D10434A242C0
:1084700005F10405EED10CF1010C5FFA8CFC53E719
:108480005D464FEA0C1C331F05EB0C00197810F801
:10849000014B614003F8011B9E42F7D10436B24202
:1084A0000CF1040CEFD105B0BDE8F08F00251CE7FE
:1084B00001010100CC2C0C00FEE700BF2DE9F04FBC
:1084C0004FEAA3095C4FDFF8ACB1DFF8ACA103F0D1
:1084D000030486464B4659488BB007EB84171C2B88
:1084E00050F824000090A8BF1C237868019703333C
:1084F00023EAE37318410790B86818410890F868B8
:1085000018410990B9F11F0F4FF00000C8460690BE
:10851000A8BF4FF01F080BE00DEB8505AC69002BE1
:1085200040EA0400B8BF6442013A41F8044B75D0F8
:108530005EF8043B13EA0B0F23F00045ECD013EA7E
:108540000A0F0BD1019CB9F1000F54F82540BABFB6
:10855000C8F10005AC4044FA08F4E0E7384C234287
:108560000DD1103D374C54F82540009D84FB056526
:10857000A8F10304002C47DB45FA04F4CFE76C04B0
:10858000B4F1006FBABF6C0504260026B4F1005F99
:10859000BCBFA40002362C4DB4F1804FBCBF6400B8
:1085A0000136AC423DDD294D294FCDE9045705F197
:1085B000F95505F5CE2505F29B150395254F264D5A
:1085C0000295254687FB05C5029F3D44274685FB4E
:1085D00007C7039D2F44254687FB05C5049F3D44DF
:1085E00085FB0474059D2C441C4D55F8265084FBD6
:1085F0000575EC00009D84FB0575194C54F8264068
:10860000A8EB0404002CB7DA66426FF0004444FA89
:1086100006F7AF4283DB05FA06F480E70BB0BDE84E
:10862000F08F104D104FDFF854C0CDE904570F4DB7
:108630000F4FCDE9025CC4E738440C0038450C000C
:10864000C0FFFF7F78430C009979825AF0CEC22791
:10865000B477F5FE63218510A4F633D338430C00BC
:1086600058430C008D496C23591858FF28482EB0E8
:10867000A9BDA029FCFFFF7FF0FFFF7F1BAA575970
:10868000844602F001007BBB60B3DCF88034DCF888
:108690008001DCF88012DCF880235B42CCF8803467
:1086A000DCF880384042494252425B42CCF88001BB
:1086B000CCF88012DCF88005DCF88016CCF880233A
:1086C000CCF88038DCF88027DCF880304042494222
:1086D00052425B42CCF88005CCF88016CCF880275B
:1086E000CCF88030002070472DE9F047C3F11F041B
:1086F000002847D04FF00047DF4000200CF18006F3
:10870000013F0CF51069804656F8802C42FA04FEB1
:10871000BEEBE27F87EAE27E18BF72469A4045468A
:1087200046F8802C82EAE275A5EBE275DCF8802041
:10873000C2F1000E4EFA04F2B2EBEE7F87EAEE725F
:1087400018BF96460EFA03F2CCF88020C64682EA9D
:10875000E27EAEEBE27E0A6845EA0E05284342FA65
:1087600004F5B5EBE27F87EAE27518BF2A460CF5FF
:10877000807C9A40E14541F8042B06F58076C3D110
:10878000BDE8F0874FF00046DE40013E0CF1800569
:108790000CF5106E074655F8802C42FA04F9B9EB37
:1087A000E27F86EAE27918BF4A469A40B84645F821
:1087B000802C82EAE278A8EBE278DCF8802042FAAA
:1087C00004FABAEBE27F86EAE27A18BF52469A4090
:1087D000B946CCF8802082EAE279A9EBE2790A680E
:1087E00048EA090840EA080042FA04F8B8EBE27FD8
:1087F00086EAE27818BF42460CF5807C9A40E6454E
:1088000041F8042B05F58075C5D1BDE8F08700BFA0
:108810002DE9F041436903F5A0430746D3F8C46D41
:10882000D3F8C08DEEB1046A0025033414F8023C7D
:1088300014F8031C14F8012C1B0203EB01431A4427
:10884000294630461BF046FA2946304601351BF0D2
:108850002FFAB5F5807F04F10304E7D197F82530AE
:108860003BBBF9683868B8F8042043189342D7E94D
:1088700001342344B8F80640C8BF111AA34216DADF
:10888000904214DA002912DDB8F80C2002FB03F341
:10889000D8F8082002EB8302BB6986B10244013A92
:1088A000194413F8010B02F8010F8B42F9D1BDE80E
:1088B000F08197F8241030461BF004FAD1E702EB60
:1088C000400297F82500FC69012809D0194413F8E3
:1088D000010B34F8100022F8020B8B42F7D1E6E7C7
:1088E00097F82450194413F8010B85421CBF34F843
:1088F000100010808B4202F10202F4D1D7E700BFD2
:108900002DE9F04100F5A04882B098F8AE1D426B09
:1089100001238DF80730036B51BBD11A4C1E40F276
:10892000F942944224D833BB044640F2FA4600F19F
:10893000540514E0636BB3421ADC236C9847616BF7
:10894000236C9DF8072001F5BD51143121442846C0
:108950009847636B9DF8072013446363D2B1D4E951
:1089600015739F424FF001020DF107012846E1DB2C
:1089700002B0BDE8F08100F5BD5213321344551822
:1089800013F8014F02F8014FAA42F9D10023C0E9C0
:108990000C31C9E7012388F8AE3D02B0BDE8F08193
:1089A00070B500F5A042002382B0436582F8B43D63
:1089B00082F8AE3D826D4FF0FF310B2AD8BF5218BE
:1089C000C0E90831C8BF0C22036C019200F5DA71CE
:1089D000044654309847019A824227D1184905220B
:1089E00004F5DA703CF072F930B11649052204F54D
:1089F000DA703CF06BF900BB94F8BE31B4F8BA11F0
:108A0000B4F8BC212160C3F302130133C4E901218E
:108A1000E260A3610146626C04F154009047A368D0
:108A2000B3F5A07F07DC012002B070BD0623002053
:108A3000E36102B070BD0223F9E70823F7E700BF46
:108A4000281C0B00301C0B0041F2167C614500F223
:108A500076812DE9F04F00F58D5A0AF1140A00F5E0
:108A6000ED5700F59B460368856A91B00E372E36A8
:108A700000F5DA7E5446A64500F0BD80725C04F82D
:108A8000012D37F811106145F5D95B1B00F1740811
:108A9000BAEB0407434400F0AE80C16A00F5A5526A
:108AA0001432039200293A46054647464FF0000B20
:108AB00000F5A046904640F39A80A86A404500F32E
:108AC0002E811A1893420BD2013B04EB000C14F8D0
:108AD000012B03F8012FA445F9D1D5E90A01644619
:108AE0002A682B69AA6202930593A8EB0008039BEE
:108AF00096F8B40D0B9700280CBFD1469946089202
:108B0000D5F804C096F8B3EDCDF824C00138CDE90E
:108B10000C9918BF01208DF83C00D5F81490CDF8C1
:108B20001890ACEB01011EF0400F07910CD00CF136
:108B3000FF3000EBD07EB1EB6E0F40F3B58040F01C
:108B40000100C0EB4100079096F8AF0D96F8B11DFB
:108B500096F8B03D01934FF0000E00F0010C61F368
:108B6000070EC0F382006CF30F2E60F3174E63F311
:108B70001F6ECDF838E0D5E9193E0A93BEF1000F1B
:108B800023D0079B02999944AB68022803FB091381
:108B90000EEB830332D0BCF1000F3AD0002A0FDD78
:108BA0009DF838C0394611F8010B844518BF18707C
:108BB0000898A1F17402521B904203F10103F2DC08
:108BC00096F8B6EDBEF1010F2CD0AB6C05A8984716
:108BD000E96A013911F0030FE96208BF4BF0010B9C
:108BE000B8F1000F03D000293B463FF766AFBBF159
:108BF000000F40F08E8011B0BDE8F08F184601994B
:108C00003CF05EFA9DF839C0089A0346BCF1000FAB
:108C1000C4D1184639463CF06FF896F8B6EDBEF16F
:108C2000010FD2D1DDE906329918AA68059BE868E0
:108C300096F8B5CD02FB0131AB6E00FB02F2BCF140
:108C4000010F03EB81010C9803EB82032A6850D9D2
:108C5000002A27DDCDE9017403334FF0000C4FF0FB
:108C6000030911F8012B02EB42070333C75D03F838
:108C7000067C12FB09E70224C75D03F8057C12FBA2
:108C800009420CF1010C825C03F8042C2A6894451B
:108C9000E7DBDDE90174D5E9023203FB02F2AB6EDA
:108CA00003EB82030B9390E700288646B8BF0CF1D4
:108CB000020EB1EBAE0F07DD20F0030040F0020022
:108CC000C0EB810107913FE700288446B8BF00F15F
:108CD000070CB1EBEC0F4FEAC10E07DD20F00701E6
:108CE00041F00401AEEB010107912DE7CDF81CE046
:108CF0002AE7002AD6DD4FF0000C11F8012B30F8DE
:108D0000122023F8022B2A680CF1010C9445F4DBA5
:108D1000C1E7284611B0BDE8F04FFFF7F1BD474667
:108D2000DA19934208D2013BE11914F8012B03F838
:108D3000012FA142F9D1A86AC01BA86257E770476A
:108D400030B5D0E900431B1B9342B8BF03F1FF329B
:108D500083B012B9104603B030BDC36805461C4647
:108D600003F1080001AB82F091FB20B9236C01985C
:108D70002B6003B030BD052078F006F938B5C56822
:108D800004460A46CB1705F1080082F00BF8286C60
:108D9000206038BD10B545F6B8520C4600213CF0B5
:108DA0008FF900F5A04383F8B54D10BD2DE9F04FC4
:108DB0000646436C856D87B00F465430002106F59A
:108DC000DA749847336C4FF48052214606F1540010
:108DD000984796F9BE1196F8BE2100290346A5EBE7
:108DE0000005C0F2F0804FF00D094FF0000E42F286
:108DF0001072CDE901E24FF0020BF2461A460397DA
:108E00000BF1FF339145049329DA4846171AB7F559
:108E1000817F034604EB000131DB09782C2942D025
:108E20003B291CD021291AD12344811C5F789878D2
:108E3000F92F00F0FD800844231802305F7867B1F5
:108E400001460F44791CE75DA2EB010907F201130B
:108E50004B455FDA002FF4D108469042D6DB039FE2
:108E6000D646ABF1020C019BBB60029BC7F800C069
:108E70000120FB60C7F804E007B0BDE8F08F3A4678
:108E800020463BF06DFF336CC7F58052E11906F1C7
:108E90005400984721463A1809782D1A2C294FF08A
:108EA00000000346BCD19042D9DA234400F10A09FC
:108EB00093F909105B7A002953DB09F1010103F2F0
:108EC0000113571ABB4239DA631809F102091F78F6
:108ED0007FB14946A946B1F5406F6EDDB9F1000F8B
:108EE00007EB01034DDCE75C591C002FF6D14D4622
:108EF000894614F809303B2B04EB090100F0B580DA
:108F0000002D6CD1A2EB09031F2B40F3AE800BF1B7
:108F1000010B75E74A46214420463BF021FFC9F585
:108F2000805204EB0901336C06F15400984700218C
:108F300009EB00022D1A002F83D18DE78A426BDCEA
:108F4000891A01F1010963184FF480522146002764
:108F5000059306F15400336C9847059B3A182D1A77
:108F6000B5E703F00703022199404FF0030011FB1E
:108F7000009909F1010103F20113571ABB42DDDA2E
:108F8000A2E7551A2A46214420463BF0E9FEC5F5E2
:108F900080524A45A8BF4A46336C611906F1540015
:108FA0009847E35D2A18A9EB0009791C002B9ED095
:108FB0000B44591CE75C002F99D00F44791CE75DE6
:108FC000002F88D193E702F007024FF0020909FA57
:108FD00002F94FF003010D2219FB012905E7B36DDA
:108FE000B3F5805F93DD002D91DDA2EB09094A46C0
:108FF00020463BF0B5FEC9F58052AA42A8BF2A46DA
:1090000004EB0901336C06F15400984709EB0002A8
:109010002D1A4FF000097AE721443A4620463BF0EA
:109020009FFE4FF00109E119C7F5805223468FE7F3
:1090300004287FF400AF1F795B7947EA0323022BF2
:10904000B8BF0223019F03EB8303B7EB430F0AEB87
:10905000430A4FEA430C02DACDF804C0EBE6029B68
:109060006345A8BF63460293E5E6DDF810C0039FA1
:10907000D646F8E6FFF794BC2DE9F04F8BB00446D6
:109080000491934609B100230B60D4E915735A1E6D
:10909000974227DA04F15402009204F5A04100221D
:1090A00081F8B42D81F8AE2D22624FF0FF3262625A
:1090B00007F1FF029A42C6BFDB1B03F1FF394FF0F5
:1090C000FF0904F5DA750591236C00984A46294694
:1090D0009847814506460ED00623E36100200BB079
:1090E000BDE8F08F636C04F15400002100909847B4
:1090F000D4E91573D1E7002F00F0978000212B46AB
:1091000089461A782C2A22D0DA46B3463B2A00F048
:10911000E581212A40F0E78105EB090209F1020807
:109120005278FE2A00F0F980FF2A00F0A980012A77
:109130006FD0F92A40F0EE8015F80820042A00F0DC
:1091400055814146C1462C2AE0D15E46D34629448A
:1091500005EB090388785A7802EB0022226108792E
:10916000CA7802EB0022626188794A7902EB002218
:109170002260087ACA7902EB002262605B7A059A63
:1091800082F8B33D1A0609F10A0800F16381059AD5
:1091900015F8083082F8B23DAA4A0297D35CA36161
:1091A000002308F10101009F636341F2B478AA46ED
:1091B000CDF804B009E03BF09FFD626B0BEB0501BD
:1091C0002A446263002D00F0C382B14201F1010B19
:1091D00080F291811AF80150606BA6EB0B094044B4
:1091E0004D4520442A460AEB0B01E4DD4A463BF09C
:1091F00083FD616B236C49446163A5EB090941441C
:1092000021444A4638469847636B314609EB0302CE
:10921000D7E715F8083008F101089844002BF8D179
:1092200015F808204146C1468DE7874905222846A2
:109230003BF04CFD38B18549052228463BF046FD00
:10924000002840F0EE8094F8BE31B4F8BA212260D4
:10925000A260C3F302120132A2610599B4F8BC21E5
:109260006260E26094F8BF2181F8B02D1A0681F89F
:10927000AF0D00F181800D2104F2C113894640E752
:109280005B46A34615F8086008F10109A3EB090441
:1092900006F11F02A24227DA09EB06080B2E08D0BE
:1092A000002EEFD15C4615F808209B464146C1468A
:1092B00049E7A94466490193324648463BF006FD1A
:1092C000019B0028DED199F80B20032ADAD199F806
:1092D0000C20012AD6D199F80E1099F80D2002EB36
:1092E0000122CBF82420CDE708F2B51159442246DB
:1092F00028463BF035FD04F5DA71DBF84030009884
:10930000594406F1200298474F4423184FF00009B2
:10931000B046C3E70123E361E0E64146A1466C5C49
:109320004E1CABEB060804F11F0343450EDA31195E
:10933000D9F838303E441BB9C9F83860A9F83C4028
:10934000002CECD14C466A5C8946FCE601F2B51172
:109350004944424628463BF003FD08F5DA7149448A
:10936000D9F84030009804F120029847374408EBC0
:10937000000B00262146DBE703F0070303F1010899
:109380004FF0030906F5DA7109FA08F9236C009821
:1093900021444A469847059B064493F8B50D012899
:1093A00042D804F58D514FF0020C12310CFA08FC32
:1093B0008C44224692F8C23192F8C1E19B084FEAF0
:1093C000DE0E5B0143EACE2392F8C3E1033243EAA7
:1093D000DE0300B15BBA21F8023F6145EAD1032107
:1093E00001FA08F10D3189466B188AE62944059B7C
:1093F000C87883F8AF0D4E790A7902EB062202EBAA
:1094000082025200012AD8BF64222262C00744BFF0
:109410008A7983F8B12D09F10809494615F8092020
:1094200091E60823E36159E604F58D504A4604F2BB
:10943000C11109F10D0914303BF05EFC494605EB02
:1094400009035EE620760C00281C0B00301C0B0084
:10945000E0190B0003F00703013306F5DA7103226C
:109460009A4001932144236C009802929847059AF0
:1094700092F8B51D029A0129064404F5A55000F2A0
:109480007781019A02239340123003EB000E0123EF
:1094900003FA02FC04EB090292F8BF3192F8BE8194
:1094A0009B084FEAD8085B0143EAC82392F8C081C1
:1094B000033243EAD80301B15BBA20F8023F864584
:1094C000EAD10CF1FF3303EB430309F10D0903EB80
:1094D0000908059A012382F8B43D58E60723E361A1
:1094E000C4F864A0FAE5A36DDB1B1F2B3FF712AF96
:1094F0000723E361F2E5DDF804B0E369C4F864B082
:10950000072B3FF4EBAD059B93F8B23D4FF6FF768A
:1095100001339E4004F5BD53143336B203936368A0
:10952000E3626FEA66062368A362B31C9BB20193F1
:1095300004F5ED530E330025721C069304F57653A3
:109540001FFA82FA2E33256320460293FFF7D8F9DB
:10955000BAF1000F14D02B4604F5ED5004F5765502
:1095600004F59B412D350C302D3141F2187701F86F
:10957000013F05F8013F0133534520F8027FF6D142
:10958000CAF580535B000993069BCDF800A003EB5E
:109590004A03F51C08930026A246059B099A93F8F6
:1095A000B28D08984FF6FF7308F1010941F2177167
:1095B00008F1010803FA09F93BF082FDDAF83000FE
:1095C000039BC8F12002B242B8BF00EBE60003EBF8
:1095D0000001B8BFCAF830001F5C4878009B07EB59
:1095E00000278878C97807EB0047B8BF06F0070660
:1095F0000FFA89F907EB016727FA06F16FEA090903
:1096000009EA010189B28B42464400F0818050464C
:109610000791FFF719FA019B07998B4200F0A6808A
:109620004FF0010B0BFA08FB534644461FFA8BFB25
:1096300007951FFA85FA98462EE0DA4515D2069B63
:10964000029A23F81A10515C02F80A1033F815E058
:1096500041F217739E4518BF029B0AF5805C16BF46
:10966000595D02F80C1003F80C100AF101031FFAFF
:1096700083FADA450BD30B2C09D8621C4FEA4B0B4B
:109680004FEA490994B21FFA8BFB49F001092946B8
:109690004046FFF7D9F92946D8F82C50002D27DD90
:1096A000C4F12005B54217DAD8F83050039B05EB1A
:1096B000E60503EB050CC8F830505F5D9CF80150DF
:1096C00007EB05279CF8025007EB05479CF8035071
:1096D00006F0070607EB056727FA06F5009B09EA7F
:1096E0000505ADB2AB4226442FD0019BAB42A4D1BD
:1096F0004446049B13B1049A236A1360D4E915030A
:10970000013B9842ACBF002001200BB0BDE8F08FB8
:10971000B24213DADAF83020039B02EBE602991822
:10972000CAF830209F5C4A7807EB02278A7807EB5B
:109730000247CA7806F0070607EB026727FA06F128
:1097400009EA010189B2464461E7079DC24624E760
:10975000059A01238E42DDE901B782F8AE3D7FF71D
:10976000CCAE0098636C39449847C6E65446C0E7CF
:1097700005EB0801143001923BF0BEFA019A9044C7
:10978000A7E600BF2DE9F04F0022164689B06C4BCA
:109790006C4C6D48CDE9022235460122196841B171
:1097A000D4F80413114204D01D6019680091009987
:1097B0001643043383424FEA4202EFD1614BD3F8A0
:1097C0007C21F1B2002A6ED00022C3F87C21D3F8AC
:1097D0007C3101934FF0A042019BD2F810255B4BE6
:1097E0000292D3F81035039300297DD10DF1100AB0
:1097F00000224FF0FF33564DDFF850810492CAF833
:1098000004200693534C07934FF0000B14F9013FCB
:109810005F1C31D0C3F3C20E0EF120020DEB020C1F
:1098200003F007021CF8086CD640F607D9B203F023
:109830003F0021D5484F3E18890996F9286057F80E
:109840002660002E5BD003295BD01F2887BF03F062
:109850001F03C64603464FF0A04E1CF818CC0EEB73
:1098600083032CFA02FCD3F800271CF0010FC2F38B
:1098700001423CD0022A4FD0A542C7D1BBF1000F14
:109880002FD04FF0A0430299D3F81035D8F8102507
:10989000994202D10399914223D0CDE90232DDE908
:1098A00004230692AEE7D1B12B4F01250024A3007B
:1098B00003F180432E4203F5C0430BD0D3F81005CB
:1098C00057F82420D3F81015C0F30520C1F3014147
:1098D00002B190470134082C4FEA4505E7D1002E2C
:1098E00084DB09B0BDE8F08F46F00046DCE7032AD0
:1098F000C2D1032921D0002EBED0B047BCE7032936
:10990000BAD11AF80E704FF0010909FA02F947EAC4
:1099100009090AF80E9098E70329ECD14FF4403C6E
:10992000D3F8002722F440320BF1010B42EA0C027B
:109930005FFA8BFBC3F80027DDE74FF4003CEFE74D
:1099400000610040006000402061004000030050C2
:10995000B1110120AF1101205811012008B50420D8
:1099600065F000FC2DE9F04FD1F80031103B102BD1
:109970008BB0064600F25681AC4A22FA03F313F08C
:10998000010F14BF8A464FF0000A91F804C1351D3B
:109990004FEA0C1C06F114092C46231F0CEB0A009D
:1099A0001A7810F8017B7A4003F8012B9C42F7D11A
:1099B0000434A1450CF1040CEFD191F80431013BC2
:1099C00006F11002DBB20492AC469A00B6469EF84D
:1099D0000D309EF809609EF805509EF801409EF8F3
:1099E00002109EF80A008EF80D608EF809509EF85D
:1099F0000E609EF806508EF805408EF801309EF8F5
:109A000007409EF803308EF802008EF80A109EF888
:109A10000B009EF80F108EF80B108EF806608EF873
:109A20000E508EF803408EF807008EF80F30714606
:109A3000002311F823007E4C205C01F82300013341
:109A4000042BF6D101318C45F2D1960065462B1FCF
:109A50000AEB0600197810F8014B614003F8011B6E
:109A6000AB42F7D11D1DA94506F10406EFD1002A2E
:109A700000F0D580CDE905A9CDE907C2F346CDF8C0
:109A800024E09BF803E09BF800A09BF801809BF882
:109A900002904FEADE164FEADA1706EB460606EBAF
:109AA000C60607EB470786EA4E0007EBC70787EABB
:109AB0004A074FEAD815C0F3C01CC7F3C01205EB24
:109AC00045050CEB4C0C4FEAD91405EBC50502EB30
:109AD00042020CEBCC0C85EA48058CEA400C009065
:109AE00004EB44048AEA080002EBC2028AEA090A8B
:109AF00082EA47028EEA0A06C5F3C01304EBC404E7
:109B000084EA490488EA0908029689EA00098EEA8B
:109B1000000603EB4303C2F3C01003EBC30300EBE7
:109B2000400083EA4503C4F3C01100EBC00080EAA3
:109B300042008EEA08085FFA87FAC3F3C01E574056
:109B400001EB4101474001EBC1010EEB4E0E81EAF2
:109B5000440101970EEBCE0EEFB28EEA430E8AEA75
:109B6000090A87EA08075D40C1F3C018DBB283EA3F
:109B70000A0308EB4808434008EBC80888EA410894
:109B800003968EEA0303029E5FFA84F988EA030AC9
:109B9000009B89EA06094C40039EC9B27940DFB2B6
:109BA0007740D2B27A405FFA8CF787EA09074240E1
:109BB0007840CCF3C01707EB47078EEA010107EBAB
:109BC000C70787EA4C0783EA0C0688EA0101019B74
:109BD0008EEA020288EA0000794078407A407740B5
:109BE00059408EEA05058AEA070388EA04048BF8DF
:109BF00003306840049B8BF8001062408BF8010032
:109C00008BF802200BF1040B9B457FF43AAFDDE9A2
:109C100007C2DDE905A9DDF824E0043AD7E60BB078
:109C2000BDE8F08F4FF0000AAFE600BF0101010070
:109C3000CC2B0C002DE9F04F89B0129E002800F0CB
:109C400047820F4609681D46904682467FF0EAFD2E
:109C5000B0F10009C0F201823968494439605046C8
:109C600080F084FA021EC0F27682396811443960AD
:109C7000D8F8000009EB020CA0EB0C00C8F80000BB
:109C8000DAF8B817DAF8B037002956D1002B55D1D9
:109C90000121CAF8B017D8F80010D7F800E0012960
:109CA000CDE903E9AEEB0C0C704622DD01F1FF3B80
:109CB0004FF0000E03E00EF1010EDE4519D0044610
:109CC00010F8019BB9F1FF0FF5D194F8019009F05C
:109CD000E009B9F1E00FEED19CF80000FF2800F098
:109CE000C5800EF1030EA1EB0E01012904F1030062
:109CF000DCDC4FF0FF32DAF8C817DAF8C4C7CAF86C
:109D0000B4270CFB01F2DAF8BC1701FB02F2002ABF
:109D100010DDA91E002021F8020FDAF8C847DAF892
:109D2000C42704FB02F2DAF8BC47013304FB02F259
:109D30009342F0DB6FF0020095E04BB1DAF8B447E4
:109D400050467CF09FFC2044CAF8CC07D8F80000AD
:109D5000002E00F0BA80DAF8D827CAF8CC07002A1B
:109D600040F05D81904240F35A81CAF8DC073E68BA
:109D700030443860D8F80020DAF8CC17521AC8F806
:109D80000020DAF8C41700229142079240F345817F
:109D9000DAF8DC4703924FEAC4080AF2DC77D146CE
:109DA0002C46D9F8BC27002A40F3BD80DDF81CA062
:109DB0000597BB460025374604945646DDF80CA0AF
:109DC00020E05BF8043F43452BDC079F01953E44B0
:109DD0009B1BCDF800A048467CF060FC0028C7EB38
:109DE000C003D9F8BC17A8EB060805F1010504EB80
:109DF0000007C0F2D680079E8D423344A8EB0308CB
:109E000080F28E8007AA3946CDE900A54346484630
:109E10007FF0F8FD041EC6EBC4063C4407AA2146A9
:109E2000CFDAD9F8C427D9F8C807D9F8BC17049DE8
:109E300000FB02F201FB02F2002ACA4611DD0021FA
:109E4000A81E0E4620F8026FDAF8C437DAF8C847C1
:109E5000DAF8BC2704FB03F3013102FB03F3994258
:109E6000F0DB6FF0070009B0BDE8F08F94F80190C7
:109E70009CF8010081457FF434AF9CF802B0A078D3
:109E80008BEA000003283FF62CAFDDE903E91BF065
:109E9000020F18BF04F1FF34A4EB0E04DAF8C81760
:109EA000DAF8C4C7CAF8B447002C0CFB01F0FFF67F
:109EB00028AFDAF8C017A1444A4401FB02F2D200ED
:109EC00092FBF0F2CAF8B8273AE7DAF8CC478442B6
:109ED00000F32181DAF8DC17DAF8D8279142C0F2D2
:109EE000BF80891A0AF11C06314430463AF038FF27
:109EF000DAF8D807DAF8CC27396830443AF0FCFEB3
:109F0000DAF8CC17DAF8D8270A44CAF8DC273A6816
:109F10000A443A60D8F80020DAF8CC17521A2EE733
:109F20003E46DDE90447039948467DF0D5F8002810
:109F3000D9F8BC27C0F2CF80002A55DDDDF80CA08F
:109F4000002501E095424FDA2A46514648467DF009
:109F5000FFFD0028D9F8BC2705F10105F2DAD9F890
:109F6000C417D9F8C80700FB01F101FB02F2002A6F
:109F7000CA4611DD0021A01E0D4620F8025FDAF866
:109F8000C827DAF8C43702FB03F3DAF8BC2701313B
:109F900002FB03F39942F0DB6FF00A0009B0BDE861
:109FA000F08FD9F8C427D9F8C807049D00FB02F246
:109FB00001FB02F2002ACA4611DD0021A81E0E464E
:109FC00020F8026FDAF8C437DAF8C847DAF8BC27A5
:109FD00004FB03F3013102FB03F39942F0DB6FF062
:109FE000080009B0BDE8F08FD9F8C817039B03FB40
:109FF00001F102FB01F104EB410148467FF08AFBCD
:10A000000028D9F8C427C0F2C780039B01339342CC
:10A01000039307F10807FFF6C4AE002023E7DAF840
:10A02000C427DAF8C807DAF8BC1700FB02F201FB14
:10A0300002F2002A11DD0021A81E0C4620F8024F72
:10A04000DAF8C827DAF8C43702FB03F3DAF8BC27DA
:10A05000013102FB03F39942F0DB6FF0050002E7E8
:10A060000AF11C002246084439683AF045FEDAF845
:10A07000CC17DAF8DC270A44CAF8DC273A680A4425
:10A080003A60DAF8CC17D8F80020521AC8F8002045
:10A09000DAF8C817DAF8C42701FB02F2DAF8BC17BD
:10A0A00001FB02F2002A10DDA91E304621F8020F42
:10A0B000DAF8C827DAF8C43702FB03F3DAF8BC276A
:10A0C000013602FB03F39E42F0DB6FF00100CAE6AB
:10A0D0006FF00400C7E6D9F8C417D9F8C80700FB29
:10A0E00001F101FB02F2002ACA4611DD0021A01E87
:10A0F0000C4620F8024FDAF8C827DAF8C43702FB1A
:10A1000003F3DAF8BC27013102FB03F39942F0DBD9
:10A110006FF00900A7E6DAF8C817DAF8C42701FBE0
:10A1200002F2DAF8BC1701FB02F2B24210DDA91EFE
:10A13000304621F8020FDAF8C827DAF8C43702FBF4
:10A1400003F3DAF8BC27013602FB03F39E42F0DB8F
:10A150004FF0FF3087E6DAF8C827DAF8C407DAF8F4
:10A16000BC1700FB02F201FB02F2002A11DD002104
:10A17000A81E0C4620F8024FDAF8C827DAF8C437D0
:10A1800002FB03F3DAF8BC27013102FB03F3994227
:10A19000F0DB6FF0060066E6D9F8C807D9F8BC17FF
:10A1A00000FB02F201FB02F2002ACA4611DD002187
:10A1B000A01E0C4620F8024FDAF8C827DAF8C43798
:10A1C00002FB03F3DAF8BC27013102FB03F39942E7
:10A1D000F0DB6FF00B0046E6012913DD821E431E03
:10A1E000114401E08B420DD09C4613F8012FFF2A49
:10A1F000F8D15A7802F0E002E02AF3D1C0F1010070
:10A20000604470474FF0FF30704700BF08B17DF0E9
:10A21000F1BB704788B338B50D46114604467FF050
:10A2200001FB013026D0D4F8D037032B22D1D4F84B
:10A23000B8372B60D4F8BC376B60D4F8C02710490E
:10A240001023C5E9022394F8D437D4F8D02703EBC0
:10A250004303013A1344D4F8BC2731F9133002FB0D
:10A2600003F32B61D4F8D0376B6194F8D437AB612A
:10A27000002038BD6FF0050038BD6FF00400704756
:10A28000886C0C007CF0ACB910B54FF0804386B000
:10A29000D3F80443620703D5D3F80821002A62D11A
:10A2A000A30605D54FF08043D3F81421002A4FD1DF
:10A2B000600605D54FF08043D3F81821002A3BD122
:10A2C000210604D54FF08043D3F81C214ABBE20598
:10A2D00004D54FF08043D3F82021B2B9A30512D59D
:10A2E0004FF08043D3F824216AB10022C3F824211F
:10A2F000D3F82421214B0592059A1B68022006B051
:10A30000BDE81040184706B010BD0022C3F8202158
:10A310001A4AD3F82031049301201368049A98470D
:10A32000DCE70020C3F81C01144AD3F81C31039366
:10A330001368039A9847CAE70022C3F81821104A05
:10A34000D3F81831029301201368029A9847B7E7AF
:10A350000020C3F814010A4AD3F81431019313689A
:10A36000019A9847A4E70022C3F80821054AD3F8C8
:10A37000083100931368009A984791E738700120DC
:10A380003470012030700120064BD3F800213AB11F
:10A39000054A00205071C3F80001136891681847FE
:10A3A000704700BF00900240107001200248032255
:10A3B000002135F0D9B900BF00B0004002480422A6
:10A3C000012135F0D1B900BF00100140024804223C
:10A3D000022135F0C9B900BF0040024008B50F4A5C
:10A3E0000F4B934208D2013AD21A22F003020D49D0
:10A3F000043218463AF080FC0B4A0C4B934208D2C8
:10A40000013AD21A22F003020432002118463AF02F
:10A4100057FE00F0FBF86BF059F800BFAC060120C6
:10A4200000000120807E0C002C7B0120C006012052
:10A430000149024876F01AB84C6F01200030004004
:10A4400002494FF0402076F011B800BF806F012024
:10A450001D4BD3F8182102B9704700B500211B4AE3
:10A4600083B0C3F81811D3F8181192F82030019175
:10A47000FF2B01990FD0917F69B9D17FB1B11F2B0B
:10A4800086BF134803F01F034FF0A040012101FADB
:10A4900003F3C0F80C35D2E900E100230D485377EF
:10A4A0001372734603B05DF804EB18471F2B86BF89
:10A4B000074803F01F034FF0A040012101FA03F306
:10A4C000C0F80835E7E700BF00300240EC6E01201D
:10A4D00000030050F46E01201F4BD3F8182102B97D
:10A4E000704700B500211D4A83B0C3F81811D3F896
:10A4F000181192F844300191FF2B019911D092F874
:10A50000421071B992F84310C1B11F2B86BF144895
:10A5100003F01F034FF0A040012101FA03F3C0F83C
:10A520000C35D2E909E100230E4882F8413082F867
:10A530002C30734603B05DF804EB18471F2B86BF21
:10A54000074803F01F034FF0A040012101FA03F375
:10A55000C0F80835E5E700BF00F00240EC6E0120CE
:10A5600000030050186F012070B5234C82B0022602
:10A57000002501A865F07EFF05280BD0019B032B69
:10A580002CD01ED8022BF4D101A8257065F072FFE3
:10A590000528F3D1194E4FF40C751948ADF8025047
:10A5A0000DF1020165F0F2FEE0B9D6F8B440002CDE
:10A5B000F3D0D4E90112246811489047002CF8D157
:10A5C000EBE7A3F10902022AD3D80A2B08D0092B02
:10A5D00014BF0120022075F015FECAE72670C8E7F7
:10A5E0000020F8E70C2801D002B070BD05490648EC
:10A5F0004AF054F902B070BD187B01204070012070
:10A60000BC6C0120E8170B0048440B0008B54FF064
:10A610008053D3F83021082A1FD0754AD2F88830E9
:10A6200043F47003C2F88830BFF34F8FBFF36F8FCE
:10A630004FF01023D3F80C22D20700F1BB80D3F8DF
:10A640000022002AC0F29080D3F80432002BC0F21E
:10A650008B80684B684A1A6008BD4FF0804000212B
:10A66000C0F80C11654AC0F81011C0F83815D3F8BD
:10A670000414C2F82015D3F80814C2F82415D3F82E
:10A680000C14C2F82815D3F81014C2F82C15D3F8FE
:10A690001414C2F83015D3F81814C2F83415D3F8CE
:10A6A0001C14C2F84015D3F82014C2F84415D3F88E
:10A6B0002414C2F84815D3F82814C2F84C15D3F85E
:10A6C0002C14C2F85015D3F83014C2F85415D3F82E
:10A6D0003414C2F86015D3F83814C2F86415D3F8EE
:10A6E0003C14C2F86815D3F84014C2F86C15D3F8BE
:10A6F0003411D3F844C4C2F870C5F1B151B14FF070
:10A700008043D3F80024D10787D56FF00102C3F846
:10A71000002482E74FF08053394AD3F830314FF4A8
:10A720000071082BC2F840167FF477AF4FF08043DA
:10A73000D3F80024D107E8D46FE7A2F5E042DFF8B0
:10A74000C8C0C2F88CC602F520424FF0FB0CC2F81C
:10A7500018C5D0F8E42ED3F8583263F30302C0F8DA
:10A76000E42E0029D6D0CAE7264A0123C2F80435D0
:10A77000D2F80034002BFBD04FF010231221214AD5
:10A78000C3F80012D2F80034002BFBD04FF0102396
:10A7900012211C4AC3F80412D2F80034002BFBD05B
:10A7A00000231849C2F80435D1F80034002BFBD03F
:10A7B00001F036FB134A0123C2F80435D2F8003405
:10A7C000002BFBD04FF010210E4AD1F80C3223F0B1
:10A7D0000103C1F80C32D2F80034002BFBD0002367
:10A7E0000849C2F80435D1F80034002BFBD0DFE76C
:10A7F00000ED00E0000001200090D00300C0004008
:10A800000090024000E001404881030001490248F5
:10A8100035F002B8346F0120009000400149024831
:10A8200034F0FABF406F012000A000400149024807
:10A8300076F032B9B46F012000200040014902488F
:10A8400076F02AB9D86F012000800240002078F00D
:10A8500003BC00BF094BD3F8002172B100B5084A10
:10A8600083B052689047054B0022C3F80021D3F80B
:10A8700000310193019B03B000BD7047000001400F
:10A8800008700120022A2DE9F0431ED0444C02EB4F
:10A89000C20204EB021404F1480601F144058C34B1
:10A8A00000F1240750F8043B54F804C956F804EBAF
:10A8B0001A468EFB028241F8042B8CFB0323B8421C
:10A8C00045F80439EED1BDE8F083354B8268D3F802
:10A8D00038C18CFB02428469D3F8205185FB0464A3
:10A8E00022440A60D3F83C71426887FB0242C46983
:10A8F000D3F8245185FB046422444A600268D3F8EB
:10A90000406186FB0242056AD3F8284184FB05E5D5
:10A910002A448A600268D3F84491964689FB0E2E39
:10A92000026AD3F82C4184FB02827244CA604268F6
:10A93000D3F848E18EFB0242C469D3F8305185FB5D
:10A94000048422440A618268D3F84C8188FB024265
:10A95000D3F83451836985FB03431A444A61436940
:10A960008CFB03238B61036987FB0323CB61C368E3
:10A9700086FB03230B62C36889FB03234B620369D5
:10A980008EFB03238B62426988FB02320023C1E9FC
:10A990000F33C1E90D33CA624B640B63BDE8F0832A
:10A9A000E0730C002DE9F047B0F85E300446002B50
:10A9B00071D0434E434D0F46904646F001064FF08E
:10A9C000000A4FF0010994F8622072B30AF00F03F5
:10A9D0004FF40041194101EA0801002313E01F2A46
:10A9E00086BF02F01F0228464FF0A04009FA02F28B
:10A9F000C0F8082594F862200133DBB202EB420272
:10AA0000B3EB420F0FDA2269D25C0029E7D11F2A8B
:10AA100086BF02F01F0228464FF0A04009FA02F25A
:10AA2000C0F80C25E6E7B4F85E30DB1B53450CDAC2
:10AA300094F834301F2B86BF03F01F032A464FF0D3
:10AA4000A04209FA03F3C2F8083594F861301F2BCD
:10AA50008ABF2A464FF0A04203F01F0309FA03F30E
:10AA6000C2F808354020B04794F861301F2B8ABFE8
:10AA70002A464FF0A04203F01F0309FA03F3C2F87D
:10AA80000C354020B0470AF1010AB4F85E301FFAD5
:10AA90008AF2934297D894F834201F2A07D84FF0AF
:10AAA000A04101239340C1F80C35BDE8F08705496A
:10AAB00002F01F0201239340C1F80C35BDE8F08776
:10AAC000407C0C0000030050054B18680368D3F865
:10AAD000402112B10022C3F8402100F03DBF00BF69
:10AAE00008120120002800F05E822DE9F843044698
:10AAF0000069002800F01A8294F8613094F862101E
:10AB00001F2B8CBFDFF82CC34FF0A04C002900F0A6
:10AB1000F2810FFA81F901EB410149000022C54E93
:10AB2000884615464FF0010E01E08A4213DA835C35
:10AB30001F2B88BF374603F01F0398BF4FF0A04775
:10AB400001320EFA03F3BC45D2B245EA0305ECD05C
:10AB50000120BDE8F883B5F1807F34BF00230123D5
:10AB6000DB0015F47F0F43F0040218BF134615F401
:10AB70007F4FEAB200F0DF81002A00F0B18143F09C
:10AB80000303012202FA03F341F20802134200F028
:10AB9000B48109EB4902022302FA03F81A4694F839
:10ABA0006310B4F85E6084F8603001238B40073690
:10ABB00006F4FF6684F86630DBB216FB03F694F801
:10ABC000653003FB06F694F8683002FB06F6E6648F
:10ABD00003B17600012108EB060060F023FE6062FD
:10ABE000002800F0A38183193246636100213AF006
:10ABF00067FA94F8610094F8603094F8626001217B
:10AC000000F01F0201FA02F28B4245EA020500F051
:10AC10009781022B00F0C981C4E90625002284F83F
:10AC200064209EB1D4E904359B5C03F01F0301FA54
:10AC300003F345F8223094F86230501CC2B203EBA3
:10AC40004303B2EB430FEDDB94F8610094F86530F9
:10AC500094F8341094F8665001229A40013A4FF467
:10AC60007A43B3FBF5F3B3FBF2F3642B38BF6423F1
:10AC70001F29C4E914338CBF6E4B4FF0A043002250
:10AC800084F86A2003F5A162A26201F01F0101228B
:10AC900002FA01F194F8442003F20C531F2AC4E98C
:10ACA0000B318CBF634B4FF0A04302F01F0103F543
:10ACB000A16503F20C5203461F2B4FF0010000FA6E
:10ACC00001F188BF03F01F03C4E90F2103F5E0730E
:10ACD00088BF584AA56398BF4FF0A04240F20331A5
:10ACE00042F8231094F861201F2A86BF02F01F0249
:10ACF00050494FF0A04101239340C1F80C3594F81E
:10AD000034301F2B86BF03F01F034A4A4FF0A04286
:10AD100003F5E07340F2033142F8231094F8342035
:10AD20001F2A86BF02F01F0242494FF0A0410123B3
:10AD30009340C1F80C3594F844301F2B86BF03F0C4
:10AD40001F033C4A4FF0A04203F5E07340F2033189
:10AD500042F8231094F844301F2B86BF354A03F085
:10AD60001F034FF0A042012606FA03F3C2F808358C
:10AD700094F862303BB32F49002340F20337226935
:10AD8000D25C1F2A88BF02F01F020D4602F5E07256
:10AD900098BF4FF0A0454FF0A04045F822702269BF
:10ADA000D25C1F2A84BF02F01F02084606FA02F294
:10ADB000C0F80C2594F862200133DBB202EB4202AA
:10ADC000B3EB420FDBDB47F6FF720C212046FFF7A7
:10ADD000E9FD40220D212046FFF7E4FD94F86230A2
:10ADE000C3B11449002301252269D25C1F2A0846F9
:10ADF0008CBF02F01F024FF0A04005FA02F2C0F82B
:10AE00000C2594F862200133DBB202EB4202B3EB73
:10AE1000420FE9DB94F86320012000FA02F3023BC1
:10AE200084F86D30002A6FD0024D0021844640F234
:10AE3000033714E0000300501F2B86BF03F01F03ED
:10AE40002A464FF0A0420CFA03F3C2F8083594F8F2
:10AE500063200131CBB29A424FEA400054D9A66C2C
:10AE600006EB01120B01127B1F2A8CBF2A464FF002
:10AE7000A04202F5A162F250A26C1A44167B1F2E6A
:10AE80008CBF2E464FF0A04606F20C565660A66CBC
:10AE90001E44327B02F01F020CFA02F2B260A26C76
:10AEA0001A44127B1F2A86BF02F01F022E464FF063
:10AEB000A04602F5E07246F82270A26C94F86D602C
:10AEC0001A440642137BB7D11F2B86BF03F01F0322
:10AED0002A464FF0A0420CFA03F3C2F80C35B6E74D
:10AEE00043F00203DBB2012202FA03F313F48B7F77
:10AEF00003D0134653E60D46894609EB4902042365
:10AF00004FEAC2081A464AE694F861301F2B10D85F
:10AF10004FF0A04303F5A16203F20C532046C4E9AD
:10AF2000012300F0A7FC0020BDE8F8830220BDE863
:10AF3000F8833D4BEEE7002A6CD043F00103D1E7E4
:10AF400027693978C1F3C101C4E9062584F8641082
:10AF5000002E3FF47BAE3A78606902F01F0203FADC
:10AF600002F2C900CA40027094F8622002EB420269
:10AF70005200012A7FF768AE1D46226994F86410DA
:10AF8000D25C606902F01F0205FA02F2C900CA40F1
:10AF9000C25494F862200133DBB202EB4202B3EBFD
:10AFA000420FEADB50E60320704727693B78C4E98B
:10AFB0000625C3F3001284F86420002E3FF446AE49
:10AFC0003B78606903F01F0301FA03F31201D340D9
:10AFD000038094F8623003EB43035B00012B7FF79F
:10AFE00033AE0A460D46236994F864109B5C606991
:10AFF00003F01F0305FA03F30901CB4020F81230D8
:10B0000094F862300132D2B203EB4303B2EB430F48
:10B01000E9DB19E6012202FA03F313F48B7F3FF414
:10B02000B3AD1346BBE500BF0003005090F860309D
:10B03000012B05D0022B01D000F000B900F046BA78
:10B0400000F000B82DE9F04F8FB090F86830446AF6
:10B0500003910546924633B190F86A30C26CC3F151
:10B06000010302FB034495F86560062E00F0E080C2
:10B07000C6F10503DBB24FF4006202FA03FC402282
:10B0800002FA03F1012202FA03F095F86670002F2C
:10B0900000F0CB80B5F85E30D5F814B0CDF82CC0F8
:10B0A00000220492DA1D4FEAD208C3EBC80354FA17
:10B0B00083F20AF1FF3300241BB208948E460993F1
:10B0C000A94634465146002C00F085800023CDE986
:10B0D0000CE0CDE905230B9DCDF828808246F4468F
:10B0E000079399F967000028B8BF4042013840B281
:10B0F000421C55D0059C039B01FB00F607FB06F69E
:10B1000010F0010E03EB860607FB01F36ED099F9F0
:10B110006720002A74DB002900F08480049A16441A
:10B1200006EB43070022CDE9000904EB0108029178
:10B1300036F8121037F8120011EA050318BF9BF811
:10B14000003011EA0C0F1CBF9BF8019043EA090381
:10B1500011EA0A0F1CBF9BF802100B4328421CBFC8
:10B160009BF803100B4310EA0C0F1CBF9BF8041054
:10B170000B4310EA0A0F1CBF9BF805100B4304F8A1
:10B18000013B7244444512B2D2D1DDE90009029973
:10B1900099F86670431E58B2431CACD199F86540CB
:10B1A000079B4FEA4C0C002B38D1052C36D94FF0B9
:10B1B000010A4FF40065069B059A0A98013306932D
:10B1C000DBB202EBC002A3420592079389D3DDE90B
:10B1D0000CE0DDF82880089B01330893DBB29F4226
:10B1E00023D9049B03EB410304936CE70029D1D0DE
:10B1F000049A164406EB43074FF0010E002292E733
:10B2000081B1089A013FBF1A01FB07F706EB470718
:10B21000099A07EB43064FF0FF3E84E76D004FEAC3
:10B220004A0AC8E7431E58B265E70FB0BDE8F08F81
:10B23000102020214FF4004C27E700BF2DE9F04FEC
:10B2400095B09246059190F868104569436AC26CC2
:10B250000E9061B1014690F86A0091F86010B2FB5F
:10B26000F1F1C0F1010000FB01F103EB81030E9845
:10B2700090F86510B0F85E40062900F02081C1F119
:10B280000501C9B24FF4006088401090402000FAD8
:10B2900001F6012000FA01F71846002139F010FFED
:10B2A00003460E9890F86220002A00F0FD80E11D10
:10B2B0004FEAD10CC4EBCC01C9B205F1180B03EB7A
:10B2C00081050AF1FF339BB20021119390F866903B
:10B2D00004910133069331460895CDF834C0B9F195
:10B2E000000F00F0D8800E9ACDF83CA0002392F811
:10B2F000652007930B930B46002A00F0BB80BDF935
:10B3000044100C91CDE9123700244946DDF8408005
:10B31000DDF83890DDF83CC009949A46BE460A94A0
:10B3200099F9674084EAE473A3EBE473013B5BB2F1
:10B33000581C00F08480089E2746604687EAE77222
:10B34000049CA2EBE772D2B204FB023200FB02F2D1
:10B35000059C01FB02F213F0010504EB820201FBE4
:10B3600000F451D0002F58DB002800F0A580079989
:10B37000571807EB440C0022CDE90290CDE90036C6
:10B3800031462C4606EB800637F812903CF81250F6
:10B3900019EA080318BF5BF8183C19EA0A0F1CBF2A
:10B3A0005BF8140C034319EA0E0F1CBF5BF8100C7A
:10B3B000034315EA080F1CBF5BF80C0C034315EAA6
:10B3C0000A0F1CBF5BF8080C034315EA0E0F1CBFE5
:10B3D0005BF8040C034351F8040B224418438E42DB
:10B3E00012B241F8040CCFD1DDE90290DDE900365C
:10B3F000069A99F8661006EB8206013B5BB25A1C6E
:10B400001AD099F9677099E70028F6D0079957186C
:10B4100007EB440C01250022AEE700284CD00B9D21
:10B420000139491B00FB01F102EB410C0CEB440715
:10B430000C9A4FF0FF359FE799F8652084460A9BE8
:10B440004FEA4A0A002B32D1052A30D94FF0010EBB
:10B450004FF40068099B08980D9C01330993DBB2F7
:10B4600000EB4410934208900A93FFF459AFDDE9D2
:10B47000123789460B9907980F9C01310B91C9B27D
:10B4800000EB4400894507903FF636AF19460E9B06
:10B4900093F86220A246049B01330493DBB29A42E4
:10B4A0000BF1180B3FF61BAF15B0BDE8F08F4FEA5C
:10B4B00048084FEA4E0ECDE7013B5BB23EE74FF442
:10B4C0000041102720261091E6E600BF2DE9F04F3D
:10B4D00095B04569059190F868101092466AC26C63
:10B4E000834659B190F86A009BF86010B2FBF1F105
:10B4F000C0F1010000FB01F106EB41069BF865106D
:10B50000BBF85E40062900F01E81C1F10501C9B2F9
:10B510004FF4006000FA01F340200E9300FA01F3AB
:10B5200001200F9300FA01FA0021304639F0C8FDDE
:10B530009BF86220002A00F0FC80E31DDF08C4EBCA
:10B54000C703DBB206EB4304109B9BF866800894AC
:10B55000013B1FFA83FC002304930CF10103CDF897
:10B5600044B00693644605F10C0B0D974046002845
:10B5700000F0D680119991F86530002207920B9265
:10B580001A460B461099D046002A00F0BA80DDE931
:10B590000E594FF0000C26B2C246CDF848800C96EA
:10B5A000CDF824C01394CDF828C0884693F967706D
:10B5B00087EAE771A1EBE77101394CB2611C00F039
:10B5C00084800899049A87EAE776A6EBE776F6B2D4
:10B5D00002FB064608FB06F6059A00FB06F614F089
:10B5E000010C02EB860600FB08F251D0002F5ADB5B
:10B5F000B8F1000F00F0A4800798064406EB42075C
:10B600000022CDE90041CDE9023801EB480E0846A1
:10B6100036F8121037F8124011EA050318BF3BF84C
:10B620000C3C11EA090F1CBF3BF80A8C43EA0803E3
:10B6300011EA0A0F1CBF3BF8081C0B432C421CBF2D
:10B640003BF8061C0B4314EA090F1CBF3BF8041C13
:10B650000B4314EA0A0F1CBF3BF8021C0B4330F8E3
:10B66000021B62440B43864512B220F8023CCFD144
:10B67000DDE90238DDE90041069A93F8660001EB46
:10B680004201621E54B2621C1DD093F9677099E7A3
:10B69000B8F1000FF5D00798064406EB42074FF0CB
:10B6A000010C0022ADE7B8F1000F49D0471E0B98FE
:10B6B0003F1A08FB07F706EB470707EB42064FF078
:10B6C000FF3C0C9A9DE793F865200A994FEA4909D7
:10B6D000002931D1052A2FD94FF0010A4FF4006516
:10B6E0000999089C0D9E01310991C9B204EB061419
:10B6F000914208940A91FFF459AF4146139CDDF83A
:10B7000048800B9D079E01350B95EDB206EB410677
:10B71000A84207963FF638AF119B93F86220C246C5
:10B72000049B01330493DBB29A420BF10C0B3FF6FE
:10B730001EAF15B0BDE8F08F6D004FEA4A0ACFE7A3
:10B74000621E54B23EE74FF400432020CDE90E3094
:10B750004FF0100AE8E600BF90B110B500F0AAFA69
:10B760000446406A08B15FF079FFA06C08B15FF051
:10B7700075FF206918B15FF071FF0023236110BDD0
:10B78000704700BF2DE9F04182B09DF82C409DF834
:10B7900024609DF830709DF834E09DF838C09DF924
:10B7A0003C500194002857D0109C002D08BF012563
:10B7B000002C51D00446052B28BF0523002D84F80A
:10B7C000675084F86520B8BF6D42019A84F8612003
:10B7D000EDB203EB4302052E109884F83470A4F800
:10B7E0005C104FEA420215FB01F137464FF00005AD
:10B7F00028BF05272060A4F85E10D0B284F844E08A
:10B8000084F868C084F86230A564656284F8637067
:10B810000121804660F006F8206130B30121380133
:10B8200060F000F80346A0642069CBB10899424655
:10B8300039F062FA66B10A9B591E2B46A26C11F8C8
:10B84000015F02EB03120133D8B287421573F5D8BA
:10B85000002002B0BDE8F081032002B0BDE8F08115
:10B8600001935FF0FBFE019B2361022002B0BDE863
:10B87000F08100BF00286BD070B590F8662090F87A
:10B880006530511E013B82B0012A80F86B3080F890
:10B890006C1088BF90F86C3090F863104FF0000285
:10B8A0008CBF03F1FF33012380F86D3080F86E20E8
:10B8B000826500293DD04FF0010C264940F2033447
:10B8C000E64612E01F2B86BF03F01F030D464FF024
:10B8D000A0450EFA03F3C5F8083590F8635001321D
:10B8E000D3B29D424FEA4C0C23D9836C03EB021375
:10B8F00016011B7B1F2B86BF03F01F030D464FF065
:10B90000A04503F5E07345F82340836C90F86D5033
:10B91000334415EA0C0F1B7BD4D11F2B86BF03F0D9
:10B920001F030D464FF0A0450EFA03F3C5F80C3582
:10B93000D3E7019000F030FA0198036801224FF438
:10B940007A715A60DA60C3F840151A6002B070BDAF
:10B95000704700BF000300502DE9F041836B026C7B
:10B960001A60D0E90B321A60836A026B1A600368AE
:10B97000A54F01265E6003685E64D3F84435C26A51
:10B9800090F86B30016B1160054603F0FF083743F8
:10B990003BBB90F863104446F9B195F86C3095F8CC
:10B9A0006D2053401E424FEA041010D0AA6C95F847
:10B9B0006CC002EB04131CEA060F996814BF1358FD
:10B9C0005B684FF400701960B84795F86310013454
:10B9D000E3B299424FEA4606DFD895F86C3085F815
:10B9E0006D3095F86B3095F865200133DBB29A42E3
:10B9F00085F86B300DD8002285F86B2095F86C30F7
:10BA000095F866100133DBB2994285F86C3040F24C
:10BA100098802A6D2B6802FA08F101225A604020B2
:10BA2000DA60C3F840151A60B847D5E90F321A60DA
:10BA3000B5F85E2095F86C1095F865C095F86B30F8
:10BA400095F860E007320CFB0133D610D10895F869
:10BA50006820C9000EFB03F301FB03F322B195F844
:10BA60006A20E96C01FB02336A6ABEF1010F02EB46
:10BA70000307D5E90640D5E9013100F0C780F2B2ED
:10BA8000561EBEF1020FF6B26CD0002A41D007EB71
:10BA9000461607F12002403652F8207C1F601C60D9
:10BAA00000BF00BF086052F81C7C1F601C6000BF14
:10BAB00000BF086052F8187C1F601C6000BF00BF08
:10BAC000086052F8147C1F601C6000BF00BF086053
:10BAD00052F8107C1F601C6000BF00BF086052F865
:10BAE0000C7C1F601C6000BF00BF086052F8087C1F
:10BAF0001F601C6000BF00BF086052F8047C1F601C
:10BB00001C6000BF00BF2032B2420860C4D195F86B
:10BB100065C0BCF1010F12D995F86B307BB92A686A
:10BB2000012353642B6DD2F84425C3EBC3031344A4
:10BB300004336A6DDB08934238BF13462B65BDE8BA
:10BB4000F08185F86C2095F86E303BB195F86A303D
:10BB5000C3F1010385F86A3085F86E20AB6D0133BF
:10BB6000AB6556E7002AD4D007EB061607F11002A2
:10BB700006F1200795F8646003EB460632F810CC16
:10BB8000A6F800C01C6000BF00BF086032F80ECCF1
:10BB9000A6F800C01C6000BF00BF086032F80CCCE3
:10BBA000A6F800C01C6000BF00BF086032F80ACCD5
:10BBB000A6F800C01C6000BF00BF086032F808CCC7
:10BBC000A6F800C01C6000BF00BF086032F806CCB9
:10BBD000A6F800C01C6000BF00BF086032F804CCAB
:10BBE000A6F800C01C6000BF00BF086032F802CC9D
:10BBF000A6F800C01C6000BF00BF1032974208606A
:10BC0000BCD195F865C084E7407C0C00002E80D044
:10BC1000013EB6B207EBC60607F1080206F11007AF
:10BC200095F864601E4412F808CC86F800C01C60C9
:10BC300000BF00BF086012F807CC86F800C01C6087
:10BC400000BF00BF086012F806CC86F800C01C6078
:10BC500000BF00BF086012F805CC86F800C01C6069
:10BC600000BF00BF086012F804CC86F800C01C605A
:10BC700000BF00BF086012F803CC86F800C01C604B
:10BC800000BF00BF086012F802CC86F800C01C603C
:10BC900000BF00BF086012F801CC86F800C01C602D
:10BCA00000BF00BF083297420860BCD195F865C05C
:10BCB0002FE700BF002860D0436A002B5DD010B48E
:10BCC00090F86E30002BFBD102684FF0010CC2F8E7
:10BCD00004C00268C2F844C0816BD2F84425026CEB
:10BCE0000A6090F86220C2B1244903F0FF030269A0
:10BCF000D25C1F2A0C468CBF02F01F024FF0A044FA
:10BD00000CFA02F2C4F80C2590F862200133DBB281
:10BD100002EB4202B3EB420FE9DBB0F85E3023B333
:10BD2000164C00224FF0010C90F861301F2B214679
:10BD30008CBF03F01F034FF0A0410CFA03F3C1F8CE
:10BD4000083500BF00BF90F861301F2B21468CBF23
:10BD500003F01F034FF0A0410CFA03F3C1F80C35B8
:10BD6000B0F85E3001329A42DED3836A026B1A6009
:10BD7000D0E90B321A6010BC7047704700030050C6
:10BD800090F8683033B1012380F86E3090F86E304F
:10BD9000002BFBD1704700BF1E4A0368934212D0AC
:10BDA00002F5805293422ED002F5805293422CD05D
:10BDB00002F5803293422AD002F58052934208BFA6
:10BDC000042201D070470022134B03EBC201002074
:10BDD00091F9041053F832304FF4803C0122814233
:10BDE0005A60C3F80405DA60C3F80805C3F8100503
:10BDF000C3F804C3E6DB4809084B01F01F018A4081
:10BE000043F8202070470122DEE70222DCE703220C
:10BE1000DAE700BF00800040487C0C0000E100E051
:10BE2000BFF34F8F0549064BCA6802F4E062134323
:10BE3000CB60BFF34F8F00BFFDE700BF00ED00E018
:10BE40000400FA05014B1868704700BF500001203C
:10BE500007EE900AF5EEC07AF1EE10FA01D400F088
:10BE600009B808B580F0004000F004F8404261EBEA
:10BE7000410108BD70B5FBF73DFA0C4B00220446AA
:10BE80000D46FBF755FCFBF77FFD0646FBF710FA66
:10BE9000074B0022FBF74CFC02460B462046294686
:10BEA000FBF7C8F8FBF770FD314670BD0000F03DB0
:10BEB0000000F04110EE101A21F000430122B3F10E
:10BEC000FF4FF0EE407A026015D2002B72D000B521
:10BED000B3F1E45F87B013D20029BEBF4FF0FF3348
:10BEE0000360B1EE400A36F0F5FFB1EE407AB0EEF5
:10BEF000470A07B000BD20EE007AB0EE470A70474F
:10BF000000295EDBB3F17E5F68D0B3F1804F65D06E
:10BF10004A0000F19F809FEDDD6ADD4A934240F2C6
:10BF2000A382DC4A934240F24A82F0EE005A75EE58
:10BF3000E75A9FEDD67A9FEDD85ADFEDD86ADFED4C
:10BF4000D84A9FEDD84A65EEA57AE7EE856AA7EE56
:10BF5000A44A9FEDD55ADFEDD54AA6EEA75AE4EEE6
:10BF6000274ADFEDD36A9FEDD34AE5EE276AA4EEB8
:10BF7000A74A9FEDD15ADFEDD14AA6EEA75AE4EECB
:10BF8000274ADFEDCF6AE5EE276A9FEDCE5AA4EE91
:10BF9000A75A66EEA56AB6EE004AE5EE276AF0EE0D
:10BFA000667AE5EEC47A37EE877A00299FDA36EEB4
:10BFB000477A9CE7DFEDB57AF7EE006A86EEA77A5E
:10BFC0009BE7B3F1964F0CD3DFEDB07AF7EE006A42
:10BFD00086EEA77AB0EE470A07B000BD9FEDAB7AB8
:10BFE00085E7B3F17A5FC0F05982B1EE407A8DED0A
:10BFF000020AB0EE470ACDE9041003938DED017AF1
:10C000002FF000F99DED017ADDED027A059AB4EE8C
:10C01000407AF1EE10FADDE9033140F09A819FEDAC
:10C02000AA7A37EE677A17EE100A00F0010007EEE1
:10C03000100AB8EEC77A8000CDE901310492CDED47
:10C04000037A062800F28A82DFE800F05DDFDF591C
:10C0500059ECEC00B3F1824F80F09B819FED8B6A2D
:10C06000DFED9A6ADFED9A5ADFED9A4ABDEEE77A84
:10C07000B8EEC75A17EE103A77EEC57A9FED965A8A
:10C08000E7EEA65A033BA7EEA45ADFED946ADFED74
:10C09000944AE5EEA76AE5EE274ADFED925A9FED56
:10C0A000925AE6EEA75AA4EEA75ADFED906ADFEDAA
:10C0B000904AE5EEA76AE5EE274ADFED8E5A9FED3E
:10C0C0008E5AE6EEA75AA4EEA75ADFED8C6AE5EE8B
:10C0D000A76AF7EE005AE5EE275A66EEA76AF6EE73
:10C0E000004A86EEA57AA7EEA47A042B3FF65DAF50
:10C0F000DFE813F0C900AC00270118012A01F7EEB0
:10C10000006A36EEC77A9FED7E0ADFED600A27EE01
:10C11000000A002000F06CFFDDE90131DDED037A5B
:10C12000049AF1EE406AF5EE406AF1EE10FA3FF43F
:10C130004BAF27EEA67A9FED720ACDED026AB0EE04
:10C14000C77A80EE070ACDE903310592CDED017A79
:10C1500036F0C0FEDDED026ADDED017AF5EEC06A73
:10C16000F1EE10FADDE90331B0EE407A03D5059A1D
:10C170004FF0FF301060B3F17E5F3FF4B8AEB3F123
:10C18000804F3FF4B4AE4800F1EE677AB0EE476AF4
:10C190007FF5C3AEB3F1824FFFF462AFB0EE670A32
:10C1A0008DED036A0291CDED017A36F093FEDDED5F
:10C1B000017A9FED542ADFED542A9FED543ADFEDCA
:10C1C000543A9FED544ADFED544A9FED547A029958
:10C1D0009DED036AF7EE006A86EEA75AF6EE005A66
:10C1E00077EEE55A65EE057A70EE666AE7EE822A2A
:10C1F000A2EEA73AE3EE273AA3EEA74AE4EE274AD7
:10C20000A4EE857AA5EEA67ACFE6F6EE006A36EEC3
:10C21000C77A9FED3B0ADFED1D0A27EE000A00F00A
:10C2200029FB79E7F7EE086A37EE667A9FED340A64
:10C23000DFED160A27EE000A00F01CFBDDE90131F4
:10C24000DDED037A049AF0EE406A6CE7F7EE006ADF
:10C25000B0EE080A37EE800A20EE260AF0EE006AF9
:10C2600077EEA67A8DED037A27EE800A8DED026ACD
:10C27000019136F02FFE9DED037A01999DED026A42
:10C2800037EE007A91E6B7EE000AE7E7000000001B
:10C290006666663F17A6DD3FA283D3376797673987
:10C2A000752C3C384584E238A1549C3A34B6053AA2
:10C2B0007E02F23BC66E3D3B01F0893D1599A83CDC
:10C2C0003F239E3D661AA53E0000004B67FF0538E0
:10C2D000B435F13ABDD7F536D6EE4B3AE440DA3C08
:10C2E00054BF983CE6DC153E6E0F303E7ACCA63E3D
:10C2F000C5D0383F5A245C3E3B2DB23F3F239EBD04
:10C30000DB0F4940E8C4D5BAD23D5B3A5C061CBAA3
:10C31000FD0C503A610B36BBABAAAA3D1D7FD63E41
:10C3200000000000F7EE006AF1EE045A77EEA55A1D
:10C3300065EEA65AF1EE006A77EEA66A66EEA56A89
:10C3400086E7F7EE005AF5E7F1EE086A77EEA66A9F
:10C35000EAE7F6EE006A27EE267ACDE90231B0EE82
:10C36000470ACDED047A8DED017A2EF04BFF9DED5D
:10C37000017A059A37EE407ADDE9023137EE077A25
:10C38000F0EE477AFEEECF7A17EE900ADDED047AF2
:10C3900052E6B3F1B94FC0F097808DED020A8DEDF2
:10C3A000010A36F097FDB7EE007A30EE477ADDED00
:10C3B000027A1FED256A019927EE277AF5E5724A80
:10C3C000934240F28480DFED716A9FED717A77EEDF
:10C3D000E66A66EEA62A9FED6F4ADFED6F5ADFED43
:10C3E0006F4A9FED6F5ADFED6F3A9FED6F3A62EE45
:10C3F000A67AE7EE844AA7EEA55A9FED6C4ADFEDD8
:10C400006C5AA4EEA74AE5EE275ADFED6A4A9FED83
:10C410006A5AE4EE274AA5EEA75AA7EEA33ADFED43
:10C42000675A9FED674ADFED673AA5EE274AE4EECB
:10C43000A75AE3EE273ADFED644A9FED645AE4EE33
:10C44000265AE3EEA74ADFED626A9FED624AE5EE07
:10C45000E76AA4EEA75AF0EE667AD2EE857A77EE16
:10C46000C47A37EE877AA0E5B0EE670ACDE90231EB
:10C470008DED046ACDED017A36F02CFD564A029B13
:10C48000DDED017A03999DED046A9342B1EE407AA5
:10C490005CD9F7EE005A75EEE75A4CE59FED4F0A6E
:10C4A000DFED3B0A0293CDE9031027EE800A00205E
:10C4B000CDED017A00F09CFDDDE90231DDED017A80
:10C4C000049AF0EE406A2EE69FED316A66E6B7EE1A
:10C4D000007A77EEC77A9FED2E7A9FED415ADFED15
:10C4E000416ADFED415ADFED414AE7EE856AE7EE4A
:10C4F000A54A9FED3F5ADFED3F5AA6EEA75AE4EE5C
:10C50000A75ADFED3D6ADFED3D4AE5EE276AE5EE2D
:10C51000A74A9FED3B5ADFED3B5AA6EEA75AE4EE41
:10C52000A75ADFED396AE5EE276AB7EE005AA5EEA5
:10C53000A75A66EEA76AFEEE004AC6EE855AF0EEEE
:10C54000656AE7EEA46A36EE877A2EE52F4A9342B3
:10C55000C3D9DFED2F6A77EEE66A3AE7F0EE006ABC
:10C5600037EE667A9FED1D0ADFED090A27EE000A15
:10C57000002000F03DFDDDE90131049ADDED037A94
:10C58000F1EE406ACFE500BF1FA69D3FC316BB3F3B
:10C590000000000027F9A3B9F7E9AF3967F8663A58
:10C5A00085300DBA6B7BA53976F4B7BAFE7771BBCF
:10C5B0009916143B3D37933CFEFC28BC3C2117BE2A
:10C5C000155A843D07E7C73B474D06BD5EB9F73EA8
:10C5D000521CE631CDCDF83D1F4A3B3FDB0F4940B1
:10C5E0005E3C5B3C78756A3EDBD5523BAF72D53D15
:10C5F000B24B7A3FDFEF443FE73ABA3F2D3908406C
:10C60000F400223FBE2E1D403F239EBD07336D3EEA
:10C610000C5BEC3E10B510EE104A884A24F0004343
:10C62000934288B0014662D9854A934222D824F0C9
:10C630000043002CDFED837A834A23F00F0340F39D
:10C64000E380934230EE670A09BFDFED807A9FED09
:10C65000807A9FED807A30EE670A70EE477A30EE8E
:10C66000670AC0ED007A30EE470A80ED010A01202A
:10C6700008B010BD784A934240D89FED787A9FED7C
:10C68000716AB0EEC00AF6EE007AE0EE077A9FED2E
:10C69000707AFDEEE77AF8EEE76A17EE900AA6EEFA
:10C6A000C60A1F2866EE877A30EE677A6BDCDFF801
:10C6B000C0C100F1FF3E24F000425CF82EC022F021
:10C6C000FF0262455FD081ED007A30EE470A002C10
:10C6D00030EE670A81ED010ACADAB1EE477AB1EEAF
:10C6E000400A81ED007A81ED010A4042C0E7002353
:10C6F00080ED000A4360002008B010BDB3F1FF4F89
:10C7000072D2DA15863AA3EBC25307EE903ABDEE29
:10C71000E77ADFED536AB8EEC77A77EEC77A8DED28
:10C72000057A67EEA67ABDEEE77AB8EEC77A77EEBD
:10C73000C77A8DED067A67EEA67AF5EE407AF1EECD
:10C7400010FACDED077A5DD1B5EE407AF1EE10FA30
:10C7500056D10123434801900220009005A803917F
:10C7600000F00AF9002C039982DA91ED007AD1EDFC
:10C77000017AB1EE477AF1EE677A81ED007AC1ED88
:10C78000017A404274E717EE102AC2F3C752C2EB97
:10C79000D352082A97DD9FED2D7ADFED2E5AB0EEA9
:10C7A000406AA6EEC76A70EE467AE6EEC77AD6EE23
:10C7B000A57A36EE677A17EE102AC2F3C752C2EB9B
:10C7C000E353192B17DD9FED287ADFED285AB0EEE1
:10C7D000460AA6EEC70A76EE407AE6EEC77AD6EEAD
:10C7E000A57A30EE677A6EE730EE400A80ED010AF6
:10C7F00080ED000A7FE7B0EE460A81ED007A64E73B
:10C800000223A7E70323A5E7934230EE270A09BFD7
:10C810009FED0E7ADFED0E7ADFED0E7A30EE070A2D
:10C8200030EE277A30EE470A80ED007A70EE277AF4
:10C83000C0ED017A4FF0FF301AE700BFD80F493F33
:10C84000E3CB1640800FC93FD00FC93F00443537B6
:10C850004344353708A3852E800F494384F9223F8E
:10C8600000008043A82F0C0000A3852E32318D24B8
:10C87000282F0C0010EE103A23F00043B3F1485F6C
:10C880002CD2FDEEC07A17EE903A002B60D060EE0D
:10C89000007A9FED317A9FED315ADFED315A9FEDED
:10C8A000316ADFED316AA7EE875A9FED307AE7EE05
:10C8B000855AA7EEA56AA7EE867AE7EE876A66EE46
:10C8C000A76A60EEC00AB6EE007AE7EEA60AB7EEF7
:10C8D000000AD7EE870A30EE600A704760EE007AF1
:10C8E0009FED1D7A9FED1D5ADFED1D5A9FED1D6ACC
:10C8F000DFED1D6A1E4AA7EE875A93429FED1B7A11
:10C90000E5EE275AA5EEA76AA6EE277AE7EE276A94
:10C9100066EEA76AD5D9174A934214D803F17F432C
:10C9200007EE103AB7EE006A36EE476A60EEC00ACC
:10C93000F6EE005A97EEA57AE7EEA60A37EE607A91
:10C9400036EE470A7047B6EE076AB5EE027AEDE7B3
:10C95000B7EE000A704700BF4ED747ADF6740F31EF
:10C960007CF293B4010DD037ABAA2A3D610BB6BA65
:10C970009999993E0000483F2DE9F04F2DED048B29
:10C98000DBB01C4603938B46C64B6899069253F85E
:10C990002150111D814604F1FF38C0F25082D31E90
:10C9A00048BF131DDB1004930133D900069B15EB20
:10C9B0000804A3EB010218D4049B9FEDBE7A699E84
:10C9C0000134A3EB08031C441EA8002BA4BFF75C92
:10C9D00007EE907A03F10103ACBFF8EE677AF0EE50
:10C9E000477AA342E0EC017AEFD1002DC0F2E68055
:10C9F000039BB8F1000F0DF58C7C464605EB030E4A
:10CA0000B8BF0020C0F2CD80039B1EAF07EB8307A9
:10CA10009C0009EB8300DFEDA77ABA464B46F3ECA6
:10CA2000016A3AED017A8342E6EE877AF7D1013660
:10CA30007645ECEC017A07F10407ECD109ABCDE9BE
:10CA400007B10DF1280A03EB85039FED979ADFEDFF
:10CA5000978A05934C440AEB850746AE019510462C
:10CA60000DEB8503002D93ED460A4FEA850B16DD8D
:10CA700006EB0B03524660EE097AB0EE407AFDEE0B
:10CA8000E77A73ED016AF8EEE77AB342A7EEE87A47
:10CA900037EEA60ABDEEC77AA2EC017AEBD102907E
:10CAA00063F052FAB0EE408AB4EE000A28EE000AB3
:10CAB0002EF0A8FBF2EE007AA0EE678A029800281A
:10CAC000FDEEC89AF8EEE97A38EE678A79DD691EDC
:10CAD000C0F108035AF821E04EFA03FC0CFA03F304
:10CAE000AEEB030EC0F1070219EE903A4EFA02F2D5
:10CAF0006344002A09EE903A4AF821E000F3F280FC
:10CB0000B5EE408AF1EE10FA6CD1019B9D420CDD2E
:10CB10000AEB0B030021944653F8042DBB4241EA73
:10CB20000201F9D1002940F03981019B013B05F157
:10CB3000010C5AF82330002B40F02E81059B012177
:10CB400053F8042D0131002AFAD02944699B049A34
:10CB500003EB020E039BAE441D441EAB03EB8505A5
:10CB600047AB9B441EF8013F07EE903AF8EE677A18
:10CB7000B8F1000FE5EC017ADFED4E7A09DB2A46C9
:10CB80004B46F3EC016A32ED017AA342E6EE877A76
:10CB9000F7D10CF1010C8C45EBEC017AE2DD0D468E
:10CBA0005EE7731C7345CCF8000006F1020605D061
:10CBB000B645CCF804000CF1080CF2D1039B9C00A4
:10CBC0003CE700F0D280F6EE007AB4EEE78AF1EEB0
:10CBD00010FA80F22381B5EE408AF1EE10FA4FF0A0
:10CBE000000292D0DDE907B1069B0295B0EE480A3B
:10CBF000019D0190C81A914663F0A6F99FED2B7A2A
:10CC0000B4EEC70AF1EE10FADDE90123C0F28B8120
:10CC1000DFED257A60EE277A5C1CFDEEE77A0832BC
:10CC2000F8EEE77AA7EEC70AFDEEE77ABDEEC00A96
:10CC300010EE101A4AF8231017EE903A4AF82430F2
:10CC40001046B7EE000A63F07FF9002CB0EE407A90
:10CC5000C0F294810AF1040347A9DFED136A03EBE4
:10CC6000840301EB8401A20046AF73ED017AF8EE74
:10CC7000E77A534567EE877A27EE267A61ED017AE7
:10CC8000F3D1002D0DF1C80CC0F295811744E64692
:10CC9000264600209046064ADFED067A39460023F4
:10CCA00012E000BF1C2F0C000000803B00008043FE
:10CCB000F02E0C0000000000F2EC016AB1EC017AE9
:10CCC0009D42E6EE877A03DB834203F10103F3DD45
:10CCD000013E731CCEED007A77D00EF1040E0130C8
:10CCE000043FD8E70133002D09EE903A40F33C8130
:10CCF00051464FF0000E51F8043B2BBB0EF1010ED4
:10CD00007545F8DC9E4600280ADD01287ED0022801
:10CD100006D1691E5AF8213003F03F0C4AF821C0B1
:10CD2000022A7FF4EDAEB7EE000A30EE488ABEF17B
:10CD3000000F3FF4E5AE0992029063F005F9029806
:10CD4000099A38EE408ADBE6C3F5807341F8043C6B
:10CD500004E00B68C3F1FF0341F8043B0EF1010E40
:10CD60007545F6DC4FF0010ECDE76B1E5AF8232017
:10CD70001212002A7FF7C4AE19EE903A002D03F18B
:10CD8000010309EE903AB3DC022A7FF4B9AEF7EE64
:10CD9000007A37EEC88AB3E66146D7E66C1E59467C
:10CDA0005AF82430019DDDF81CB0E146A0F10802DC
:10CDB000002B7FF445AF0B4609A90B4453F8041D23
:10CDC000013C083A0029F9D03AE74246689B022B19
:10CDD0005EDC002B37DC10D10CF104035FED4B7AE5
:10CDE000134433ED017A634577EE877AF9D1B9F1CF
:10CDF000000F40F0A980CBED007A19EE903A03F0D5
:10CE000007005BB0BDEC048BBDE8F08F691E5AF8DB
:10CE1000213003F07F0C4AF821C081E719EE903AE7
:10CE2000002D03F1010309EE903AC8BF02223FF73B
:10CE30005FAFF7EE007A37EEC88A022260E6002381
:10CE400008210493B2E50CF10401DDED327A1FED07
:10CE5000677A0A4472ED016A624537EE267AF9D1A3
:10CE6000B9F1000F67D177EEC77A8BED007A64B124
:10CE70000123B1EC017A01339C4277EE877AF8DA2C
:10CE8000B9F1000F01D0F1EE677ACBED017AB4E78A
:10CE9000689B032BB1D1002C00F08A800CEB0200C0
:10CEA00090ED007A0346014671ED017AF0EE476A93
:10CEB00037EE277A614577EEC77A81ED007A77EE13
:10CEC000A67AC1ED017AEFD1012C71D090ED007AF4
:10CED0000CF1040173ED017AF0EE476A37EE277A20
:10CEE000994277EEC77A83ED007A77EEA67AC3EDA2
:10CEF000017AEFD15FED917A8B180CF1080C33EDCC
:10CF0000017A9C4577EE877AF9D1DDED326A9DEDA5
:10CF1000337AB9F1000F1AD1CBED006A8BED017AAB
:10CF2000CBED027A69E7BDEEC00A1C4610EE101A7E
:10CF30004AF8231084E6F1EE476A77EEC77ACBED24
:10CF4000006A002C94D19EE7F1EE677A53E7F1EE88
:10CF5000666AB1EE477AF1EE677ACBED006A8BED47
:10CF6000017ACBED027A48E7012815D002287FF438
:10CF70000BAF0EF03F034AF8213005E7689B022B08
:10CF800012DC002B25DC7FF438AF5FEDB67AB9F107
:10CF9000000F3FF430AFD7E70EF07F03022A4AF8C4
:10CFA00021307FF4ADADF2E6689B032B7FF425AF13
:10CFB0005FEDC07AA9E70020614623460860002B98
:10CFC0003FF404AF023B5D1C486001F10801F5D15C
:10CFD000FCE6DDED327AB9F1000F04D04FF00043EA
:10CFE000CBF800304FE70023CBF800304DE700BF0F
:10CFF00010EE103A23F00043B3F1485F04D2FDEE87
:10D00000C07A17EE903A5BB360EE007A9FED157A26
:10D01000DFED155A9FED156ADFED156AE7EE875AC9
:10D020009FED147AA5EEA76A20EE275AE6EE276A4E
:10D03000A6EEA77A30B9DFED106AE7EE876AA6EEB2
:10D04000850A704727EE457AF6EE006AA0EEA67ACA
:10D05000DFED0A6AD7EE270AE5EE260A30EE600A0F
:10D06000704700BFD3C92E2F342FD7B21BEF3836ED
:10D07000010D50B98988083CABAA2ABEABAA2A3E4A
:10D0800010EE103A23F00042B2F1465FF0EE407A23
:10D0900010D2BDEEC07A17EE101A01BB431C134329
:10D0A00000F0A080012800F09C80BFEE007A87EE9F
:10D0B000270A70474F498A4211D39FED4F7ADFED1F
:10D0C0004F6A002BBCBFF1EE600AF1EE407A77EEBA
:10D0D000677A36EEE07ADFED4A0A77EE277A67EE76
:10D0E000A76ADFED484ADFED485A9FED485A9FEDA9
:10D0F000486A404926EEA67A8A42E7EE245AA7EE0D
:10D10000056ADFED444A9FED445AE5EE874AA6EEF4
:10D11000075ADFED425A9FED426AE4EE875AA5EEC8
:10D12000076ADFED404A9FED405AE5EE874AA6EEDA
:10D13000075A9FED3E6ADFED3E5AA4EE876AE5EEA0
:10D14000075AB0EE467AA5EEA67A27EEA65AB0EEBA
:10D15000606AA7EE056ADFED374AE6EE260AE5EEDD
:10D16000240A37EEA00A1ED201283AD0BFEE007A78
:10D17000C7EE006A10EE103A6FF30B0306EE103A9A
:10D1800016EE903A76EE677A6FF30B0300EE103AE4
:10D1900070EEE70AF7EE007AE6EE007AE0EE807ACB
:10D1A000A7EEA60A704707EE100AF8EEC76A20EE4F
:10D1B000007A30EE260A9B1787EE006A03F002031E
:10D1C000C3F10103F0EE005A36EE606A07EE103A42
:10D1D00077EEC67AB8EEC77AE7EEE56A26EE870AFA
:10D1E00070477047F0EEC07AB7EE007A87EE270AF4
:10D1F000704700BF40A12C3FDA0F493F682122331E
:10D20000000000005FAE9BB745F4A3388453D937C4
:10D210007AC09538C8261A3AB937813916696B3BF6
:10D2200048DEBE3AA427B33C1F37113C8988083E2C
:10D23000D10D5D3DABAAAA3E42084B0802F0553223
:10D2400003F05533801AC91A8A08830801F0333174
:10D2500000F0333002F0333203F0333303448818E4
:10D2600003EB131300EB101003F00F3300F00F303B
:10D27000184400EB002000EB0040000E704700BF98
:10D280002DE9F04782B00646DDF828E00846B446AE
:10D290000D46002B4ED18A4214466DD9B2FA82F265
:10D2A00042B1C2F12003954026FA03F394401D4396
:10D2B00006FA02FC260CA7B2B5FBF6F14FEA1C43B6
:10D2C00006FB115543EA054301FB07F0984209D9D3
:10D2D000E31801F1FF3580F00381984240F20081AC
:10D2E000023923441B1A1FFA8CFCB3FBF6F006FB31
:10D2F00010334CEA034C00FB07F363450AD914EBE7
:10D300000C0C00F1FF3580F0ED80634540F2EA80BF
:10D31000A444023840EA0140ACEB030C0021BEF10A
:10D32000000F04D02CFA02F30022CEE9003202B042
:10D33000BDE8F0878B4209D9BEF1000F01D0CEE9DC
:10D3400000610021084602B0BDE8F087B3FA83F11E
:10D35000174600294DD1834202D3B24200F20F8119
:10D36000B6EB070C60EB030301201D46BEF1000F76
:10D37000DDD0CEE900C5DAE7002A00F098801A4631
:10D38000B4FA84F3002B40F0AF800B1B270CA6B23D
:10D390000121B3FBF7F54FEA1C4007FB153340EAC8
:10D3A000034306FB05F8984507D9E31805F1FF305C
:10D3B00002D2984500F2E8800546A3EB08031FFA65
:10D3C0008CFCB3FBF7F007FB10334CEA034C06FB75
:10D3D00000F3634508D914EB0C0C00F1FF3602D2C0
:10D3E000634500F2CE803046ACEB030C40EA0540CA
:10D3F00095E7C1F120058B4022FA05FC4CEA030CAD
:10D4000000FA01F426FA05F3E84002FA01F943EACA
:10D4100004084FEA1C4206FA01FAB0FBF2F71FFAC1
:10D420008CF602FB17004FEA184444EA004407FB5D
:10D4300006F0A0420AD91CEB040407F1FF3380F088
:10D440009C80A04240F29980023F6444241A1FFA53
:10D4500088F3B4FBF2F002FB104443EA044300FB00
:10D4600006F69E4209D91CEB030300F1FF3480F05D
:10D4700082809E427FD90238634440EA0740A0FB85
:10D4800009749B1BA3423E46A04664D361D0BEF103
:10D49000000F0AD0BAEB060263EB080303FA05F5A6
:10D4A000CA401543CB40CEE9005300213FE7730843
:10D4B00043EAC1734A08190C41EA02414FEAC67CAB
:10D4C0009BB2B2FBF4F02646A04627461F2243EA51
:10D4D0000143B1FBF4F1A3EB080341EA004158E733
:10D4E0002946FFE6284615E71A46C3F120019C406D
:10D4F00026FA01F320FA01F190400343270C06FAC3
:10D5000002FCB1FBF7F0A6B207FB1015190C41EABB
:10D51000054100FB06F58D423BD9611801D28D42D1
:10D5200020D8491B0138B1FBF7F5019505FB06F83A
:10D53000019D9BB207FB151143EA0143434526D2E7
:10D54000E31805F1FF31C6D24345C4D2A91E2344D6
:10D55000C1E7BA459BD2B7EB090664EB0C0401386E
:10D56000A04694E7651B29440238B1FBF7F5019505
:10D5700005FB06F8DCE720467FE71F4666E708461E
:10D58000F4E6A44402382FE7023D234415E701994D
:10D59000A1E7491BB1FBF7F5019505FB06F8C7E7C5
:10D5A00070B590F82A30DC0657D4054640F2165084
:10D5B0000E4647F081F9044688B1436830469847E3
:10D5C000A36801219B6906469847002847D1A368B4
:10D5D00005F1080130469B68BDE8704018472349B3
:10D5E000304640F0BDFA0446C0B190F85030D9063C
:10D5F00035D443F0100305F1080180F8503029F0CC
:10D6000051FD95F82A3013F00C0F204618BF012168
:10D61000BDE8704008BF002129F034BD14493046F0
:10D6200040F09EFA0446E8B190F82A309A0716D4E2
:10D6300043F0020305F1080180F82A3028F050FD7C
:10D6400095F82A3013F00C0F204618BF0121BDE8D1
:10D65000704008BF002128F0F3BC0EF06BFC0548B9
:10D6600073F0F6FC044873F0F3FC00BF00EC0B0011
:10D670004CE90B00148C0B00048C0B0010B5144605
:10D6800084B01A6030B1104600215EF0CBF898B13A
:10D6900004B010BD084603A9019364F03DFA019B54
:10D6A00020B90398002801DD1860EDE71868002113
:10D6B0005EF0B8F80028EBD1014620465EF0B2F8E3
:10D6C0000028E5D1092061F04DFD00BF12F000BD3A
:10D6D0002DE9F04385B007460024084601AA6946B3
:10D6E000009442F071FF0099022950D97868012214
:10D6F00089002FF0A9FA009B7C6006463C81002B34
:10D7000040D02546019B23490022029253F8250070
:10D7100040F2015238F0E4FC019B03AA53F82500C3
:10D7200002A945F0DDFB40F201520221029838F0D7
:10D7300055FC039B40F29661186838F025FD47F6CA
:10D74000FF72154940F29663814638F037FC039B1F
:10D7500040F29C61586838F017FD40F29C630E4916
:10D7600047F6FF72804638F029FC06EB850326F861
:10D770002590A3F80280009B0134A4B29C42254668
:10D78000C0D35B007E603B8105B0BDE8F0830348F9
:10D7900073F04AFCFC640B000080FFFF74890B00EF
:10D7A0002DE9F0472DED028B1C4696B0C368BDF8FD
:10D7B0008470BDF88C600546B0EE408A8A46002B26
:10D7C00000F0D18041688B4200F014818E4B1878B4
:10D7D0004FF00008FF2885F8458013D0019262F0D1
:10D7E000DFFD2946814689480AF08AF939F00803A5
:10D7F000019AC5F80C8085F84480484602D00EF0A6
:10D80000EFFA019A1F2F66D9BAF1000F40F0A480F9
:10D81000002E40F0D68025964FF00A09002A00F02D
:10D820008F8040F20123ADF83830002C00F0998051
:10D83000631C0DF13808ADF83A30404600230F93D1
:10D8400062F0D0FD0346002B3FD1DFED717A9FEDF2
:10D85000716A259A099228EE277A229A0D93C7EECB
:10D86000067A9E4208BF1A4622920692209A049295
:10D87000694A089302FB04F4684A0B93A2FB042450
:10D880000122640BF6EE006A77EEA67A8DF8352059
:10D89000FCEEE77A082241461846ADF81470ADF860
:10D8A0001C608DF820900C93CDED0A7AADF82C40D9
:10D8B00001930CF04BF800285BD1534808AA04A947
:10D8C00062F06AFD0346002861D0184616B0BDEC30
:10D8D000028BBDE8F0871F2E3BD8BAF1000F75D040
:10D8E000259B002B00F08C801B799DF80810F0EE32
:10D8F0000C7A03F07F03B4EEE78A63F34701F1EE9D
:10D9000010FA259B8DF8081066D807EE904A9FED17
:10D91000447AF8EE677AF4EEC77AF1EE10FA5BD843
:10D92000D3F80530CDF80930259BB3F80930ADF8B0
:10D930000D3002AB25934FF00209002A7FF471AF3E
:10D940000DF138084046CDE90E2262F04BFD03464A
:10D9500079E7BAF1000F34D0002325934FF0060980
:10D960005CE7234665E71F2F80F845303FF64CAF54
:10D97000B1E7C2B20199404662F022FD0346002899
:10D980009BD0184616B0BDEC028BBDE8F0871E4C4C
:10D990001E492A4605F128000AF088F821789DF9E9
:10D9A0009020012062F028FD034600288DD12078C8
:10D9B000012162F0F3FC0346002886D1209AEA6038
:10D9C00083E7CDF894A04FF0080927E7A6B1CDF87A
:10D9D00094A04FF0040921E7D3F80530CDF80930C1
:10D9E000259BB3F80930ADF80D3002AB25934FF00D
:10D9F000030913E7112368E725964FF005090DE7A2
:10DA00004FF001090AE700BFA70601200501030046
:10DA10000024744900401C4440420F005917B7D1FC
:10DA20006666A63F38B5DFED117A416020EE270A21
:10DA30000446BCEEC00A049D80ED020A11461A4657
:10DA40009DF8143084F820300C3061F043FE35B17D
:10DA5000224628460649BDE838400AF027B8214644
:10DA60000348BDE8384009F0EDBF00BF00007A442C
:10DA700059BC0300F0B583B0416017464A680446BC
:10DA800090790A9A84F82C0022858D7D05F0300665
:10DA900005F0060500283DD14FF6FF72E284002E06
:10DAA00044D1089BE36194F82C20099B2362002356
:10DAB00084F82D3084F82A30A3840B9BDAB1002B34
:10DAC0003BD023492246184609F0F0FF5EB116F01C
:10DAD000040118BF012160681ABF84F82B100022CE
:10DAE000012213F0A7F825B1AA060ED5022384F867
:10DAF0002B3003B0F0BD2BB316492246184609F06F
:10DB0000D5FF002DF5D06B07F0D5012384F82B301D
:10DB100003B0F0BD4A680193D0680AF045FE324672
:10DB20002E46019BE0841546002EBAD01A4639468F
:10DB300004F1080061F0CEFDB3E70548214609F085
:10DB400081FFC3E70348214609F07CFFD9E700BF06
:10DB5000199E0800919E08002DE9F0414FF6FF76CE
:10DB600082B003610023154681608371C360C27176
:10DB700004468680084601A90BF0D0FA681C221DD5
:10DB800001A9C0B262F056FC074618B1384602B08F
:10DB9000BDE8F0810F4AA5881388DFF84080AB42CA
:10DBA00028BF2B4613800C4A1388AB4238BF2B4644
:10DBB0001380044638F81400B0422A46294601D0A2
:10DBC00062F03CFC4434B4F5AA7FF3D1384602B08D
:10DBD000BDE8F081A40601208C780120A00A012074
:10DBE0002DE9F04F89B081461D4640689DF8488078
:10DBF0008A46164657F082FF002D4FD088F0010864
:10DC0000DFF8ACB04FEA4818002701E02D1B45D0E3
:10DC1000B5F5806F2C46424628BF4FF4806403A9B7
:10DC20004846CDE90667CDE904478DF80C708DF8BC
:10DC30000DA001F035FE58452644E7D00190D9F8F3
:10DC4000040057F03DFF184A019B934219D00BD9AD
:10DC5000164A934210D0013A23F00203934218D09F
:10DC6000002009B0BDE8F08F043A93420ED16FF066
:10DC7000730009B0BDE8F08F6FF0120009B0BDE885
:10DC8000F08F6FF00F0009B0BDE8F08F03329342C0
:10DC9000E6D16FF0040009B0BDE8F08FD9F80400B8
:10DCA00057F00EFFDCE700BF0B00AD0B0100AE0B21
:10DCB0000000AD0B2DE9F04F804685B0002A40F002
:10DCC000378201F10C0698F80030002B00F0218318
:10DCD000D1F800A001924FF000090C465746CB4600
:10DCE000292B5BD05E2B00F2E981232B3FD9243B0B
:10DCF0003A2B3CD8DFE813F0D8013B003B003B0057
:10DD00008D013B004F012D013B003B0024013B00F6
:10DD10003B003B003B003B003B003B003B003B002B
:10DD20003B003B003B003B003B003B003B00F8005E
:10DD30003B003B003B003B003B003B003B003B000B
:10DD40003B003B003B003B003B003B003B003B00FB
:10DD50003B003B003B003B003B003B003B003B00EB
:10DD60003B003B003B00B00074003B006B002768A9
:10DD7000002E00F08A827B1C23600123F355236868
:10DD80005A1C226098F80020F2544546636801331B
:10DD900063606B7805F10108002BA1D14046BBF10F
:10DDA000000F0DD02368A3EB0B03013B5AB29A423C
:10DDB00018BF49F001095FFA89F90EB106F80B3076
:10DDC000B9F1000F00D0002005B0BDE8F08F236846
:10DDD0005F1C2760002ED8D05022F2542768D4E769
:10DDE00098F80130002BEED0276843F02002642A17
:10DDF00008F1010507F1010100F0F78143F0240368
:10DE0000772B00F0F281002E00F042820123216086
:10DE1000F355236898F80120581CA2F16101206095
:10DE20003344152900F2EE81DFE811F070026D0233
:10DE3000EC01EC01EC016102EC01EC01EC01EC0104
:10DE4000EC01EC01EC016402EC01EC01EC01670275
:10DE5000EC016A02EC01EB0198F8013027685E2BB7
:10DE600007F1010000F0F68108F10105002E00F035
:10DE7000158203232060F355236801332360636810
:10DE80000133636098F801305D2B00F044824FF05D
:10DE9000000C5C2B00F06081002B94D02A46517856
:10DEA0002D2900F0B7812168002E00F0BC814D1CA7
:10DEB000256073542368591C21601178F1545378FC
:10DEC0005D2B02F101050CF1010CE2D14FFA8CF34C
:10DED000634518BF49F001095FFA89F9002E3FF444
:10DEE00058AF06F800C054E72268BA423FF46BAF5F
:10DEF00008F10105002E00F06681B81CD21BF11953
:10DF0000304436F02DFF23680233236098F8013047
:10DF10003F2B0CBF62236123F355236807F10102F5
:10DF2000A3EB0703A3F10203B35459B218BF45464C
:10DF3000994218BF49F0010927685FFA89F925E776
:10DF400027687B1C2360002E3FF41FAF0223F3558C
:10DF50001BE72368BB423FF436AF98F801203F2A05
:10DF600000F08E81002E00F0A48145466222F2541A
:10DF70002368FF1A0133023FF7547AB2BA4218BF3E
:10DF800049F0010923685FFA89F99F1C63682760DB
:10DF900001336360FDE62268BA423FF414AF08F132
:10DFA0000105002E00F0F680B81CD21BF119304498
:10DFB00036F0D6FE2368023360222360F2542168D3
:10DFC0007B1A3144023B4B7021680231216098F882
:10DFD000011058B2984218BF49F001093F290CBFFF
:10DFE00062236123F355236807F10102A3EB0703C2
:10DFF000A3F10203B35459B218BF454627689942AA
:10E0000018BF49F001095FFA89F963680233636058
:10E01000BFE698F8013027683F2B00F01181A36814
:10E0200001335A0051B2914218BF49F00109A3606F
:10E030005FFA89F9002E00F02E81791C21607E2183
:10E04000F1552168481C2060725462680132626098
:10E0500001220292019A039308F101002146FFF781
:10E0600029FE054600283FF4AEAE0278292A7FF447
:10E07000AAAE029B002B3FF48CAE039B5B000133E6
:10E080005AB29A4218BF49F001095FFA89F9226829
:10E09000002E00F01D81511C21607E21B1542268A8
:10E0A000511C2160B35471E623685F1C2760002E69
:10E0B0003FF46BAE5122F254276866E67C2B7FF466
:10E0C00056AE2268BBF1000F34D0A2EB0B03013B2C
:10E0D00059B2994218BF49F001096EB306F80B30E6
:10E0E000226806EB0A050AF102002946A2EB0A02A1
:10E0F000304436F035FE2368F11860200333236086
:10E100008870D4F800B061220BF10103236006F897
:10E110000A202368A3EB0A03023B5AB26B709A42AF
:10E1200018BF49F0010927685FFA89F945466CE78D
:10E130000026C8E5002ED4D1171DA7EB0A03023B29
:10E1400002F1030B5AB29A4218BF49F00109276045
:10E150005FFA89F9454658E76B7843F02001642956
:10E1600005F101026AD043F02401772966D0A3F1BA
:10E17000610115290CD8DFE801F0A9A70B0B0B5D95
:10E180000B0B0B0B0B0B0B5B0B0B0B590B470B5FB1
:10E19000154681E6131DD91BBA1A043A02392360C9
:10E1A0001F4648B253B2884208BF934214BF0123AE
:10E1B000002349EA03035FFA83F998F801303F2B03
:10E1C00018BF454621E702322260D31B174698F854
:10E1D0000120023B3F2A18BF45465AB29A4218BF57
:10E1E00049F001095FFA89F9D0E5002E50D00523E6
:10E1F0002160F35523685A1C226098F80120F254DC
:10E20000C4E50B221A70C1E551782D294FF009039E
:10E210007FF449AE91785D293FF445AE2168023222
:10E22000002E7FF444AE0231216048E60D2336E62D
:10E230000A2334E60C2332E60B2330E6002332E6D1
:10E2400098F802303A2B7FF4EAAE002308F1020876
:10E250000293FFE6002E3ED004232060F35523688E
:10E260000133236063680133636098F802305D2BEB
:10E2700008F1020508BF4FF0000C7FF408AE2DE650
:10E2800008F101054EB3612271E6BB1C23607CE5F9
:10E29000BB1C23607AE5BA1C2260D6E663680133B2
:10E2A0006360BB1C236098F801305D2B7FF4EFADF9
:10E2B0006FE5FF1A023F7AB2BA4218BF49F001096E
:10E2C00045465FFA89F960E60823E8E50723E6E5B5
:10E2D000023222605AE50346C2E7FA1A023A51B204
:10E2E000914218BF49F001095FFA89F94DE60C2205
:10E2F0001A704BE50A221A7048E50D221A7045E59E
:10E3000009221A7042E508221A703FE507221A70A6
:10E310003CE5404658E54FF0000CE2E508B502F058
:10E32000BBF908B1012008BD02F0ACFB70B902F0E6
:10E33000DDFB68B9074B1868C20705D4C303F1D4E5
:10E34000800C00F0040008BD052008BD022008BDB7
:10E35000032008BD7C740120034B53F8203013B117
:10E360009A6801329A607047FC250120114B53F8DE
:10E370002000F0B1017942791F298ABF0E4B4FF07E
:10E38000A04301F01F01D3F810351F2A23FA01F32F
:10E390008ABF09494FF0A04102F01F02D1F81015C1
:10E3A00003F00103D1405B0001F00101194365F066
:10E3B000B3BD7047243C0120000300502DE9F04F0D
:10E3C000ABB0044603910020214646F075FA0028C0
:10E3D00000F03083012120463DF0CCF94268CDE9C0
:10E3E0000C4200230E938DF86030082104A877F0CA
:10E3F00099FB0023CDE90A33DDE90C040EAB0122C1
:10E4000018A9A0470E9B002B40F02C83002800F099
:10E410006C819DF86090DFF8F082DFF8F0B20026A2
:10E420003446B2464D46002D00F066810EAB0C9886
:10E430000D9F012218A9B8470E9B002B40F01283B4
:10E4400008B98DF860007D2D00F256815A2D40F2FA
:10E450005F815B3D222D00F24F81DFE815F0360031
:10E460004D0123004D014D014D014D014D014D0167
:10E470004D014D01F6004D014D014D014D014D0184
:10E480004D014D01B2004D014D014D014D014D01B8
:10E490006B004D014D014D014D014D014D015400E9
:10E4A0004D012300002C00F027810A9B002B00F077
:10E4B000DC82013B0B9A0A9352F82340204640F03D
:10E4C000BDFE82469DF86050ADE70021084642F04F
:10E4D000A3FC054694B18A4B9A451DD0002E00F04E
:10E4E0000B8131462A4620463FF02EFE0B9B00262C
:10E4F000CBB1214608A842F023F8284640F09EFE02
:10E500002C468246DEE7002042F07AFA0546002CCF
:10E51000F4D07B4B9A45E1D12946204642F010F8D1
:10E520000B9B002BE5D1012108A842F05DF80B9B65
:10E530001C60E2E79DF86030722B40F0DD800EAB8E
:10E540000D9D0C98012218A9A8470E9B002B40F0A6
:10E550008982002800F0CD809DF86030752B40F056
:10E56000CB800EAB0D9D0C98012218A9A8470E9BDD
:10E57000002B40F07782002800F0BB809DF86030CF
:10E58000652B40F0B9800EAB0D9D0C98012218A9A7
:10E59000A8470E9B002B40F0658208B98DF86000FB
:10E5A000002C00F01C82564B9A4500F02D82002E64
:10E5B00000F005823E22314620463FF0C5FD002690
:10E5C00080E79DF86030752B40F096800EAB0D9D76
:10E5D0000C98012218A9A8470E9B002B40F04282FC
:10E5E000002800F086809DF860306C2B40F084801D
:10E5F0000EAB0D9D0C98012218A9A8470E9B002B6D
:10E6000040F03082002874D09DF860306C2B73D1BC
:10E610000EAB0D9D0C98012218A9A8470E9B002B4C
:10E6200040F0208208B98DF86000002C00F0CF8106
:10E63000334B9A4500F0E381002E00F0C2810E2298
:10E64000314620463FF080FDB9E79DF86030612BF0
:10E6500052D10EAB0D9D0C98012218A9A8470E9B14
:10E66000002B40F0FF81002843D09DF860306C2BD8
:10E6700042D10EAB0D9D0C98012218A9A8470E9B04
:10E68000002B40F0EF81002833D09DF86030732BD1
:10E6900032D10EAB0D9D0C98012218A9A8470E9BF4
:10E6A000002B40F0DF8120B39DF86030652B23D133
:10E6B0000EAB0D9D0C98012218A9A8470E9B002BAC
:10E6C00040F0D08108B98DF86000002C00F08F81F7
:10E6D0000B4B9A4500F09D81002E00F06E811E22AA
:10E6E000314620463FF030FD69E78DF860008146F5
:10E6F00091E600238DF86030024872F0A9FC00BF5B
:10E700000C590B0090740B000020FF030110000453
:10E710003A2DF1D81F2D40F24A81A5F12002D2B244
:10E720000123934013EA080F40F0AB8013EA0B0378
:10E730007FF4C8AE222DDFD19DF8601005933546D9
:10E740000029D9D022297BD05C2913D004A877F0E6
:10E7500077F80EAB0D9E0C98012218A9B0470E9BBE
:10E76000002B40F07F8110B19DF86010E8E78DF834
:10E770006000C1E70EAB0D9E0C98012218A9B047AE
:10E780000E9B002B40F06E8118B98DF86000014699
:10E79000DCE79DF86010A1F16203132BD6D801A22B
:10E7A00052F823F005E802004DE702004DE70200B1
:10E7B0004DE7020001E802004DE702004DE70200CC
:10E7C0004DE702004DE702004DE702004DE7020071
:10E7D0004DE70200FDE702004DE702004DE70200B1
:10E7E0004DE70200F9E702004DE70200F5E70200FD
:10E7F00009E802000921A9E70D21A7E70A21A5E7F9
:10E800000C21A3E70821A1E74FF0000904260EAB75
:10E810000C980D9F012218A9B8470E9B002B40F0C1
:10E820002181002840F0A3808DF86000C923013EBB
:10E8300043EA0919EBD1494604A877F02BF888E799
:10E840000EAB0C982E4601220D9D18A9A8470E9BD1
:10E85000002B40F0078108B98DF86000DDE9051054
:10E8600042F086FB0246002C51D0834B9A4500F0C3
:10E870009780002E00F08780314620463FF064FCF0
:10E880009DE6002305939946294604A876F0D8FF13
:10E890009DF86050452D15D82A2D15D9A5F12B03CB
:10E8A0001A2B11D8DFE803F01410142310101010E5
:10E8B0001010101010101010101010101010101058
:10E8C00010102300652D12D0284672F0AFFA88B1DF
:10E8D0000EAB0C980D9F012218A9B8470E9B002B78
:10E8E00040F0C0800028CFD18DF86000CCE74FF019
:10E8F0000109EDE70346DDE90510B9F1000F44D049
:10E900001A46009345F098FB0246002CADD1914683
:10E9100040F094FC039BDBB99DF8600072F0AEFA06
:10E9200088B10EABDDE90C04012218A9A0470E9BAB
:10E93000002B40F097800028EED18DF8600072F037
:10E940009DFA0028EDD19DF86030002B7FF4D4AE05
:10E95000B9F1000F3FF4D0AE0A9B002B7FF4CCAE90
:10E9600004A877F05FF848462BB0BDE8F08F9DF81B
:10E97000602042F02002A2F13003DBB2092B84BFF9
:10E98000573AD3B253E716469CE50A224B4645F068
:10E9900085FC0246002CBAD0374B9A457FF469AF0C
:10E9A0001146204641F0CCFDDFF8CCA08AE50A2DC7
:10E9B00009D8082D3FF686AD9EE61E2682E53E2646
:10E9C00080E50E267EE50D2D3FF47CAD94E60E200D
:10E9D00040F034FC039B4BBB4FF00E099CE73E20FC
:10E9E00040F02CFC039BCBB94FF03E0994E71E206E
:10E9F00040F024FC039BABB94FF01E098CE70E21BD
:10EA0000204641F09DFDCFE73E21204641F098FD94
:10EA1000CAE71E21204641F093FDC5E70A9B4FF04F
:10EA20003E099AE70A9B4FF01E0996E70A9B4FF0B2
:10EA30000E0992E70FAA20467E2100260027CDE985
:10EA400016673EF005F90D4A0D4B12920121402246
:10EA5000CDE913120CAC1AA912AACDE90C431591F9
:10EA60001192C2E4184672F08FFA039BA146002B64
:10EA70007FF476AF50E700BF0C590B00084D0B0038
:10EA8000A90806000288112A0B4608D0362A0BD1A5
:10EA900019B181889A89914208D0012070474FF6B8
:10EAA000FF71012299811A740020704700B5C28855
:10EAB00083B0DA81C289009300F110015868824264
:10EAC00028BF02461868019236F016F9DDE90032D7
:10EAD000012101209A60197403B000BDC2070346EA
:10EAE00020D400B510F0030283B00BD1114A0168A5
:10EAF00091421AD0184640F0A1FB5E22C1880E4810
:10EB000072F09AFA022AF5D10C4A0240062AF1D094
:10EB100040F0ACFAFCEEC07ACDED017A9DF804002D
:10EB200003B000BDC0F34700704740F061FBC0B2C6
:10EB3000F6E700BFE4570B009C810B00070080FF45
:10EB400070B588B014460DF11E030DF11F02CDE91A
:10EB500000320E460DF11D0307AA214604460EF0B1
:10EB600079F89DF81C209DF81D300B490592204630
:10EB700004939DF81E409DF81F503EF0F1FF039056
:10EB80003EF0F2FECDE90045DDE90432039831465E
:10EB90005BF056FF08B070BD6CC30B002DE9F04F61
:10EBA0000446E3B0674812F089FCB0F1000A21DBAB
:10EBB000654E7388B3F57F7F80F0B2801A1DA24244
:10EBC0001CD85A1E341D6148A15C614D2F290BBF12
:10EBD00000230022A354E25405A92BF073FB286004
:10EBE00010B12BF0A3FC68B940F25133504633808A
:10EBF00062F07CF9002063B0BDE8F08F012063B0C3
:10EC0000BDE8F08F2868059A803006A97CF0FFFBEC
:10EC10000023C6E90133F36040F25113054644F87E
:10EC2000043C002840F082801AA906A87CF0DFFC92
:10EC3000044620B180E07CF0DAFC013428B99DF86C
:10EC400082301AA906A8002BF5D1002106A802944B
:10EC50007CF0CDFC029BB360002B54D04FF0000B36
:10EC60000DF18207D846CDF80CA01AA906A87CF0B1
:10EC7000BEFCBDF87230BDF87010C6F804B003F0E9
:10EC80001F0252000192480AC3F344120092DB0AA9
:10EC900001F01F0200F2BC70C1F343116DF064FC7F
:10ECA0009DF874302B4A13F01003A0FB0202C6E952
:10ECB000040214BF01231A9AF36018BF00223846D9
:10ECC000B26168F04BFC05467080039862F00EF963
:10ECD00095B10024A5EB040ABAF1040F28BF4FF048
:10ECE000040A39191748CDF80080002352465444CD
:10ECF00012F0C2FCA542EDD8029B0BF1010B9B4523
:10ED0000B3D1DDF80CA006A87BF0A6FE0023B26804
:10ED1000738050467260F360B36162F0E7F869E7B0
:10ED200040F25123338062F0E1F863E70323504659
:10ED3000737062F0DBF85DE7294606A87CF057FCAB
:10ED4000B560E0E71045012000480120044801209B
:10ED50008846012000CA9A3B38B52B4A2B4B044603
:10ED6000012110681D6856F09BFD294A02F1200C14
:10ED700052F8043F13B11979A14202D06245F7D18C
:10ED800038BDDA791ABB5A699969AA1A411AC2EBD5
:10ED900002420A444FF6FF718A4228BF0A46D989C7
:10EDA0001C8AA4B214FA81F19C89B1FBF4FC04FB27
:10EDB0001C119C6824F811201A8A998992B28A42FF
:10EDC00018D21A8A01321A825D61986138BD1F2CEF
:10EDD00088BF104A597994BF4FF0A04204F01F0435
:10EDE000D2F81025E24002F001029142ECD000225C
:10EDF000DA71E9E7DA8992B20132B2FBF1F401FB90
:10EE00001422DA81E0E700BF147601204C7401205F
:10EE10000C0A0120000300502DE9F04110F8017C9C
:10EE20000578A7F10306B6FA86F67609CDB18846CD
:10EE3000841C06E000F01CF880B9013D04F10204D6
:10EE40000FD014F8013C41462046002BF2D098F830
:10EE500000209342F1D823789342EED33046BDE8A8
:10EE6000F081FE1E18BF01263046BDE8F08100BFCC
:10EE700003780A7843F020016429C3F340101DD0C1
:10EE8000732910D022F02001413919290AD9A2F1A1
:10EE90003001092906D96FEA531303F001035F2AF1
:10EEA00018BF18467047202AFCD06FEA5313093A5E
:10EEB00003F00103042A88BF184670476FEA531312
:10EEC000303A03F00103092A88BF1846704700BF93
:10EED0002DE9F04F95B0814600F15804D0E91403B4
:10EEE00000AF5B6821469847D9F8583033B109F133
:10EEF000080318463B6226F0D9FC18B95437BD46C2
:10EF0000BDE8F08F99F84810002940F0A381D9F8A6
:10EF10000800002800F01C8126F026FE8346002809
:10EF200000F01681B9F838305A2B6D4600F08F8109
:10EF3000B3F5877F00F08B81B9F836200732D21005
:10EF4000D31D23F00703ADEB030D0021684636F017
:10EF5000B7F8D9F85430D9F850005B682146984783
:10EF6000EA464FF001087D60C7F82C90386AC7F870
:10EF70000CD007F13802594626F0A2FB002800F019
:10EF8000D680FB6A93F83A10072915D893F84430D5
:10EF900093B1B7F93C200823B3FBF1F31A44013ACB
:10EFA00092FBF3F212FB03F2BA87B7F9382092FB17
:10EFB000F3F202FB03F33B8707F1380025F088FBEF
:10EFC000FB6A786307F1380093F83A402023B3FBDB
:10EFD000F4F425F09FFB054607F1380025F09AFB75
:10EFE000B0EBC41F4FEAC41600F2B980C5F34A1350
:10EFF00001339B007B610733ADF5007D23F00703F0
:10F00000C7F828D007F13800ADEB030DC7F810D0D2
:10F0100025F05EFB4FF400720123C7E90623844606
:10F0200000253D63C7F808B0C7F824C07A6A786B3A
:10F03000398F3E69A7F844100023521B92B2FB643B
:10F040007B8F904203EB050188BF7A6AA7F84610D0
:10F0500098BF1B18B7F93C10A7F848108CBF9B1835
:10F060005B197A69A7F84A300021304636F028F853
:10F07000BC6ABA690021204636F022F8234632469F
:10F08000386A07F1440126F05FFBB7F94620B7F96B
:10F090004A3094B29C423CDAF96AB7F9440091F8DC
:10F0A0003A30B1F87660B1F87410D7F828B006FBA2
:10F0B000021113FB00F2002AB8BF073201EBE20194
:10F0C000B7F94820121A03FB02F2FB6A002A9B6D73
:10F0D000B8BF073201340B444FEAE209A4B2601E04
:10F0E000C0F3CC0200F007001AF8021008FA00F092
:10F0F00008430AF80200594618464A4635F0FCFD16
:10F10000B7F94A10A14200EB0603CB4404F1010415
:10F11000E5DC05F079FC73F08DF87A6B3B6B1544F8
:10F12000FA6901339A423B6380D1D7F808B0DBF823
:10F1300008B0D7F80CD0BBF1000F7FF417AFD7F8A9
:10F140002C907D68D9E9140351469B689847AD46D9
:10F15000386A26F009FB5437BD46BDE8F08F07F149
:10F16000380025F091FBFA6AB6FBF0F692F83A30D7
:10F17000002E57D0B1B2072B79630CD892F84420F7
:10F180004AB9796B0822B2FBF3F2B1FBF2F302FB4E
:10F1900003F39BB27B6307F1380025F099FA7D6B8E
:10F1A000B0FBF5F307F138009EB225F091FA721C1E
:10F1B000B0FBF5F303FB150392B29BB2002B14BF17
:10F1C00011463146F96107F1380025F05DFB7B6B94
:10F1D00010FB03F39BB2B3FBF4F204FB12340CB14B
:10F1E000013292B292005B09BA6101339A00BB69A5
:10F1F0007A61073323F00703ADEB030DD31DDB0862
:10F200006A46A2EBC303C7F828D007F138009D4631
:10F21000C7F810D025F05CFAFB698446002B7FF418
:10F22000FFAE84E7072B06D8FA6A92F8442012B999
:10F2300001227A63A5E707F1380025F049FAF86161
:10F2400007F1380025F044FA01237B63BBE7B9F8E6
:10F25000342073E60023C9F8303009F1280B61E649
:10F260002DE9F04F00F1080B93B0814602AF5846EC
:10F2700026F01CFB18B94437BD46BDE8F08F99F85D
:10F280004810002940F04C81D9F80800002800F00F
:10F29000D68026F069FC8446002800F0D08009F171
:10F2A000B2037B60C7F81CB0C7F808C0B968F8693A
:10F2B00007F128026D4626F003FA002800F0B68018
:10F2C00007F1280025F004FA044607F1280099F810
:10F2D0003A8025F01FFA99F8822083B2002A00F0C4
:10F2E000B780C4F3CF027A614FF40072BA61082488
:10F2F0005B0901339A00BB693A61073323F00703C6
:10F30000ADEB030DD31D23F0070302AEADEB030DF0
:10F3100002AB07F12800FB6025F0DAF97B6986462D
:10F32000002B00F003814FF0000A3D60D04609F148
:10F33000500B3546C7F820E049E025F0EBF999F885
:10F340003A60F60816FB00F6B3B27B62D7E90362B7
:10F350000021304635F0B4FEBA690021284635F068
:10F36000AFFE3246FE692B4607F13401304626F0E7
:10F37000EBF9584607F13402314626F031F8584689
:10F3800025F084FF002861D099F8801041B901234D
:10F39000D9F8500000931A46D9F860607B68B047EE
:10F3A0007B6AD9F85000009300222B460121D9F83E
:10F3B0006060B047584626F001F805F025FB72F072
:10F3C00039FF7B6908F101084345A2442AD0798DB1
:10F3D0003B8DBB860AEB0102FA863A6AB7F92C60CC
:10F3E0003E87A2EB0A02002392B2A242FB6301EB2A
:10F3F0000403534499F83A203CBF3B6ACB18072AD0
:10F4000007F134007B8798D807F1340025F082F9A2
:10F4100099F83A300822B2FBF3F3B0FBF3F6B3B23B
:10F420007B6293E73D68584625F0CCFFBB689B683C
:10F43000BB60AD46002B7FF439AFD7F81CB05846FF
:10F4400026F092F94437BD46BDE8F08F3D68EDE700
:10F4500007F128007B6225F05DF92026B6FBF8F65F
:10F46000B0EBC61F7B6A4FEAC61818D85B09013398
:10F470009B003B610733ADF5007D23F0070302AE2F
:10F48000ADEB030D02AB07F12800FB6025F020F97E
:10F4900001234FF40072C7E90532864643E707F1BE
:10F4A000280025F0F1F999F83A20B8FBF0F000288F
:10F4B0003FD0072A84B20AD899F844303BB90823D0
:10F4C000B3FBF2F2B4FBF2F302FB03F39CB207F1DD
:10F4D000280025F0FDF8B0FBF4F307F1280099B2FD
:10F4E000796125F0F5F87969B0FBF4F34A1C03FB68
:10F4F000140392B29BB2002B18BF1146796107F139
:10F50000280025F0C1F910FB04F39BB2B3FBF6F21F
:10F5100006FB12360EB1013292B29200BA61E7E6F2
:10F520000023C9F8303009F1280CB8E609F1500B76
:10F5300079E7072A02D899F8443053B107F1280037
:10F5400025F0C6F8786107F1280025F0C1F80124FC
:10F55000D5E70124B3E700BF2DE9F043884690F8D2
:10F560002A1011F0100785B06BD14368DB680446A0
:10F5700053F8281040F2165045F09EF90646002830
:10F580005DD06368DB6853F8280073689847B368F8
:10F5900001A95B6881469847B36839469B68054670
:10F5A00048469847B36839469B6948469847636818
:10F5B0002549DB6853F828003EF0D2FA064668B1C8
:10F5C00090F8503023F0100301A980F8503027F054
:10F5D000A7F900210546304627F064FD63681B4902
:10F5E000DB6853F828003EF0BBFA064668B190F895
:10F5F0002A3023F0020301A980F82A3026F05EFAAF
:10F6000000210546304626F06BFD7DB194F82A3086
:10F61000DB070ED504F1180201A9104625F0E6F823
:10F6200094F82A3043F0010384F82A3005B0BDE88D
:10F63000F08304F1180101A825F00CF8F0E7054665
:10F64000B5E70CF077FC00BF00EC0B004CE90B00B9
:10F6500070B586B005460191164619F0FDF990B9CE
:10F6600001983FF071FD0622044603A930463CF0A4
:10F670000BF803AA2146284619F004FA002804DBF7
:10F680000E2006B070BD5EF041FA404271F07CFC85
:10F6900070B586B005460191164619F0DDF990B9AE
:10F6A00001983FF051FD0522044603A930463BF086
:10F6B000EBFF03AA2146284619F040FA002804DB94
:10F6C0000E2006B070BD5EF021FA404271F05CFC85
:10F6D000242B2DE9F047884601D8012B06D1FCF7F1
:10F6E000B1FB162303600020BDE8F087344E0D46C1
:10F6F000294615F8014B375D17F00807F8D12D2C76
:10F7000010D12C7801278D1C33F0100115D1302C2D
:10F710000DD1297801F0DF01582908D16C78023524
:10F7200010230AE02B2C04BF2C788D1CECE7002B57
:10F73000F6D1302C14BF0A23082307F1004E0EF136
:10F74000FF3E0021BEFBF3F90E4603FB19EAA4F1CC
:10F75000300CBCF1090F10D86446A3421EDDB1F194
:10F76000FF3F07D0B14516D301D1A24513DB06FBFD
:10F770000346012115F8014BE9E7A4F1410CBCF166
:10F78000190F01D8373CE8E7A4F1610CBCF1190F5F
:10F7900004D8573CE1E74FF0FF31EBE74B1C05D1B4
:10F7A00022230360764632B930469DE707B17642A0
:10F7B000002AF9D009B105F1FF38C2F80080F3E75B
:10F7C0007D7D0C002DE9F043344E86460D462846DB
:10F7D00015F8014B375D17F00807F8D12D2C10D123
:10F7E0002C780127851C33F0100015D1302C0DD159
:10F7F000287800F0DF00582808D16C7802351023F3
:10F800000AE02B2C04BF2C78851CECE7002BF6D1EA
:10F81000302C14BF0A2308234FF0FF380026B8FB12
:10F82000F3F803FB08F96FEA09093046A4F1300C3C
:10F83000BCF1090F10D86446A3421EDDB6F1FF3FAC
:10F8400007D0804516D301D1A14513DB00FB03404F
:10F85000012615F8014BE9E7A4F1410CBCF1190FA1
:10F8600001D8373CE8E7A4F1610CBCF1190F04D8CA
:10F87000573CE1E74FF0FF36EBE7731C06D122233C
:10F88000CEF80030304632B9BDE8F08307B14042CF
:10F89000002AF9D006B1691E1160F5E77D7D0C00E4
:10F8A000F0B583B004460D4601926AF0CDF8636866
:10F8B000019A07460120587260680E46294656F0A4
:10F8C0001FFA134B984204D0636800225A7203B0A7
:10F8D000F0BD17F57A7546F1000605E06AF0B4F858
:10F8E000854276EB01010CD363685A7A002AF5D180
:10F8F0009B7A042B96BF074A074852F8230003B0AF
:10F90000F0BD6368054800225A7203B0F0BD00BF25
:10F910000000AD0B68B10B000100AD0B0700AD0B93
:10F92000F8B543689A6852B3054600240BE0736843
:10F930009847B36805F108019B6898476B689A6817
:10F94000013494421BD2DB6840F2165053F8241065
:10F9500044F0B2FF6B68DB680646A70053F824004A
:10F96000002EE4D10D493EF0FBF848B105F1080145
:10F9700027F098FB6B689A6801349442E3D3F8BD92
:10F980006B680749DB68D8593EF0EAF80028D5D003
:10F9900005F1080126F0A4FBD0E700BF00EC0B0046
:10F9A0004CE90B0090F950302149B0F90C2000B51A
:10F9B000002B836AB4BFB0F812C0B0F810C0002B9F
:10F9C00008BF0B469444997B92B2C1B193F90510DC
:10F9D00011FB02F259880A4412B2A0F8462093F9AA
:10F9E0000510B3F802E011FB0CE31BB29A42D2BF40
:10F9F000A0F84A30A0F84A20A0F8463000BD93F99C
:10FA0000041011FB02F219880A4412B2A0F8442033
:10FA100093F90410B3F800E011FB0CE31BB29A4217
:10FA2000D2BFA0F84830A0F84820A0F8443000BD6C
:10FA30001C03012090F950302149B0F90E2000B587
:10FA4000002B836AB4BFB0F810C0B0F812C0002B0E
:10FA500008BF0B469444997B92B2C1B193F904104C
:10FA600011FB02F219880A4412B2A0F8442093F95B
:10FA70000410B3F800E011FB0CE31BB29A42D2BFB2
:10FA8000A0F84830A0F84820A0F8443000BD93F911
:10FA9000051011FB02F259880A4412B2A0F8462060
:10FAA00093F90510B3F802E011FB0CE31BB29A4284
:10FAB000D2BFA0F84A30A0F84A20A0F8463000BDD6
:10FAC0001C03012010EE102A22F00043B3F17E5FE8
:10FAD00005D34BD1002A71DB9FED5C0A7047B3F16F
:10FAE0007C5F05D2B3F14A5F47D89FED590A704752
:10FAF00000B5002A83B0F7EE007A62DB77EEC07AB9
:10FB0000B6EE007A67EE877AF5EE407AF1EE10FAFB
:10FB100000F18580B1EEE76ADFED4E6A9FED4E5A47
:10FB20009FED4E7A9FED4E4AA7EEA65A16EE103A7A
:10FB30006FF30B03A7EE857A06EE903AF0EE674A74
:10FB4000F7EE005AE7EE845AE6EEE64A36EE865ABB
:10FB500067EE277A84EE850A87EEA57AA7EE060A75
:10FB600030EE260A30EE000A03B000BD70EE407A97
:10FB70009FED367A87EE270A704760EE006A9FEDA8
:10FB8000356ADFED357A9FED357AE6EE867A9FEDC0
:10FB9000346AA6EEA77AF7EE005AE6EE865A27EE0A
:10FBA000267ADFED2B7AC7EE256A9FED2E7AA0EE3E
:10FBB000667A30EE470A37EEC00A70479FED2A0A90
:10FBC000704730EE270AF6EE007A60EE277AF5EEFF
:10FBD000407AF1EE10FA2DD4F1EEE75A9FED1D6A4E
:10FBE0009FED1D7ADFED1D6A9FED1D5A9FED180AEE
:10FBF000A7EE867AB7EE006AE7EE876AA7EE856A17
:10FC000066EEA77AC7EE866ADFED187AE6EEA57A89
:10FC100077EEA57A30EE670A30EE000AA4E7B0EE80
:10FC2000670ACDED017A65F049FBDDED017AB0EEB2
:10FC3000406A71E7B0EE670ACDED017A65F03EFBF0
:10FC4000DDED017AF0EE405AC8E700BF0000000089
:10FC5000DA0FC93F6BD30DBCBA132FBD75AA2A3E6C
:10FC6000AEE534BF6821A233DA0F49406821A2B360
:10FC700000B510EE103A5A0083B0F0EE407A26D567
:10FC800023F00043B3F18B4F07D333F023F9DFEDBB
:10FC9000267A30EE270A03B000BDBFEE000AA7EEB9
:10FCA000A70A77EEA76AB5EE400AF1EE10FA24D45F
:10FCB000B1EEC07A77EE877AB7EE007A87EE270A40
:10FCC00036EEC00A03B05DF804EB33F003B9B7EECB
:10FCD000007A70EE477A37EEA77AA7EEA77AB5EEEC
:10FCE000407AF1EE10FA15D4B1EEC70A37EE800A69
:10FCF00003B05DF804EB33F037B8CDED017ACDED0C
:10FD0000006A65F0DBFADDED017ADDED006AB0EE48
:10FD1000407ACFE7B0EE470ACDED007A65F0CEFA33
:10FD2000DDED007AE2E700BF1872313F30B50846DA
:10FD300087B011461A460F4B0DF10C0CCDE9003C73
:10FD4000032336F0DFF80C49039C0C2040F05CFDE7
:10FD50009DF81020214605460CF02CFD9DF814302E
:10FD600013B9284607B030BD28460CF045FD28469B
:10FD700007B030BDB0C10B0028C20B0000B583B086
:10FD800001900CF01BFD019803B000BD08B5086898
:10FD90000CF05EFD0E2008BD10B58EB003AB51F81F
:10FDA000044B0193184B00930138032336F002F8FB
:10FDB000606840F2335106AA3CF04AFF227A049B65
:10FDC000039C0994520042F001020892059A6FF0D8
:10FDD00000415B0040F6261043F001038A420A907E
:10FDE0000B930ED0520040F2E64342F00102CDE9FF
:10FDF0000C32022106AA022037F0B4FF0E200EB00A
:10FE000010BD0121F6E700BFC8C10B0010B58EB0D0
:10FE100003AB51F8044B0193184B009301380323B3
:10FE200035F0C8FF606840F2946106AA3CF010FF0C
:10FE3000227A049B039C0994520042F0010208922A
:10FE4000059A6FF000415B0040F6261043F0010375
:10FE50008A420A900B930ED0520040F2E64342F0E1
:10FE60000102CDE90C32022106AA022037F07AFF06
:10FE70000E200EB010BD0121F6E700BF10C20B002E
:10FE800030B597B002AB51F8044B01932F4B009360
:10FE90000138062335F08EFF606840F2956108AAAC
:10FEA0003CF0D6FE049B227A029C0B945B0043F04C
:10FEB000010352000E93059B42F001026FF00041D6
:10FEC00044F6B6500A928B42039A0D900C9234D0AD
:10FED0005B0044F6865143F001030922CDE90F137C
:10FEE0004FF00B0E4FF00A0C14460321069B0DEB4E
:10FEF00082000DEB8C0C5B0043F00103079A44F287
:10FF000066250562CCF820306FF000439A420DD090
:10FF10000DEB8E0E0DEB8404520042F00102013114
:10FF200044F23623CEF82030C9B2E26208AA032098
:10FF300037F018FF0E2017B030BD07224FF0090E22
:10FF40004FF0080C14460221D0E700BFE0C10B00BF
:10FF500010B508468EB011461A46174B0DF11C0C11
:10FF6000CDE9003C072335F0CDFFDDE9074013491B
:10FF700040F2153236F01EF908980E2803D0002200
:10FF8000012113F093F90E49182040F03DFC9DF833
:10FF900034209DF830300590CDE902329DF82C20B8
:10FFA0000A9B2146CDE900329DF82430089A0CF0D6
:10FFB0005FFC05980EB010BDB4C20B0090E40B00BE
:10FFC000ECC20B000CF066BC08B508680CF0B2FC83
:10FFD0000E2008BDF0B5054685B001F134000E468F
:10FFE00004F076FC2B88102B2FD0112B2AD1002265
:10FFF000A888424C134634F81210814202F14402A0
:020000023000CC
:1000000003D00133052BF6D1042303EB031304EBD8
:10001000C3013B480193009107F072FD019B0099D9
:100020004FF6FF7224F83320CB6D00220E2B81F89F
:100030005A2002D05A602A7A1A720023B361012032
:1000400005B0F0BD002005B0F0BD00222B4C1346DA
:100050004FF6FF7034F81210814202F1440203D0CF
:100060000133052BF6D1042303EB0312D700A88834
:10007000E05304EBC202002082F85A00A2F8760096
:100080000E20D065E87B009219010B44022804EB96
:10009000C30314BF96F845000120D87007F108008B
:1000A0004FF000024FF6FF71204483F87820A3F848
:1000B000581083F8792009F0EDFB07F16000009AF1
:1000C0000F49204407F0F2FC0023B36128696969F5
:1000D00007F16C03234403C302A860F07FF9BDF865
:1000E00008302A8A9A4202D86A8A9A4203D2A88899
:1000F00002A960F05BF90023F360A0E7A00A0120E9
:10010000B107050038B50388102B0C4618D0262BF4
:100110002ED11A4B1878FF2810D060F041F92146F3
:100120000546174807F0ECFC0023E36084F84430F0
:1001300035F00803284601D00BF052FE012038BDEF
:1001400081880022032060F057F90C4B1878FF28B3
:100150000ED060F025F921460546094807F0D0FC8D
:100160000023E36084F8443035F00803284601D1C9
:10017000002038BD0BF034FEFAE700BFA7060120CF
:100180000501030030B587B0044615460846052230
:1001900069463BF079FA03A9062228463BF074FA37
:1001A0000199049A204674F01FF8DDE900120398C3
:1001B00034F0A2FD2046DDE903120CF039FF0E20D9
:1001C00007B030BD30B587B0044615460846052255
:1001D00069463BF059FA03A9062228463BF054FA37
:1001E0000199049A204673F0FFFFDDE9001203989D
:1001F00034F082FD2046DDE903120CF02BFF0E20C7
:1002000007B030BD90F80C01400040F0010070478D
:1002100070B508468CB011461A46224B07ACCDE9A2
:100220000034052335F06EFE0522079804A93BF043
:100230002BFA059DA5F11002102A30D81A4BD34095
:10024000DB072CD5089C022C1CDD062C1CD1099840
:10025000049E20B104A901223BF016FAB8B9034666
:10026000124903934FF48A7040F0CEFA00940A9C2E
:10027000039B01942A46314602900CF0B7FE029887
:100280000CB070BD002CE2DC094870F069FE0598E6
:100290004FF4B772102135F0A1FE049BE0E705484A
:1002A00070F0D6FEE0C40B000101010018C50B0080
:1002B0009C880B00308C0B0070B551F8043B88B063
:1002C0001D4603AB0193184B00930138022335F010
:1002D00071FD0522039805A93BF0D6F9069CA4F10F
:1002E0001002102A1CD8114BD340DB0718D5DDE9CA
:1002F000040620B105A901223BF0C6F940B9034626
:100300002846224631460CF0B7FE0E2008B070BDDC
:1003100006984FF4B772102135F060FE059BEFE7A9
:10032000034870F095FE00BF08C50B0001010100F5
:10033000308C0B0010B5044608463EF005FF02283D
:1003400007DD062807D1014620460CF0B1FE0E203D
:1003500010BD0028F7DC014870F002FE9C880B00FD
:1003600030B5114B87B005ADCDE90035044601230A
:1003700000200D4635F01EFD2946204674F084F815
:10038000059840F097F8421004D0084840F20B510D
:1003900070F0EEFD2946204604AB03920CF03EFFC0
:1003A000039903487CF069F9D8C50B0018950B0038
:1003B000EC500B0010B90E231846704730B50D46AF
:1003C00083B0044674F060F8294620460CF092FE93
:1003D0000022019046F2B67104483CF0B1FD019B49
:1003E00000B14360184603B030BD00BF6C0001206F
:1003F000E0B130B50F4BDFF840C01C780439002263
:1004000001E090420FD051F8043F9D0702F1010234
:10041000F7D11D686545F4D15D6895F804E0A645FF
:10042000EFD1184630BD0E23184630BD0E231846B6
:10043000704700BF4C7B012098C60B0010B50846E2
:1004400088B011461A46104B0DF1100CCDE9003C56
:10045000042335F057FD049840F2F74173F0D0FFC4
:100460000A4904460C2040F0CFF99DF81C20009268
:100470009DF818309DF81420039021460CF088FE5A
:10048000039808B010BD00BF78C60B0098C60B00DB
:1004900008B50CF091FE002808BF0E2008BD00BF73
:1004A00008B50CF08BFE00280CBF1E203E2008BDB6
:1004B00008B5054B1A7802B108BD20F0A1F8024B2F
:1004C00001221A7008BD00BF137B01200E4A0F499C
:1004D000506810B50E4C0023C008C4E9001310D0BA
:1004E0000C49D26891F800E002F1040C01E083426B
:1004F00007D05CF833201179714503F10103F6D17F
:100500006260034810BD00BF88B20B0098C60B00A4
:10051000904601204C7B01202DE9F041184F194EE7
:1005200000240125D6E90001D7E90032A4F1200C0E
:10053000C4F1200805FA0CFC25FA08F803430A4325
:100540004CEA080C05FA04F10B4002EA0C021343D2
:10055000E0B207D05EF01AFE204654F05BF8204669
:1005600054F090F90134402CDCD1074900220023DB
:10057000C7E90023C6E90023C1E90023BDE8F081F3
:100580004011012050110120D8110120002975D0FF
:100590002DE9F04F3A4B1C685E683A4B87B0D3E9BF
:1005A0000098394B009400251C680194043ACDE969
:1005B0000255CDE904505F68344C02EB81014FF0E5
:1005C000FF3C4FF0010E01E091422CD052F8043F65
:1005D0009807F9D11868A042F6D1586893F808B086
:1005E00090F804C0ACF12000CCF1200A2EFA0AFAEF
:1005F0000EFA00F040EA0A000EFA0CFABBF1000F06
:100600002FD049EA0A0948EA0008CDF808B05B7A19
:10061000002BD9D0019D049345EA0A05914201952A
:1006200047EA0007D2D1DDE904501DB1164B019A0B
:10063000C3E90027039B1BB1114B009AC3E90026B5
:10064000029B13B10F4BC3E90098BCF1FF3F05D0EB
:1006500078B10F490F4A00230B60137007B0BDE853
:10066000F08F009D45EA0A05009501250643039594
:10067000CDE707B0BDE8F04F1FF0C2BF704700BF25
:100680005011012040110120D811012098C60B0003
:100690007C740120137B0120054B1B78012B01D0BA
:1006A00000207047034B1878FF3818BF01207047AF
:1006B0004D7B01204C7B012008B500F009F8FFF7C5
:1006C0002BFF00F0D3F9BDE8084000F00BBA00BFE3
:1006D00010B5124C124A23686FF3172393421CD0B3
:1006E0004FF4807200210F4834F0EAFC0E490F4BA2
:1006F00000220A701A704FF080404FF4403113010D
:1007000003F180430132082AC3F80419F7D1044BDE
:100710004FF47C12C0F88429236010BD487B01206F
:10072000AF0000AD507B01204D7B01204C7B0120B0
:10073000002A75D070B514468A0788B005460B4666
:1007400003D1464A0968914230D028462E68019369
:100750000CF092FD019A0146002330463AF0CEFF9C
:10076000042C064615D020463EF0EEFC4223FF2224
:100770000021044635F022FC012305AA3146284613
:100780008DF814400CF07CFD002846D00E2008B0F7
:1007900070BD01460123284605AA0CF05DFD9DF8B9
:1007A0001400400040F0010008B070BD01930CF04F
:1007B00063FD019902AA45F00FF8002844D0DDE955
:1007C0000232042CA2EB03062FD0A3072AD1236800
:1007D000234A934208D0234A934205D0224A9342A7
:1007E00002D0224A93421DD1052205A920463AF0A3
:1007F0004BFF069BB3422DD19DF81C10059C002297
:10080000402035F00DFD012821D1029933462246C2
:1008100028460CF035FD0028B8D1154870F0E4FBEF
:1008200010467047134870F09BFB304632F046FC90
:10083000029904460246334628460CF00DFD214637
:10084000304640F01BF8A2E70B4870F089FB0B48DC
:1008500070F0FEFB0A4870F0FBFB00BF6C600B0001
:100860008C4C0B00084D0B00C04C0B0038630B0088
:10087000CC850B0004830B0070770B00CC910B0030
:1008800044880B0010B5044608460CF0F5FC042C17
:1008900009D0052C01D0002010BD064B03EA400012
:1008A00040F0010010BD80B200280CBF1E203E2089
:1008B00010BD00BFFEFF0100F0B1DFF84CC00439ED
:1008C000002351F8042F12F0030F03F1010311D19B
:1008D00010B4146864450AD0984210D051F8042F1F
:1008E000940703F10103F7D114686445F4D110466D
:1008F00010BC70479842E4D10E22104670470E2279
:10090000104610BC704700BF14C70B0038B5084B29
:10091000D3E9004554EA050305D019F06DFE201A0D
:1009200065EB010138BD4FF0FF30014638BD00BF17
:100930000012012010B52DED028B08468AB0114639
:100940001A46324B05ACCDE90034022335F0DAFA11
:10095000DDE90504B0F10E0218BF0122B4F10E0367
:1009600018BF01239A424BD00E2846D03EF07EFBA2
:10097000B0EE408A19F040FEF6F72CFE9FED247A87
:1009800006EE900A0E2CC6EE877A23D00698CDED9F
:10099000037A3FF06FFA04465EF0D4FF07A966F0D1
:1009A000F5FE9DF822009DF821109DF820309DF85D
:1009B0001F20CDE900109DF81E10BDF81C006BF043
:1009C000A9FE231A08EE103ADDED037AB8EEC88AC4
:1009D00038EE278AB4EEE78AF1EE10FA13D40D4907
:1009E00008203FF011FFB0EE480A04460CF05AFC14
:1009F00020460AB0BDEC028B10BD9FED078AB9E717
:100A0000064870F025FB064870F022FB04C70B0077
:100A100000007A4414C70B0000000000D8870B00C8
:100A2000E8860B0008B50CF041FCB4EE400AF1EE8C
:100A300010FA08D610EE103A23F0030040F002003E
:100A4000A0F1FF4008BD014808BD00BF0200400002
:100A5000704700BF0349044A0A6000234B60084600
:100A6000704700BF9046012014C70B0008B5012055
:100A70005AF0E0FD024B00200021C3E9000108BD4F
:100A800000120120034B1878A0F10200B0FA80F0A8
:100A9000400970474D7B012010B5084686B01146CD
:100AA0001A460C4B0DF1140CCDE9003C012335F036
:100AB00029FA059840F2F74173F0A2FC0649044672
:100AC00008203FF0A1FE214603900CF0F3FB0398B1
:100AD00006B010BD60C70B0068C70B0040687047C8
:100AE0000E207047704700BF704700BF002070475E
:100AF00010B5094B094C1B680BB1A34208D1C022A9
:100B00000021074834F0DCFA40F8044C043810BDEA
:100B1000044870F069FA00BFA84C0120E05D0B00AA
:100B2000AC4C0120B4860B0010B5094B094C1B6876
:100B3000A34203D013B1084870F056FAB422002142
:100B4000064834F0BDFA054B43F8044C181F10BD9D
:100B5000C80D0120E05D0B00AC860B00CC0D012020
:100B6000164B0122002186B0C3F80025C3F81011EE
:100B7000D3F8101101910199DA60D3F81021002AFD
:100B8000FBD00022C3F81021D3F81011059105996C
:100B9000C3F80421D3F8041104910499C3F808217F
:100BA000D3F8081103910399C3F80C21D3F80C1161
:100BB00002910299C3F8002506B07047007000400A
:100BC00008B50CF0B3FB0E2008BD00BF10B582B015
:100BD000084611464FF00212019335F0B1F8019B1F
:100BE00018680CF057FC0649044608203FF00CFE3C
:100BF000214601900CF07AFB019802B010BD00BFB5
:100C0000B4C70B0010B504460CF0B0FBC8B92046C1
:100C10000CF0B2FBB5EEC00AF1EE10FA0DD9B4EE4D
:100C2000400AF1EE10FA0AD610EE103A23F0030053
:100C300040F00200A0F1FF4010BD0E2010BD0248A0
:100C400010BD5CF063FF00BF0200400010B5044619
:100C50000CF08CFB30B920460CF094FB400040F0C7
:100C6000010010BD5CF052FF08B50CF01FFC0E2017
:100C700008BD00BF10B582B0084611464FF0021201
:100C8000019335F05DF8019B40F2F741186873F06D
:100C9000B7FB0649044604203FF0B6FD214601900B
:100CA0000CF0FCFB019802B010BD00BF40C80B0067
:100CB00030B583B004460D460CF0FAFB80B90190C4
:100CC00028463EF041FA0199A2234FF6FF7235F013
:100CD00075F981B220460CF0EDFB0E2003B030BD5B
:100CE0005CF014FF2DE9F04F2DED088B804B8FB099
:100CF00009ACCDE90034052335F05CF800210998F2
:100D00004FF0B4FF002107460A984FF0AFFF0546A9
:100D100000210B984FF0AAFFEB790290012B40F0D5
:100D2000E380C379012B40F0DF80AA68012A40F2FA
:100D3000DB808368012B40F2D7809A4240F0D48058
:100D40006621B86852F0D6FAEC69297981462046C6
:100D500050F0D2F8AB68A8692979013B00FB034049
:100D6000F0EE408A50F0C8F80C98029B0E28DC691F
:100D7000B0EE40AA00F0A2803EF078F90D980E285F
:100D8000B0EE409A00F0A4803EF070F9F0EE409A88
:100D9000BB68C3B3EB690493029BD7F81CA0DB6963
:100DA000D9F81C6003934FF00008BB46CDF81C90A7
:100DB0000EE0B4EEC0AAF1EE10FA2AD5F0EE697A90
:100DC000E6EC017ADBF8082008F10108424518D961
:100DD00050469BF8041050F08FF8DBF81820F4EE22
:100DE000C08AF1EE10FAB0EE408A9244E1DDF0EEF6
:100DF000497AE6EC017ADBF8082008F1010842455F
:100E0000E6D8DDF81C9048460FB0BDEC088BBDE875
:100E1000F08FAC68013C012C27464FF000091ED929
:100E2000CDE905862E46049D04E0A7EB0804012CBD
:100E3000C14610D9B0693179640804EB090800FB98
:100E4000085050F059F8B4EEC80AF1EE10FAECDB95
:100E5000012C4746EED83546DDF81480069E049CEA
:100E6000A869297900FB094050F046F8A86929795A
:100E700000FB0740F0EE40BA50F03EF8029C039BA6
:100E8000A069217900FB0930F0EE40AA50F034F857
:100E9000A069039A217900FB0720B0EE40BA50F018
:100EA0002BF838EE6B8A30EE4B0A7AEEEBAA28EE7E
:100EB000008AC8EE2A7A77EE8B7A81E72046197984
:100EC00050F01AF80D980E28B0EE409A7FF45CAFFF
:100ED000029A906893691179013803FB004050F041
:100EE0000BF8F0EE409A53E7024870F0B1F800BFFB
:100EF000483A0C00547B0B002DE9F0472DED068B92
:100F00005D4B88B005ACCDE90034032334F052FFCB
:100F1000059800214FF0AAFE8368012B75D9C57989
:100F2000012D044640F0A58000794FF083FF07466D
:100F30000698E6690E286ED000214FF097FEC5791D
:100F4000012D814640F09280A26883689A4240F069
:100F50008D8000794FF06EFF80463046D9F81CA096
:100F6000B847A36903935046B0EE408AC047A368D0
:100F7000012BF0EE408A74D9039B9FED40AA1E44DA
:100F8000D9F818309A443046B847A3695046B0EEB5
:100F9000489A1E44B0EE408AC047F0EE689A38EE98
:100FA000099A70EE699AF0EE4A6A07EE905AD9EE05
:100FB000896AA368D9F81820B8EE677A0135C6EEB9
:100FC000877AAB429244F0EE408A3AEE27AADAD80A
:100FD000F6EE007A2AEE27AA013B07EE903AF8EEE9
:100FE000677A67EE8A7AF4EE677AF1EE10FA3BD60A
:100FF00017EE903A23F0030040F00200A0F1FF400A
:1010000008B0BDEC068BBDE8F0871D4808B0BDEC0C
:10101000068BBDE8F0870798DFED188A3EF026F8CA
:101020003046B0EE40AAB847A368012B16D92A462D
:101030002179E069B0EE408A4FF01AFF07EE905A2E
:1010400030EE088AB8EE677A38EE688AA368C8EE90
:10105000077A0135AB4278EEA78AE8D82AEE28AAAB
:10106000B6E79FED06AAB7E70648C9E706486FF05E
:10107000EFFF06486FF0ECFF303A0C000000000074
:101080000200808002004000F0730B00E4730B004C
:101090001E280ED03E280CD010F001030AD110F00B
:1010A000030209D10168094A914208BF0123184689
:1010B0007047012318467047022AFBD16FF3D60010
:1010C000831F18BF01231846704700BFE4570B0069
:1010D00010B54268FF2A82B004460B460ED9D4E907
:1010E0000221207935F07AFED4E901320E20013256
:1010F000A3F58073C4E9013202B010BD0191002252
:101100000179402035F08CF80246D4E9021008310C
:1011100002FB01F1009232F017F8009AA168D4F8AE
:1011200004C0E06001FB02210844082161F31F2C88
:10113000C2EBC202C4F804C0002133F0C1FF019B1E
:10114000CDE700BF2DE9F04313468BB005460C46B2
:10115000242820D8DFE800F024242424241F1F1F83
:101160001F1F1F1F1F1FA61F131F1F1F1F1F1F1F14
:101170001F1F1F671F131F1F1F1F1F1FB30013F009
:10118000010240F0B18013F0030104D1B24A1868A3
:10119000904200F0A980002420460BB0BDE8F08307
:1011A00009790393002201F07F01402035F038F8DF
:1011B000E368AA4A21681E46A368994623799142AA
:1011C00098460746039B00F0F3801846012207A9C2
:1011D0003AF05AFA002800F0828008F07F03012BD1
:1011E000099A00F0EB805A2B94BF20330020012A8B
:1011F00000F0C1805A2A00F317812032934240F058
:10120000B08023F00203642B00F0AB80089B0093B6
:1012100009FB07F2079B3146284644F007FA0028ED
:101220005DD03E24B8E78D4D0A68AA42B3D0097953
:101230000393002201F07F01402034F0F1FFA26807
:10124000E36802FB00F8227902F07F062268AA42D6
:101250001F46039B00F0BB80184607A905223AF001
:1012600013FA00223146402034F0DAFFA168089BCF
:1012700005463046B3FBF5F31944039300F02AFA10
:10128000044639464246C06833F036FDE068039BA9
:10129000079903FB05F2404433F02EFD20460BB0C6
:1012A000BDE8F0836D4A096891423FF474AF194676
:1012B000204600F047F920460BB0BDE8F083184601
:1012C000012204A903933AF0DFF9039B00283FD0E1
:1012D00014F0030203D1624B216899424FD01E24BF
:1012E00020460BB0BDE8F08318463DF02DFF217974
:1012F000002201F07F018146402034F091FFE36835
:101300002668A16822799846544B9E4201FB00F75B
:1013100000F08480102D60D009FB01F102F07F0005
:1013200000F0D8F9C3680446002F3FF435AFB9F197
:10133000000F3FF431AF09F1FF35414618463A46F8
:1013400033F0DAFC013D691C00EB0703F5D123E71C
:10135000DA0706D413F0030206D13F4A1B68934212
:10136000BDD100206FF0FCFD022AB8D16FF3D60387
:10137000062BF6D1B3E7622B3FF448AFF1E72179B2
:10138000364D01F07F01402034F04AFF0246D4E997
:10139000023003FB02F12368AB4256D00124DDE9A1
:1013A0000423009429F054FB00287FF43AAF96E719
:1013B0006268C2F3172200FB026606E7012A3FF4C7
:1013C00025AF5A2A3DDC422A3FF420AFC9E76268C4
:1013D000C2F3172200FB02773EE7114640200022AD
:1013E00034F01EFFA36809FB03F300FB03F1E06880
:1013F00031F0AAFEA368E06009FB03F3A360636811
:1014000003F0FF036360B9F1000F3FF4C5AE09F1CB
:10141000FF39C319002F3FF4BFAE88E76368C3F3F9
:10142000172300FB038875E793429AD123F0020348
:10143000642B96D0022D3FF4E9AE00287FF4E6AE8F
:101440008FE7622A3FF4E2AE8BE76368C3F31723AA
:1014500002FB0300A2E700BFE4570B00C04C0B00E7
:10146000084D0B00F0B5012885B007460E463FD069
:101470008B0736D030463FF02DF8002857D0451066
:101480002946384600F026F90021044630463AF055
:1014900091F906463AF03EFC68B17DB100252A4636
:1014A0000346E168384635F099FC304601353AF09C
:1014B00031FC0028F3D1204605B0F0BD014620469E
:1014C000FFF706FE30463AF025FC0028F3D001462F
:1014D0002046FFF7FDFD30463AF01CFC0028EDD118
:1014E000E9E70B68144A934202D0144A9342C1D1EF
:1014F000012201A930463AF0C7F80028BAD039468F
:101500000022402034F08CFE029BB3FBF0F100FB84
:1015100001F5AB420DD1384600F0DCF801990446E4
:101520002A46C06833F0E8FB204605B0F0BD05460A
:10153000A6E703486FF08CFD38630B00084D0B00E5
:10154000F8810B0070B50E4686B00446012203A94F
:1015500030463AF099F800283AD02179002240200C
:1015600034F05EFE6268049BB3FBF0F3B3EB122F22
:101570000546C2F31721E06813D8C91A61F31F2288
:101580006260A2680399019302FB050003FB05F268
:1015900033F0B2FBA268019B0E201A44A26006B091
:1015A00070BDA1680193194405FB01F131F0CCFD38
:1015B0006268E06002F0FF026260B442019BE0D129
:1015C000052203A920463AF05FF8E068019BD8E7BE
:1015D000014630463AF0EEF8054601E0FFF778FDA7
:1015E00028463AF097FB014620460029F6D10E2006
:1015F00006B070BD70B50D460179044601F07F015B
:1016000016464020002234F00BFEE2682A60A368F0
:1016100000FB03F36B60237903F07F03AB60216869
:10162000094B994201D0002070BD94F90430002B81
:1016300003DBB30701D5012070BD6368C3F3172333
:1016400000FB03222A60EEE7C04C0B004268C3682F
:1016500091688B4284460BD21079D168DCF808205F
:101660001A44013300F07F00CCF80C3035F02CB870
:1016700000207047084A0023C1E90233C1E9002075
:10168000064B02689A4201D0084670474368C3F38C
:1016900017238B6008467047544C0B00C04C0B005E
:1016A00038B50C461D4611462046094A34F048FB21
:1016B000286841F00DF9012C007804D06968BDE874
:1016C0003840FFF7CFBEBDE83840002100F002B837
:1016D000040002007828F8B51CD005460E4600220A
:1016E0000146402034F09CFD012D0CBF0B490C49F4
:1016F000074610203FF088F805714368866003F0C4
:10170000FF030446436006FB07F031F011FDE06083
:101710002046F8BD03486FF09BFC00BF084D0B004E
:101720008C4C0B0070820B0070B50D79012D0C46AE
:1017300006462FD01F492A4643F0B0F8A3682BB9BC
:1017400030461D49BDE8704043F006B81B4930469D
:1017500043F002F8A3689BB1002501E042F0FCFFD2
:101760002A46E168207934F0AFFF01220146304675
:101770003FF0E8FDA36812490135AB423046EDD891
:101780001049304642F0E8FF30460B49BDE8704052
:1017900042F0E2BF0C4942F0DFFFD4E902213046BB
:1017A0002B4644F0B7FC30460349BDE8704042F098
:1017B000D3BF00BF78100B0098110B0084100B00F2
:1017C00088100B008C100B006C100B002DE9F047FB
:1017D00088B0002A35D011F0030304468C46806897
:1017E00015461E4603D1904B0A689A422ED0624697
:1017F00001460023206839F081FF8C4B216894F862
:1018000004C09942024609D0042D0FD1E1680CF0C2
:101810007F0008B0BDE8F04734F056BF6368042D80
:1018200000EB1322F2D01CF0800F0AD02B46E168A7
:101830000CF07F0035F0D2FA0E25284608B0BDE83E
:10184000F0870025284608B0BDE8F08702AA43F0DB
:10185000C3FF002800F0E2802179042D01F07F0110
:1018600032464FF0400078D034F0DAFC15F0030235
:1018700080464BD12968887B30B101EB8000036939
:101880006B48834200F0AD806A4A91423ED1B8F184
:10189000010F40F0C680052205A9284639F0F4FE64
:1018A000DDE9059761484FF0000ADDE9022126686D
:1018B000E3688D1A8642A7EB05052AD0002D34DD9A
:1018C0006068B5EB102F65D8D019A26801932A443F
:1018D000121A08FB013108FB02F208FB003033F05A
:1018E0003FFADDE9013009EB0A0108FB07F200FBD2
:1018F000083033F035FA6368C5EB132262F31F2317
:10190000A26863602A44A2600E2596E74A486FF0F9
:1019100027FB94F90410002993DA002D40F0818010
:101920006168C1F3172108FB013308FB023009EBA2
:101930000A0108FB07F2019333F012FA0399A26837
:101940000298019B521A384408FB02F208FB01314D
:1019500008FB003033F004FACDE734F061FC334B80
:101960002168029A9942064629D1B2F1807F51DA64
:1019700010203EF049FF054694E80F0085E80F006F
:10198000029A02EB112363F31F216960039B9B1AE8
:10199000AB6052E7A26801932A4408FB02F11846A3
:1019A00031F0D2FB6268E06065F31F226260019B48
:1019B0009945DDE90221034608BF814684E7039982
:1019C0002079891AFFF786FEDDE902130546E068F3
:1019D0005B1A06FB03F206FB0101E86833F08CF9A1
:1019E0002BE72979402001F07F0134F019FC4045B4
:1019F00017D1AB680D482A681F46EB6882429946AA
:101A000002D04FF0000A50E76A68C2F3172208FBC1
:101A100002FA4AE709490A487AF02FFE09486FF0AE
:101A20009FFA09486FF014FB6C600B00C04C0B0070
:101A3000CD17030038630B0004830B0084790B007F
:101A400004540B0070770B004C7A0B00042808D06C
:101A5000052801D0002070478868400040F0010050
:101A600070478B68002B0CBF1E203E20704700BFC4
:101A700010EE102A22F00043B3F17E5FF0EE407AC0
:101A800007D30FD070EE407A9FED3B7A87EE270A9E
:101A90007047B3F17C5F27D2A3F50003B3F1645F15
:101AA00007D270479FED357A9FED350AA7EE870A7A
:101AB000704760EE006A9FED336ADFED335A9FEDA9
:101AC000337A9FED335AE6EE865AB7EE006AA6EEF9
:101AD000A57AA6EE856A27EE267AC7EE066AE0EEBC
:101AE000267AB0EE670A7047B7EE007AF0EEC07A59
:101AF00077EE677A00B5B6EE007A67EE877A83B044
:101B0000F5EE407AF1EE10FA28D4F1EEE76A002AF9
:101B1000DFED1C5A9FED1C6A9FED1C7A9FED1C5A4D
:101B20009FED160AA7EEA56AF7EE005AA7EE867A91
:101B3000E7EE855A67EE277AB0EE005A87EEA57A6F
:101B4000DFED147AE7EE266AE6EE857A30EE670A74
:101B500001DB03B000BDB1EE400AFAE78DED010AEA
:101B6000B0EE670ACDED007A63F0A8FB019ADDEDD7
:101B7000007AF0EE406ACAE700000000DA0FC93FC1
:101B8000000080036BD30DBCBA132FBD75AA2A3E8B
:101B9000AEE534BF6821A2B300B585B08DED010A72
:101BA000019B23F00042B2F18B4F00EE102A4FEA66
:101BB000D37127D25B000ED4B2F1665F2BD2DFED7A
:101BC0001F7A70EE277ACDED037A039B09B1B1EE4F
:101BD000400A05B000BDB7EE007AF0EE476AE0EECD
:101BE000006A0191B0EE006AF1EEE67A77EE807A53
:101BF000C7EE276AE0EE066AB0EE660A31F06AF9CF
:101C00000199E3E7019131F065F9DFED0D7A019972
:101C100030EE270ADAE720EE007AF7EE006A37EEB8
:101C2000266A0191F1EEC67A77EEA67AC7EE276AA8
:101C300036EE800A31F098F80199C7E70000807B02
:101C40001872313F08B559F015FE044B02689A42EC
:101C500000D108BD0D205DF085FA00BFEF297801A5
:101C600000B585B040F2FF1C01A903AB02AACDF874
:101C70000CC02BF0F5FA024803996FF0F1F900BFA0
:101C8000D8940B00F4EE400AF1EE10FAF0EE407A30
:101C900053D610EE901AB1F17E5F49D010EE102AA3
:101CA0008B0F03F0020343EAD27332F0004208D1F3
:101CB000022B3FD09FED397A032B08BFB0EE470AC5
:101CC000704731F000412ED0B1F1FF4F21D001F12A
:101CD0005060904227D3B2F1FF4F24D000B598074F
:101CE00083B030D502F150628A4251D387EEA00A08
:101CF0000193B0EEC00A00F063F8019B022B3ED1C5
:101D00009FED277ADFED277A30EE070A37EEC00A1B
:101D100025E0B2F1FF4F03F1FF3328D0022B20D989
:101D20009FED210A7047DB070AD49FED200A704718
:101D300000F046B89FED1B0A704730EE800A7047EE
:101D40009FED1B0A704787EEA00A0193B0EEC00A10
:101D500000F036F8019B012B01D1B1EE400A03B02F
:101D600000BD144A02EB830393ED000A7047022B77
:101D700011D8114A02EB830393ED000A70479FEDDF
:101D8000087ADFED087A30EE070A30EE670AE6E7F8
:101D90009FED050AB2E79FED090A7047DB0F49C0C6
:101DA0002EBDBB33DB0F494000000000DB0FC93FF5
:101DB000DB0FC9BF70300C007C300C00DB0F493FDB
:101DC00010EE102A22F00043B3F1994F4FEAD2717E
:101DD00009D3B4EE400AF1EE10FA0ED6002943D032
:101DE0009FED4A0A70474A48834207D8B3F1665FBD
:101DF0003DD212F0FF4F00F081807047454A934278
:101E0000B0EEC00A4ED9444A93426ED8F7EE087A33
:101E1000F7EE006AE0EE276A70EE677A9FED3F7A90
:101E20009FED3F0A87EEA66A26EE065ADFED3D7A61
:101E3000DFED3D4A9FED3D4ADFED3D5A65EE056A17
:101E4000E6EEA74ADFED3B7AE6EE847AE6EEA45AA8
:101E500067EEA67AE5EE257A97EE867A77EE467AF1
:101E600030EE670A89BB70479FED330A704720EE5A
:101E7000006ADFED2C7ADFED2C5A9FED2C5ADFED56
:101E80002C6A26EE067AE7EE275ADFED2A7AE7EE8D
:101E9000057AE7EE256A67EE877AE6EE267AA7EE00
:101EA000C00A7047A2F5D002934211D8F0EE007A32
:101EB000FFEE006AE0EE276A70EE277A9FED1F7A48
:101EC0009FED1F0A86EEA76AAEE7B1EE400A7047A3
:101ED000F7EE007A70EE676A30EE270A9FED197A06
:101EE00086EE806A9FED180A9EE7FFEE007A87EE85
:101EF000806A9FED167A9FED100A95E760EE007AF2
:101F000082B0CDED017A019B02B07047DA0FC9BFF4
:101F1000FFFFDF3EFFFF973FFFFF1B40B40F14336F
:101F20005E987B3F25AC7C3D0DF5113E4712DABD36
:101F3000A9AAAA3E98CA4CBEDA0FC93F6937AC318C
:101F40003863ED3E68212233DA0F493F6821A2331E
:101F500000B585B08DED010A019B23F00042B2F17E
:101F60007C5F00EE102A4FEAD37124D2B2F13E5FBB
:101F70000CD213F0FF4F04D160EE007ACDED037A5E
:101F8000039B09B1B1EE400A05B000BD30EE007A06
:101F9000F7EE007A77EEC07A67EE006A019186EE7E
:101FA000A70A30EE070A30F0DFFEF6EE007A20EEE8
:101FB000270A0199E5E7F7EE007A77EEC07A0191FA
:101FC00080EE277A37EE070A30F0CEFEF6EE007A82
:101FD00020EE270A0199D4E7014B18682AF034BB98
:101FE000A846012010B5D1F800C001280C461346C0
:101FF00000F1FF3188BF221D604698BF002260F0CB
:10200000D9F8206810BD00BF10B5044C206831F02D
:1020100053F8034A00231360236010BDA846012033
:10202000B046012000B583B0019001A860F02EF900
:102030000E2003B000BD00BF08B50BF0B9FA0E20AA
:1020400008BD00BF70B508468EB011461A461F4B3A
:1020500008ACCDE90034062333F054FF9DF834403A
:10206000089840F2DB213CB372F002FA4FF4D161E0
:102070000646099872F0FCF902460A9807924FF456
:10208000547172F0BDF940F2754106900B9872F0F0
:10209000CFF90F49054628203EF0BEFB02949DF87B
:1020A00030400095DDE906323146019405900BF091
:1020B00003FA05980EB070BD72F0A2F94FF4D16129
:1020C0000646099872F09CF90246D6E720C90B0033
:1020D00060C90B0010B504460BF0B8FA38B92046B9
:1020E0000BF0BCFA00280CBF1E203E2010BD5BF098
:1020F0000DFD00BF10B504460BF0A8FA38B9204614
:102100000BF0B2FA00280CBF1E203E2010BD5BF081
:10211000FDFC00BF10B504460BF098FA40B920460C
:102120000BF0A2FA30B120460BF0B2FA0E2010BD2F
:102130005BF0ECFC01486EF057FF00BF588A0B00C3
:1021400030B50C6887B005462046CDE902210BF07A
:102150007DFADDE9022188B904AB0193084B0093B5
:10216000681E0223043133F025FE20469DF814201A
:1021700004990BF095FA0E2007B030BD5BF0C6FC59
:1021800050C90B0010B504460BF060FA50B9204658
:102190000BF064FA08B90E2010BD20460BF086FB48
:1021A0000E2010BD5BF0B2FC10B504460BF04EFAE9
:1021B00020B920460BF082FB0E2010BD5BF0A6FC80
:1021C00008B50BF0D3FB0E2008BD00BF2DE9F0478A
:1021D0002DED028B08468CB011461A462B4B05ACF0
:1021E000CDE90034072333F08DFE4FF44771059895
:1021F00072F006F940F253318046069872F000F909
:102200009DF8204062073BD19DF828506B0732D1E2
:1022100081460B98DDF81CA09DF8246040B33CF08B
:1022200025FFB0EE408A40F2EA52B0EE480A0121A2
:10223000002033F07DFE164908203EF0EDFA5346AB
:102240004A464146CDE90165009407460BF046FB3E
:10225000DFED107A28EE278AFCEEC87A17EE900A96
:1022600039F0FAFA38460CB0BDEC028BBDE8F087C5
:102270009FED098AD7E709484FF49C616EF0F0FEA4
:1022800006484FF437716EF0EBFE00BF38CA0B0002
:1022900070CA0B0000007A44AE47E13D28940B0061
:1022A00010B504460BF076FB30B920460BF07CFBF2
:1022B000400040F0010010BD5BF028FCF0B585B097
:1022C00006460C4617460BF065FB00283CD1054638
:1022D00040F25E41384633F057FF294640F25E42F5
:1022E000074633F093FEA30703D11D4B22689A42A1
:1022F00032D0062201A9204639F0C6F99DF80C100B
:10230000029C0022402033F08BFFB4FBF0F4BC426F
:102310001CD330460BF046FB039B482B0FD01028F4
:1023200017D0422B01D0012B09D101993A463046F2
:102330000BF03EFB400040F0010005B0F0BD082866
:10234000F3D108486EF084FE5BF0E0FB06486EF0C7
:102350007FFE06486EF07CFE05486EF001FE00BF71
:10236000609B0B00287F0B00F08E0B000C7F0B0096
:1023700038900B0090F82C20012A5CD190F82D3079
:10238000002B58D090F82E30002B54D090F82B30E2
:10239000002B50D0036A002B4DD030B5044683B0DB
:1023A00000926DF029FB94F82B30009A591E8A4058
:1023B000D2B2216A002818BF134603FB01F1CDE910
:1023C00000136DF019FB236A0099002814BF4FF425
:1023D000FA524FF47A721D46B1FBF2F200926DF0A0
:1023E0000BFB94F82D10009A019B002894F82E0006
:1023F00002F1010201FB00F012FB00F2218A92B20D
:1024000014BF4FF4FA5E4FF47A7E914214D303FB6B
:1024100005F1A2EB000CB1FBFEF30EFB13111FFA4A
:102420008CFC89B100216CF30F016CF31F416162D8
:10243000228503B030BD70474FF0E023D3F8F03D64
:10244000DB07F6D500BEF4E7ACEB0000A084A4F8EF
:1024500026C02285EDE700BF2DE9F04F01298BB0A2
:102460000546164605D0022918D001200BB0BDE85C
:10247000F08F127812F060010F4637D173780A2B73
:1024800053D00B2B7FD0012BEFD04FF0E023D3F8AC
:10249000F03DDB0700D500BE0020E7E7137803F02E
:1024A000E002202AE1D103F01F03012B00F0F280AB
:1024B000022BEAD1B3880DF12701D8B2DFB200F0C8
:1024C00067FB0028E8D09DF827303BB9984B1C46A5
:1024D0005B681BB1DB79002B00F09F8171F0AEF8D7
:1024E0003146024628466CF0A1FCBFE72029CCD13A
:1024F000B38802F01F010129D8B200F0F28002294E
:10250000C3D10DF1270100F043FB0028C4D096F998
:102510000030002BC0F2AD8171F090F840230246EC
:10252000314628466CF0AEFDA0E7814AB188536879
:102530001446C9B2002BAFD09089002896D0184419
:1025400004E01A781344C21A002AA5DD5A78042A36
:10255000F7D19A788A42F4D100238DF82730A37CF2
:102560008B4202D1E37C8DF82730A37E8B4204BFDF
:10257000E37E8DF827300DF12702012331462846EE
:102580006CF080FD72E76A49B3884A680C46DBB29A
:10259000002A81D0888900283FF47EAF104405E0EE
:1025A00011780A44811A00297FF776AF51780429FF
:1025B000F6D191789942F3D1A27C71889A428846EB
:1025C00000F0E480A27E9A4200F0F780A289616860
:1025D00001EB020CA268ACEB0201002952DD5FFAAC
:1025E00088FE05E011780A44ACEB0201002949DDC0
:1025F00051780429F6D191789942F3D1D178714577
:10260000F0D111798946B1B34FF0000163F30701AE
:102610006EF30F21CDE9043E03919046E2469346C6
:1026200004E098F80030B945984421D9AAEB080392
:10263000002B1DDD98F80130052BF2D141462846CC
:1026400070F072FF00283FF420AF636898F8021022
:102650001BB1DB79002B00F0FB8098F80330D80623
:1026600040F1C080284670F02BFF7B1CDFB2D8E71A
:10267000B9457FF411AF314628466CF05DFB002868
:102680003FF40AAF2A48FFF775FE314628466CF042
:10269000E3FCEAE6B388D8B21B0A4BD1244B1C46B4
:1026A0005B68002B3FF4F8AEA18900293FF4F4AE3B
:1026B000194405E01A781344CA1A002A7FF7ECAED1
:1026C0005A78042AF6D19A788242F3D100238DF801
:1026D000273070F0B3FF3146024628466CF0A8FB65
:1026E000C4E6190A41D1124B1C465B68002B3FF42B
:1026F000D3AEA18900293FF4CFAE03EB010C06E075
:1027000019780B44ACEB030100297FF7C5AE59786B
:102710000429F5D199788142F2D1002312068DF86F
:1027200027307FF5F9AE314628466CF097FA9DE6E2
:1027300010120120D9B20DF1270200F0FFF9002894
:102740003FF4AAAE9DF827303BB9864B1C465B6828
:102750001BB1DB79202B00F0918070F06FFF3146C8
:10276000024628466CF038FB80E60DF1270200F0A7
:10277000E5F900283FF490AE96F90030002BBFF643
:10278000CBAE314628466CF0E9F96FE6A17B0393A6
:1027900000222846628270F0AFFE73486BF0FCFFA7
:1027A000314628466CF0F6FA00283FF475AE002258
:1027B000039BA2736262228504E7A17D039300223A
:1027C0002846628370F098FE68486BF0E5FF31465A
:1027D00028466CF0DFFA00283FF45EAE0022039B2F
:1027E000A275F3E62846069170F06AFE0699CB09B9
:1027F00061D1049BA376059BA175E376B8F80430FC
:1028000000200090C3F30A03A26C2383284670F0D3
:10281000DBFE00287FF429AF3EE6A37BBB427FF4BA
:102820005DAE73881B0A012B7FF458AE7378012BC1
:102830007FF454AE70F002FF9DF8273002685021FB
:1028400001FB034022F07F420262FFF793FD45E661
:1028500098F80330284603F00C03CDE9061370F016
:102860002FFE0699079BCA0922D1002B3FF4FDAE2B
:10287000BFE7314628466CF0EFF9F7E594F82A30C7
:102880008B427FF46AAF73881B0A012B7FF465AF1C
:102890007378012B7FF461AF70F0D0FE9DF8273084
:1028A0000268502101FB03400262FFF763FD54E719
:1028B000002B3FF4DAAEBDF80C30A1736382B8F898
:1028C0000430C3F30A032382B4F840305B08A382C8
:1028D0009BF80030069300200BEB03026CF006FA25
:1028E0000128069B25D05078242809D00023009386
:1028F000E26C284670F068FE00287FF4B6AECBE5A7
:1029000090780128F2D1907A84F82D00507984F8DB
:102910002C001BF803301A445378242BE6D193780B
:10292000022BE3D1D378012B04BF137984F82E3026
:10293000DCE71BF8033013445A78242AD6D19A785E
:10294000022AD3D1DA7884F82C20012ACED11A7940
:1029500084F82D205A7984F82E209B6823F07F4339
:102960002362C3E7101201204C1201204012012003
:102970000020704710B50D4C0C485022002132F059
:102980009FFB0B4901234FF4446204F13C006BF0C0
:1029900007FF0848E064012307494FF4446204F14B
:1029A00030006BF0FDFE054BA36410BD101201203A
:1029B000804D01202C6B0120C0590120F06B0120BB
:1029C0004B79012B02D18B79012B01D0002070476C
:1029D000CB7913F0DF0FF9D10B7801EB020C0B442C
:1029E0006345F3D210B593F800E09E44F44507D355
:1029F0005C78042C04D0E6457346F4D3002010BD67
:102A0000ACEB030EBEF1080FF8DD93F805E0BEF164
:102A1000010FF3D19B79022BF0D10B79012B2BD82D
:102A20002AD0CB78002BE9D1384B5B6823BB374BDE
:102A3000596018700B78D21A002A60DD0B44092007
:102A40000AE00B2A20D01A781344ACEB030E0244A0
:102A5000BEF1000F90B217DD5A78042AF1D15A79ED
:102A6000012A11D19A79022A0ED1284A9268002AA5
:102A7000E9D1264A9360E6E74FF0E023D3F8F03D32
:102A8000D907BBD500BEB9E7204B988198B301EBBD
:102A9000000C0B460AE091F807E0BEF1200F1AD0B7
:102AA0001A781344ACEB0302002A24DD5A78052A75
:102AB000F1D1DA7802F0030EBEF1010FF0D193F8F4
:102AC00002E05FEADE1EEBD0D206E9D40F4C9A7921
:102AD00084F82B20E4E7242AE2D19A78032ADFD174
:102AE000B3F804E040F201129645D9D1074C1A7AA6
:102AF00084F82A20D4E7054A0123137710BD034B3D
:102B00000920988101EB000CC3E700BF10120120DF
:102B100010B530220021054832F0D2FA04486BF09B
:102B20003BFEBDE8104003486BF036BE101201209A
:102B30004C12012040120120704700BF10B5134C09
:102B40006368FBB193F802C08646F4454FF000007D
:102B500000D010BD1878D4F808C01C5C034423448E
:102B6000ACEB0300002806DC0EE018780344ACEB65
:102B70000300002808DDD8788842F6D100231370BE
:102B8000012010BD184610BD002010BD10120120FC
:102B90000E4B5A68C2B1B3F80CC09B689444ACEBBE
:102BA0000302002A06DC0FE01A781344ACEB0302A0
:102BB000002A09DD5A78052AF6D19A788242F3D1A3
:102BC00000230B7001207047002070471012012075
:102BD000002070472DE9F04F514CA27B8A4283B010
:102BE00080461F4625D0A37D8B420BD1A16C0023CC
:102BF000BAB204F130006BF09DFE38B9012003B089
:102C0000BDE8F08F002003B0BDE8F08F0122238BD8
:102C10000092A26CA17D404670F0D6FC0028EDD059
:102C2000E27EA37D0092B9B2002240466CF082F8A9
:102C3000E4E7E37C002BE1D0B4F84430B4F846205C
:102C4000B4F84010208A92B29BB29342B6BFC2EB56
:102C500041029A1AD21892B2E38C8A4228BF0A46DD
:102C6000002B38D0B3EB810F35DCA18C8A4236D3F0
:102C7000258DA68ADFF8B0E0A5EB030C1FFA8CFCCB
:102C8000AA46B346DEF80050A6EB0C06B242A946AF
:102C900027DA002D33D1884228BF08460A2302468E
:102CA000CEF80030E16C1F48002315466BF01EFE85
:102CB00001230093E26CA17B2B46404670F084FC1C
:102CC00000289BD0E27CA37B0092B9B20022404650
:102CD0006CF0B0F892E7824228BF0246E2E7002299
:102CE000E0E7DC44624513DD4DB98245524628BF1A
:102CF00002468B42D6D00A23CEF80030D2E7984263
:102D000028BF184609F1FF330246CEF80030C9E764
:102D1000002DF4D1984228BF18460246C2E700BFF2
:102D2000101201204C120120FC47012008B50AF0C6
:102D300095FE0E2008BD00BF70B590F80FE0D0F8EA
:102D400008C0BEF1000F13D0049CC4F800C0D0F836
:102D500010C081B390F80DE0007BB2FBFEF10EFBDA
:102D60001121C008C9B201FB00C11960002070BD6B
:102D7000049C4FEA5C0CC4F800C0856890F814E02D
:102D800004694FEA550C0EFB0CFC41B904EB0C0234
:102D90001A60037DC3F101030375002070BD457BFC
:102DA000017BB2FBF5F605FB1622C908D2B212FB75
:102DB00001C2A218ECE7C3F800C0002070BD00BF3C
:102DC00010B508468EB011461A462B4B0AACCDE919
:102DD0000034042333F096F80A98052207A938F046
:102DE00053FC099B622B2FD0682B2AD0422B2ED06C
:102DF00030DC012B08BF002430D19DF834204AB9C3
:102E00000B9A089903FB02F25200B1FBF2F002FBAD
:102E1000101159BB1949059318203DF0F5FC9DF898
:102E2000342003920C9A02929DF82C200192059B6B
:102E3000089A0799009404900AF0FCFD04980EB0DB
:102E400010BD01240223D8E701242346D5E700243E
:102E50000123D2E723F02003482B04D0084840F296
:102E6000FB216EF0FDF800240223C6E7054840F27E
:102E7000FB216EF0F5F800BF24CB0B0044CB0B0018
:102E800044940B00EC8B0B00704700BF08B50AF0B0
:102E9000CBFE0E2008BD00BFF0B50446856B85B0A3
:102EA0001F46E9B1012A164670D0A26A636BE2B9E7
:102EB000AB426DD0E18C01350D44ED1AEB0753D5D3
:102EC00023693B600A9A63691360002E53D1A36B98
:102ED0000133A363A06A003818BF012005B0F0BD1C
:102EE000A26A636B0E46002AE2D0AB42E18CE2D1CB
:102EF000E36A9A4228BF1A46C9074CBFA1692169F3
:102F00003960206B0192083003AB78F0BFFA0028DB
:102F100044D1039B019A934240D1A16A891AA162CC
:102F200081B912F003000DD01318227B0393082AF5
:102F300037D0102A06D13A6823F001031A4422F848
:102F4000021C039B0A9A1360E18CCA074CBFE36121
:102F500063610131636B89B2013501330D44ED1AB0
:102F60006363EB07E184ABD4A3693B600A9AE3692E
:102F70001360002EABD0012EACD1E36B227B01336A
:102F8000E3633B6803EBD2033B60A3E7C56B8CE7CD
:102F90000A9B3A6010461A6005B0F0BD022005B0E9
:102FA000F0BD4FF0800C3A685B1A1A44013102F808
:102FB00001CC8842039BF6D1C4E700BF70B51E4622
:102FC0000D4686B0114628461F4A32F0B9FE3468D5
:102FD0001E4B2340062B05D0A20722D123681C4A92
:102FE000934209D121461B4845F2E62234F08AFE7D
:102FF0008307044615D10368174A934211D1012D66
:1030000012D800231E461549019340203DF0FCFBD9
:10301000019B3246214605460AF024FD284606B0AB
:1030200070BD0F486EF000F87068062203A938F0F2
:103030002BFB40F2FB230498039E4FF4806208218F
:1030400032F0F0FF0346DEE7040002000F0080FFCD
:1030500088630B00AC990B00609B0B00B8CB0B0096
:103060000C7E0B0009B1012A12D010B50146006B8D
:103070000C6A8A8C82B000238C620830019177F050
:1030800091FE01990023C1E90D33CB6302B010BD5D
:10309000704700BF08B50AF0FDFD0E2008BD00BF57
:1030A0002DE9F04F2DED068B824693B01E462298F7
:1030B000DAF82430E1B1012A154600F05184DAF83B
:1030C00018200260DAF820109AF81C20994229D0C2
:1030D00082B9DAF8103033608DB9DAF82430013370
:1030E000CAF82430012013B0BDEC068BBDE8F08F88
:1030F0000D46E4E7DAF814303360002DEDD0012DF1
:10310000F0D1DAF828309AF80C200133CAF82830C8
:103110003368012003EBD203336013B0BDEC068BA0
:10312000BDE8F08FDAE90437002A18BF1F46376080
:103130009AF81C3083F001038AF81C30DAF8183052
:103140004FEA930B9AF82C30002B00F00D840024EA
:103150009FED96AADFED969A9FED969ADFED968AFF
:103160000D971095119605945F460AF13005564665
:1031700055F804BFDBF808200392002A00F0DC8039
:10318000002F00F0D7800D9B04930BF11003CDE9C5
:103190000737CDE90945DBF81420029742BB9BF8BD
:1031A0000D304BB99BF80C30002B00F0D383DBF8CB
:1031B0000800114601F0E8FADBF80800002800F0EA
:1031C00053810BF11403002200931146079B01F079
:1031D0003FFA022800F0A983DBF81420A0F10100D7
:1031E000B0FA80F0400992088BF80D00CBF814205B
:1031F000039B717B587BDBF810A088424FEA0123C8
:1032000040F037810298834228BF0346934228BF8B
:10321000134698467068B8FBF1F189B25EF06EFF14
:10322000F7EE000A0BF11800B0EE4A0A66F074FEE1
:10323000F0EE690AB0EE408A0BF11C00B0EE490ACC
:1032400066F08CFE28EE288A727BBCEEC88A022AC1
:1032500018EE103A9FB240F00A81030400F1FD809D
:10326000C0F5FF407F3080B24FF4004307FB00F011
:1032700007FB03F3C013DF13039B597B059BDBE9BB
:103280000845002B40F09A80337B102B40F07E8164
:10329000B37B002B00F0D7818A4240F0D382B8F193
:1032A000000F00F00481049BAAF10402DDF814A0D1
:1032B000CDF818A0A3F1040E4FEA880C02EB8809A0
:1032C000A04252F8041F63D1AF4261D1230433FB03
:1032D00001F34FEA054A3AFB11F123F3CF3321F30F
:1032E000CF31C3EA01434A454EF8043FE8D1039B7E
:1032F000727B5B7B9A4240F0C880029BDBF8142013
:10330000A3EB08030293049B63440493DBF810309F
:10331000A2EB08026344CBF81030029BCBF81420D8
:10332000CBE90807002B7FF439AFDDE908740A9D6B
:1033300096F82C30012205920134A3423FF718AFD2
:10334000059B109DBB46B2460D9F119E002B00F0C1
:103350000B839AF80E30ABB99AF80C30102B00F0B2
:103360004F85BBF1000F0DD00BF1FF3307EB83034B
:103370004FF08031043F57F8042F82FA41F29F4208
:103380003A60F8D1DAF820300133CAF82030A3E6E9
:10339000B1F5803F5ED38BB2002B5BD0069B1BB197
:1033A0004B4013F0802F55D106918FE700000000AD
:1033B00000FE7F3F00FE7FBF00000047337B102BE5
:1033C00077D196F80EC0BCF1000F00F07E818A42E2
:1033D00040F0C481B8F1000F69D0AAF10402049B47
:1033E0004FF0000AA04202EB8809A3F1040E52F844
:1033F000041FCDF818A04FEA880C1BD1AF4219D199
:10340000230433FB01F34FEA054A3AFB11F123F39E
:10341000CF3321F3CF31C3EA01435EF8041F93FA9F
:1034200011F34A45CEF800303FF461AFA04252F8A4
:10343000041FE3D0B1F5803F09D38BB23BB1069BAB
:103440001BB14B4013F0802F01D10691D8E73D46C8
:103450000446D5E73D46044638E700F5FF407F3097
:1034600083B24FF4004001E7DBF81420C0E6384691
:1034700002E74FEA4208029A934228BF1346984552
:1034800028BF9846C6E64FEA880C049BDBF8141068
:1034900063440493029BA3EB08030293DBF8103010
:1034A0004FEA580803EB8803A1EB080233E7C44650
:1034B00023E78A424FEA480340F00683002B00F0DE
:1034C0003182049A0693AAF1020C0021A2F1020AA9
:1034D0000B918E46624632F802CF96F80E904FEA74
:1034E0000C414FEA0C2C01F07F411FFA8CFC41EAA1
:1034F0000C01B9F1000F03D14FF0802391FA43F191
:10350000A0422FD1AF422DD14FEA044C3CFB01FC2D
:103510004FEA054939FB11F92CF3CF3129F3CF39A3
:10352000C1EA09413AF8029F4FEA094C4FEA0929DA
:103530001FFA89F90CF07F4C4CEA090C91FA1CF146
:103540004FEA114C069B0EF1010E0CF47F4CC1F3B7
:1035500007214CEA01017345AAF80010BBD14FEADC
:10356000880CC4E6B1F5803F0BD31FFA81FCBCF197
:10357000000F06D00B9B3BB181EA030C1CF0802F9F
:1035800002D03D460446BFE70B91BDE78A4240F0BA
:103590000E825FEA480300F0C58104990693A1F109
:1035A000020905990B91AAF102028A4632F802CF6C
:1035B00096F80EE04FEA0C414FEA0C2C01F07F41E7
:1035C0001FFA8CFC41EA0C01BEF1000F03D14FF051
:1035D000802391FA43F1A04221D1AF421FD14FEA9B
:1035E000044C3CFB01FC4FEA054E3EFB11FE2CF364
:1035F000CF312EF3CF3CC1EA0C414FEA114C069B70
:103600000AF1010A0CF47F4CC1F307214CEA0101D5
:103610009A4529F8021FC9D14FEA880C67E6B1F52F
:10362000803F0BD31FFA81FCBCF1000F06D00B9B2F
:103630003BB181EA030C1CF0802F02D03D460446CA
:10364000CDE70B91CBE78A4240F0DB82B8F1000F67
:103650003FF42DAF049ACDF818B0AAF10403A2F1FB
:10366000040E059A0B924FEA880C03EB880A4FF080
:10367000802953F8042F92FA49F2A04215D1AF42A3
:1036800013D1210431FB02F14FEA054B3BFB12F24F
:1036900021F3CF3122F3CF32C1EA024153454EF834
:1036A000041FE6D1DDF818B021E6B2F5803F07D35C
:1036B00091B229B10B9931B1514011F0802F02D054
:1036C0003D460446DDE70B92DBE78A4240F0148377
:1036D000B8F1000F3FF4EBAEAAF10403049ACDF861
:1036E0002CC003EB880AA2F1040E53F8041FCDF896
:1036F00018B04FEA880C4FF0802991FA49F1A042A6
:103700001CD1AF421AD1220432FB01F24FEA054B21
:103710003BFB11F122F3CF3221F3CF31C2EA014258
:103720005EF8041F92FA11F25345CEF80020B9D08A
:1037300053F8041F91FA49F1A042E2D0B1F5803F5D
:1037400007D38AB22AB10B9A32B14A4012F0802FC5
:1037500002D03D460446D6E70B91D4E7B8F1010FFD
:103760007FF691AE04994FEA5803AAF1040C01EBDD
:10377000C30E8A4600210C91CDE90EB601040691D4
:1037800039040B915CF8042FA04293B243EA024340
:1037900048D1AF4246D121044FEA054931FB03FB32
:1037A00039FB13F32BF3CF3B23F3CF33CBEA0343A4
:1037B000DAF8006093FA16F3CAF80030130C1B0411
:1037C000A04243EA12431AD1AF4218D131FB03F1B0
:1037D00039FB13F321F3CF3123F3CF33C1EA034293
:1037E000DAF8043092FA13F2CAF804200AF1080A4F
:1037F000F245C7D1DDE90EB64FEA880C77E5B3F59F
:10380000803F07D39AB22AB10C9A4AB15A4012F0BB
:10381000802F05D00699DDF82C903D460446D5E76B
:103820000C93D3E7B3F5803F07D399B229B10C9934
:1038300031B1594011F0802F02D03D460446AAE72D
:103840000C93A8E7C446B8F1000F3FF41EAE0499EC
:10385000CDF838B008F1FF3308315B0801EBC30342
:10386000AAF10409DDE904A10C91010406913904CF
:103870000B919B4659F8042FA04293B243EA0243AE
:1038800040D1AF423ED121044FEA054E31FB03FC4B
:103890003EFB13F32CF3CF3C23F3CF33CCEA0343AB
:1038A000CAF80030130C1B04A04243EA124316D19D
:1038B000AF4214D131FB03F13EFB13F321F3CF31BF
:1038C00023F3CF33C1EA0341CAF804100AF1080A0E
:1038D000DA45CFD1DDF838B04FEA880C07E5B3F50B
:1038E000803F07D39AB22AB10C9A4AB15A4012F0DB
:1038F000802F05D00699DDF82CE03D460446D9E737
:103900000C93D7E7B3F5803F07D399B229B10C994F
:1039100031B1594011F0802F02D03D460446B2E744
:103920000C93B0E74FEA880CE7E4DDE90874002364
:103930000A9DCBF80830CBF814308BF80D30059B7E
:103940002BB9029BDDE904019A0031F0B9FB96F82E
:103950002C30EFE4DDE908740A9DCBF80820EEE78F
:10396000DAF82830FFF7ABBBBBF1000F3FF40AAD2C
:103970004FEA8B020021384631F0A2FB9AF80E3054
:10398000002B7FF4FFAC9AF80C30102B7FF4ECACDA
:103990000BF1FF3107EB81013B1F4FF0802053F803
:1039A000042F92FA40F28B421A60F8D1EAE44FEA0F
:1039B0004803012B7FF667AD049ACDF838800104E7
:1039C00008F1FF3306913904AAF102090AEB430E0C
:1039D000CDE90B1B02F1020A059A904639F8023F25
:1039E000B27B19041B0201F07F419BB219431AB943
:1039F0004FF0802391FA43F18BB2A04243EA014396
:103A000050D1AF424ED122044FEA054C32FB03FBAA
:103A10003CFB13F32BF3CF3B23F3CF33CBEA03432E
:103A20004FEA134B0BF47F4BC3F307234BEA030B13
:103A30000B0C1B04A0422AF802BC43EA11431CD120
:103A4000AF421AD132FB03F23CFB13FC22F3CF331B
:103A50002CF3CF32C3EA02431A0C02F47F42C3F3C1
:103A600007231343F1452AF8043BB7D1DDF838802A
:103A7000DDF830B04FEA880C39E4B3F5803F0BD362
:103A800099B249B1B8F1000F00F0B68183EA08019C
:103A900011F0802F00F0B081069ADDF82CC03D4671
:103AA0000446CFE7B3F5803F0BD39AB24AB1B8F1E1
:103AB000000F00F09F8183EA080212F0802F00F0CF
:103AC00099813D4604469EE7012B7FF6DCAC049AC3
:103AD00008F1FF330AEB4303AAF1020E02F1020AD6
:103AE0000022069202040B923A04CDE90EB80C9221
:103AF0009B463EF8023FB27B19041B0201F07F4156
:103B00009BB219431AB94FF0802391FA43F18AB25C
:103B1000A04242EA014264D1AF4262D123044FEA9B
:103B2000054C33FB02F83CFB12F228F3CF3822F3AA
:103B3000CF32C8EA02493AF8028C4FEA08424FEA0B
:103B400008281FFA88F802F07F4242EA080299FA30
:103B500012F24FEA124808F47F48C2F3072248EAFB
:103B600002080A0C1204A0422AF8028C42EA11420E
:103B700025D1AF4223D133FB02F33CFB12F223F3F6
:103B8000CF3322F3CF32C3EA0243BAF800100A045B
:103B9000090289B202F07F420A4393FA12F31A0C27
:103BA00002F47F42C3F307231343F3452AF8043B8F
:103BB0009FD1DDE90EB84FEA880CFFF798BBB2F54C
:103BC000803F09D391B239B1069919B1514011F032
:103BD000802F01D10692CEE7DDE90B3C3D4604463D
:103BE000C9E7B2F5803F09D393B23BB1069B1BB145
:103BF000534013F0802F01D106928FE73D460446D3
:103C00008CE7B8F1010F7FF63EAC049ACDF838800E
:103C10004FEA580302EBC30301049146059A06914B
:103C20003904CDE90B1BAAF1040AB346984616469F
:103C30005AF8043F4FF0802293FA42FC1FFA8CF3AB
:103C4000A04243EA0C4347D1AF4245D122042904A4
:103C500032FB03FE31FB13F32EF3CF3E23F3CF33BE
:103C6000CEEA0343C9F800304FEA1C431B04A042CC
:103C700043EA1C431AD1AF4218D132FB03F231FBA5
:103C800013F322F3CF3223F3CF33C2EA0343C9F84D
:103C9000043009F10809C145CAD1DDF838805E4613
:103CA0004FEA880CDDF830B0FFF721BBB3F5803F59
:103CB0000DD31FFA83FCBCF1000F08D0002E00F0DA
:103CC0009D8083EA060C1CF0802F00F09780069AF6
:103CD0000B993D460446D0E7B3F5803F09D39AB22D
:103CE0003AB1002E00F0848083EA060212F0802FA1
:103CF0007ED03D460446A9E7B8F1010F7FF6C3AB7D
:103D0000020404990B924FEA58033A04CDE90EB825
:103D1000AAF1040A0C9201EBC30EB046CDF818C00C
:103D20005AF8043F4FF0802293FA42F91FFA89F3C0
:103D3000A04243EA09434BD1AF4249D122044FEAA2
:103D4000054C32FB03FB3CFB13F32BF3CF3B23F37C
:103D5000CF33CBEA03430E6893FA16F30B604FEAB6
:103D600019431B04A04243EA19431BD1AF4219D1A6
:103D700032FB03F23CFB13FC22F3CF332CF3CF32A4
:103D8000C3EA02424B6892FA13F34B6008318E4546
:103D9000C6D14646DDF83C80DDF838B04FEA880CE5
:103DA000FFF7A5BAB3F5803F0DD31FFA83F9B9F138
:103DB000000F08D0069E26B183EA060919F0802F6D
:103DC00001D10693D4E7DDE90B2C3D460446CFE74D
:103DD000B3F5803F09D39AB23AB1069A1AB15A4064
:103DE00012F0802F01D10693A8E73D460446A5E7CF
:103DF0001E462BE7984606E6984623E61E463CE715
:103E0000BBF1000F7FF4C4ADFFF7BCBA2DE9F0435E
:103E100008468BB011461A462E4B04ACCDE900344F
:103E2000062332F06FF84FF4CF63FF22012104988C
:103E300032F0C4F840F211330222012107460698FD
:103E400032F0BCF84FF4B16204460121099832F017
:103E5000A9F8079D082D804601D0102D37D107F114
:103E60000D001D4980003CF0CFFCE4B29DF82030ED
:103E70000093059ACDF808800194EBB2F9B206469A
:103E800009F0D8FE002F17DDDFF8548098F80830CD
:103E900008EB830306F13005D3F8109000240023CB
:103EA00019461A464046C847013445F8040F3146C2
:103EB00009F084FFA742F2D196F82C0006F13401F4
:103EC0003DF034F9306330460BB0BDE8F083034871
:103ED0006DF0BEF8ACCC0B00FCCC0B0050820B009C
:103EE000F0CD0B0000B583B0019000F0A5FB019868
:103EF00009F0DCFE00280CBF1E203E2003B000BDF0
:103F000000B583B0019000F097FB0198006B03B0FF
:103F100000BD00BF30B551F8044B89B005462046BE
:103F2000CDE9022100F088FB05AB01930E4B009315
:103F3000DDE902210323681E31F03CFF94F82C20B8
:103F40009DF818309A420AD904EB83039DF81C208F
:103F5000586B059909F0EEFE204609B030BD40F2DD
:103F6000776031F019FF00BFE4CC0B0030B551F899
:103F7000044B87B005462046CDE9022100F05CFBEA
:103F800005AB01930C4B0093DDE902210123681E70
:103F900031F010FF94F82C209DF814309A4207D984
:103FA00004EB8304606B09F00BFF0E2007B030BDFB
:103FB00040F2776031F0F0FEDCCC0B0090F82C3052
:103FC0007BB170B5064600F13005002455F8040FAA
:103FD00009F0C2FE013496F82C20E3B29A42F5D8DB
:103FE00070BD704700B5084683B01146002231F01D
:103FF000A7FE054928203CF007FC019009F070FE5F
:10400000019803B000BD00BFF0CD0B0008B509F06A
:104010007FFE0E2008BD00BF09F080BE08B509F084
:104020007FFE00280CBF1E203E2008BD09F07ABE8E
:1040300008B509F079FE00280CBF1E203E2008BDFF
:1040400010B584B002AB51F8044B0193074B0093B9
:104050000138022331F0AEFE20469DF80C20029973
:1040600009F068FE0E2004B010BD00BFE0CD0B00CB
:1040700008B509F091FE0E2008BD00BF10B504463A
:1040800008463CF0D7F90146204609F08DFE0E2087
:1040900010BD00BF08B509F089FE0E2008BD00BFA5
:1040A00010B584B003AB51F8044B0193054B00935A
:1040B0000138012331F07EFE204609F081FE0E20FA
:1040C00004B010BDD8CD0B0008B509F0DDFE0E2000
:1040D00008BD00BFF0B5456A87B0002D00F0A48090
:1040E000044600295CD011460C98A568056094F937
:1040F0005400884256D0C2F1010284F8542094F84A
:104100004420B2FA82F2520904EB820184F844207E
:1041100084F855204A6B1A602046174631F0E4FCBB
:104120000021204631F09EFC014600286CD0D4E9E5
:104130000B239B1A0493636A134405930023009393
:1041400020693B4604AA05A9F5F774FD431C44D039
:10415000236B049A9B1AE362064650B100212A465B
:10416000384630F0ADFF94F84530002B3ED1023692
:104170003CD1A36D03EB55032046A36531F0B4FC9D
:104180000021204631F06EFC0546D4E90B01A26AFD
:10419000091A521AB2F5007F18DC284607B0F0BDA4
:1041A0000A46A1E794F9551004EB81010120496BFF
:1041B00001EB42021A60FF210C9B84F854101A682C
:1041C000A36D03EB5203A36507B0F0BD1849224667
:1041D00004F1140000F078FBDFE700212A4638469E
:1041E00030F06EFF94F84530002BC2D0A268002159
:1041F000384630F065FF0C99002201230A6084F8EC
:104200004530022007B0F0BDA2680391384630F077
:1042100057FF0C9B0399196094F8450080F001004A
:104220004000C0B207B0F0BD0C9B1D60E9E700BFC5
:10423000D55C060070B51E460D4686B01146284670
:104240001C4A31F07DFD34681B4B2340062B1ED0E9
:10425000A30718D00121204637F08CFA037C13F015
:10426000010324D1012D1AD81E46144901935C2064
:104270003CF0D2FA019B32462146054609F0A4FDE6
:10428000284606B070BD0E4B22689A42E2D1214604
:104290000C4845F2E62233F035FD0446DAE7706853
:1042A000062203A937F0F0F9DDE90363DDE70648EC
:1042B0006CF0BAFE040002000F0080FF14CF0B0068
:1042C00088630B00AC990B000C7E0B0000B583B02B
:1042D000019000F0B1F90198006C03B000BD00BF7F
:1042E00000B583B0019000F0A7F9019809F0DEFD58
:1042F000B4EE400AF1EE10FA09D610EE103A23F0AF
:10430000030040F00200A0F1FF4003B000BD0148EF
:10431000FBE700BF0200400000B583B0019000F051
:104320008BF9019809F002FE400040F0010003B053
:1043300000BD00BF10B582B00446019100F07CF9C9
:104340000199064845F2E62233F0DCFC014620469E
:1043500009F0EEFD0E2002B010BD00BFAC990B00BD
:1043600038B50C46054600F067F90121204637F0C4
:1043700001FA037CDB0705D42846214609F0D8FD65
:104380000E2038BD01486CF04FFE00BF0C7E0B00C4
:1043900009B1012A24D010B5044682B000F0E8FA31
:1043A00094F8453023B902B0BDE8104000F0BCBA23
:1043B0000022206C114662F0C5FC0028F3D1FF23D7
:1043C000C4E90B0084F84500A065019084F85430DE
:1043D000204631F089FB0199204631F043FBE2E7AA
:1043E000704700BF08B509F077FE0E2008BD00BF7A
:1043F00010B5084688B011461A46114B0DF1140C41
:10440000CDE9003C032331F07DFD059840F25B418E
:104410006FF0F6FF40F267510446069870F008F816
:104420000849039024203CF0F7F9BDF81C30039AAA
:104430000290214609F018FE029808B010BD00BF96
:1044400030D00B0058D00B0010B5044609F086FEA2
:1044500038B9204609F088FE00280CBF1E203E20F7
:1044600010BD59F053FB00BF10B5044609F076FEAD
:1044700038B9204609F07AFE00280CBF1E203E20E5
:1044800010BD59F043FB00BF10B5044609F066FEAD
:1044900040B9204609F06AFE30B1204609F072FEAC
:1044A0000E2010BD59F032FB01486CF09DFD00BF9D
:1044B000588A0B0030B50C6887B005462046CDE918
:1044C000022109F04BFEDDE9022188B904AB01931A
:1044D000084B0093681E0223043131F06BFC204628
:1044E0009DF81420049909F055FE0E2007B030BD48
:1044F00059F00CFB48D00B0010B5044609F02EFE15
:1045000050B9204609F030FE08B90E2010BD2046F3
:1045100009F0F4FE0E2010BD59F0F8FA10B504466B
:1045200009F01CFE20B9204609F0F8FE0E2010BD4F
:1045300059F0ECFA3E4BD3F80021D00050D510B51D
:104540003C4B84B003F1100453F8040BB8B1C27FA4
:1045500042B98168D1F804C1BCF1000F02D04277A2
:10456000C1F80421427F52B1827F62B18268D2F8E1
:10457000101141B3D2F8141169B3012151609C426A
:10458000E2D104B010BDC27F002AF8D190F82220F9
:10459000002AF4D18168D1F808C1BCF1000F38D1EC
:1045A000D1F80C214ABB90F91C20002AE7DB510905
:1045B000DFF87CC002F01F026031012000FA02F235
:1045C0004CF82120DBE7D2F808110029D7D1D2F826
:1045D00014110029D1D1D2F80C110029CFD1CCE788
:1045E000D3F804219107AAD4D3F804215207A6D402
:1045F000D3F804319B04A2D47047002102930190A8
:1046000026F016F80198029B82680021C2F80C116E
:10461000C9E70121CDE90232019026F009F801989D
:10462000039A8168029BC1F808218168B8E700BF3E
:1046300000E100E0380A012008B5437B03B108BD62
:1046400059F064FA407BB0FA80F04009704700BF2F
:10465000F0B583B004460E46014640F21450CDE951
:104660000032089D40F03AF907462046FFF7EAFF7E
:10467000DDE9003240B90895BD6831462046AC46B8
:1046800003B0BDE8F0406047002202201A602A60B3
:1046900003B0F0BD00234373704700BF30B583B053
:1046A0000C46054640F21450019240F017F920469E
:1046B000FFF7C2FF61686B68019A994211D16B7B69
:1046C00062B9627B9A421BD1227B2B7B9A4212D128
:1046D000A27BAB7B9A4209D103B030BD022BF0D153
:1046E000F2E70A484FF4B1616CF0BAFC074840F2B7
:1046F000BD516CF0B5FC05484FF439716CF0B0FC5D
:10470000024840F211316CF0ABFC00BF7C870B001B
:1047100008B5437B23B1007B400040F0010008BD99
:1047200059F0F4F9407B18B1400040F001007047A7
:1047300008B559F0EBF900BF00B5437B83B063B116
:104740000146019040F2145040F0C8F801994868C1
:10475000400040F0010003B000BD59F0D7F900BFA0
:1047600038B5437B6BB104460D46014640F2145008
:1047700040F0B4F828463AF0E7FC034663600E20A8
:1047800038BD59F0C3F900BF2DE9F04104460F468A
:1047900040F214502146164640F0A0F80546204647
:1047A000FFF750FF30B96B68324639462046BDE806
:1047B000F0411847BDE8F081704700BF014B00226F
:1047C0001A707047057B01200349044B0120002229
:1047D00008701A60704700BF057B0120286B01201C
:1047E000014B1878704700BF057B0120024B186809
:1047F000003818BF01207047286B012008B50D4B09
:10480000186818B10C4A12680AB1002008BD65F09A
:10481000FDF8084B1A681B688242A0EB030088BFB2
:1048200000F1FF3040F2EE23984294BF00200120B7
:1048300008BD00BF286B01209C460120014B0022CF
:104840001A607047286B0120024A136823EA0003AC
:10485000136070479C460120024A136803431360AB
:10486000704700BF9C460120134B1B7813B1134BBC
:104870001B6803B1704700B5114B83B01A680192F1
:1048800065F0C4F80E4B019A1860196811B132B185
:1048900003B000BD196801311960002AF8D1012068
:1048A00064F0A0FB074B03F178029A6203B05DF855
:1048B00004EB56F0E9BF00BF057B01209C460120B8
:1048C000286B012040700120C0E9001200F000B800
:1048D00000B583B0019012F033F80198C368BBB9FA
:1048E0000F490A68824213D00E4A8360D2F800C092
:1048F0001368C0F80CC00BB1136898600B6863B103
:10490000106012F063F803B05DF804EB56F0BCBF22
:1049100003B05DF804EB12F059B80860F0E700BF8F
:10492000AC460120B446012008B512F009F8044A4B
:104930001368013B1360BDE8084012F047B800BFA0
:10494000A046012010B5054B1C682CB1606827F00B
:104950007BFEA468002CF9D110BD00BFAC4601203D
:10496000024B1868003818BF01207047AC46012080
:1049700008B511F0E5FF044A136801331360BDE880
:10498000084012F023B800BFA04601202DE9F043F3
:10499000DFF8709083B00027019711F0D1FFD9F8AC
:1049A00000504DB30DF104083E4602E00023E360E1
:1049B000ADB12C462846AD68A66028F035F9002830
:1049C000F4D1606828F030F90028EFD13B46C8F8F0
:1049D0000040274604F10808E360002DE9D1019A60
:1049E0000649074BC9F8002000220F601A6011F039
:1049F000EDFF03B0BDE8F0832F46F0E7B446012099
:104A0000A0460120AC4601202DE9F041164E56F09B
:104A100003FE336833B3DFF8588011F091FFD8F804
:104A20000050DDB93468114B35600122C8F8002010
:104A30001D608CB12346D3E90067A468C3E9025521
:104A400011F0C4FF384606B1B04711F079FF002CD1
:104A5000F0D1D8F80050013DC8F80050BDE8F04151
:104A600011F0B4BFBDE8F081AC460120B44601208E
:104A7000A046012008B53AF0E1FB03460348D98877
:104A8000972914BF972242226CF0D6FA68810B0056
:104A9000014A042357F038BC74160C0000B50846D0
:104AA00089B011461A460B4B0DF1100CCDE9003CB4
:104AB000042331F027FA084918203BF0ADFEDDE968
:104AC0000631059A0091049903905DF0FBFB039871
:104AD00009B000BD58D10B00F0D10B0008B55DF056
:104AE00037FC0E2008BD00BF10B504465DF04EFC3B
:104AF00038B920465DF0DEFC00280CBF1E203E20A9
:104B000010BD59F003F800BF10B504465DF03EFC3F
:104B100020B920465DF0E0FC0E2010BD58F0F6FFF5
:104B200038B504460D465DF031FC78B920465DF09D
:104B300031FC68B128463AF007FBC1B220465DF06F
:104B40002BFC00280CBF1E203E2038BD58F0DEFF95
:104B500007F040F9F0B50C6887B0064620460D46D0
:104B600017465DF013FCC0B920465DF013FCB0B1F0
:104B700002AB01930B4B00930423E9183A46701ED5
:104B800031F018F9DDE90430DDE902120090204629
:104B900059F0B4FC0E2007B0F0BD58F0B7FF07F095
:104BA00019F900BFD0D10B0070B505465DF0EEFBE2
:104BB000F8B9044628465DF0EDFBE0B121462046F9
:104BC0003CF02AF90824064602E00134782C0ED085
:104BD000E1B228465DF0E0FB0028F6D0610041F02C
:104BE0000101304601343BF0ABFC782CF0D130466B
:104BF00070BD58F08BFF07F0EDF800BFF0B50C6802
:104C000087B0064620460D4617465DF0BFFBD0B97B
:104C100020465DF0BFFBC0B102AB01930C4B00938B
:104C200004233A46E918701E31F0C4F8DDE9043176
:104C30000120CDE90010039A0299204671F0C2FBD1
:104C40000E2007B0F0BD58F061FF07F0C3F800BFB9
:104C500078D10B002DE9F0410C688AB00746204658
:104C60000E4690465DF092FB18BB054620465DF06F
:104C700091FB00B3114B009303AB4246311D781EEC
:104C80000193072331F096F8DDE90631049ACDE966
:104C900000152046039971F095FBDDE90830059A6F
:104CA00000900399204659F029FC0E200AB0BDE877
:104CB000F08158F02BFF07F08DF800BF98D10B0062
:104CC0002DE9F0410C6886B0074620460E46904616
:104CD0005DF0EAFC88BB054620465DF0E9FC70B358
:104CE000184B009302AB4246311D781E01930423FA
:104CF00031F060F82946039840F20353012231F065
:104D00005DF92946064640F2F3430498012231F04A
:104D100055F940F2E223054609220598082131F0B1
:104D20004DF9C0B2009002992046EBB2F2B25DF0AC
:104D30000FFC0E2006B0BDE8F08158F0E7FE0248F7
:104D40006CF052F938D30B00608D0B0000B50846AB
:104D500089B011461A460A4B0DF1140CCDE9003CFE
:104D6000032331F0CFF8074918203BF04DFDDDE972
:104D70000623059903905DF013FC039809B000BD6C
:104D8000B8D20B0058D30B0008B55DF05FFC0E20C5
:104D900008BD00BF10B504465DF086FC38B920465A
:104DA0005DF098FD00280CBF1E203E2010BD58F07D
:104DB000ADFE00BF10B504465DF076FC20B920467C
:104DC0005DF09EFD0E2010BD58F0A0FE2DE9F041D3
:104DD0000D688CB0074628460E4690465DF064FC90
:104DE000002842D1044628465DF062FC002839D0F4
:104DF0001F4B009308AB4246311D781E01930423DC
:104E000030F0D8FF062205A9089836F03DFC22466E
:104E10009DF81C10402031F003FA0446DDE9090139
:104E200004AA039003A8069BB3FBF4F304934FF08A
:104E30008DFADDE9031304FB01F103FB04F2CDE974
:104E400003121AB90E200CB0BDE8F08105989DF848
:104E50002C30014428465DF02FFC0028F2D10520BB
:104E60006CF092F803486CF0BFF858F04FFE00BFAA
:104E700000D30B00608D0B002DE9F0410D688AB066
:104E8000074628460E4690465DF00EFC002840D1AD
:104E9000044628465DF00CFC002837D01E4B0093DA
:104EA00004AB4246311D781E0193032330F082FF8C
:104EB000052207A9049836F0E7FB22469DF8241046
:104EC000402031F0ADF90446DDE9050103AA029066
:104ED00002A8089BB3FBF4F303934FF037FADDE924
:104EE000023204FB03F304FB02F2CDE902321AB9E9
:104EF0000E200AB0BDE8F0810799284619445DF0FC
:104F000005FD0028F4D105206CF03EF803486CF054
:104F10006BF858F0FBFD00BF20D30B00608D0B0039
:104F20002DE9F0410E6892B0074630460C46904697
:104F30005DF0BAFB002866D1054630465DF0B8FB4F
:104F400000285DD0314B00930CAB211D4246781EEA
:104F50000193062330F02EFF052206A90C9836F0A7
:104F600093FB2A469DF82010402031F059F9044661
:104F7000DDE90E0103AA029002A8079BB3FBF4F33C
:104F800003934FF0E3F9062209A90D9836F07CFB54
:104F90002A469DF82C10402031F042F90546DDE903
:104FA000100105AA049004A80A9BB3FBF5F305932E
:104FB0004FF0CCF9DDE90213049A059804FB03F3E2
:104FC00005FB02F200FB05F504FB01F1AB42CDE964
:104FD00003320291059510D11BB90E2012B0BDE825
:104FE000F0810998069C0244214430465DF0ECFBB8
:104FF0000028F2D105206BF0C7FF05486CF028F8B7
:1050000004486BF0F1FF58F081FD00BFD0D20B00D7
:1050100018820B00608D0B002DE9F843047B076EAE
:10502000064604F01F044FF0FF33A3408C42006893
:105030007568884627EA030728D24FF0000919E06F
:1050400038B9B568B36F4FF40072294630469847B7
:1050500070B315F8013B0138B9F1000F10D023B33C
:1050600086F864304FF00009FF230834A04543EA76
:1050700007270BD996F86430002BE1D0FF23F4E723
:10508000FF2BF2D1A0454FF00109F3D8C6E9000586
:105090002346A3EB0803A4EB080404F01F043766BF
:1050A000337327FA04F0BDE8F8839946FF23DCE761
:1050B0006FF00100BDE8F8830EF000BA2DE9F0436F
:1050C00017885488B2F80480D58893B02422E41B52
:1050D00006468946013400210DEB02002FF0F0FF57
:1050E00004EBD4735B104FF48871B6F94A2EADF817
:1050F0003030B6F9463EADF83210A5EB0805012177
:1051000001350D9193424FF6FF71CDF82C90ADF81B
:105110002840ADF82A50ADF844103BDCB6F9440EF7
:10512000B6F9481E884231DCC91BA142A2EB080235
:10513000A8BF21469542A8BF1546B6F8402EB6F83E
:10514000424EA3EB0803C01B4ABF121A00B2002054
:10515000002BB6BFE41A1BB20023CDE9000309B24D
:105160002DB20291039523B296F8554ED6F83C0E17
:105170000794D6F8504E069496F8544E0594D6F8F7
:105180004C4E049412B209A909F0A6FC012013B0F8
:10519000BDE8F083002013B0BDE8F083F0B50E2A1F
:1051A00083B06CD0154604460E460EF043F9002835
:1051B00068D1B2072CD0F30731D5A188E38801FB71
:1051C00003F3B3EB660F4FEA660052D990FBF1F29E
:1051D00001FB1200042D06B217B240D0284639F068
:1051E000B3FF054620460EF067F94FF0FF32C0F1DD
:1051F0002003DA402846A223002130F0DFFE3A46A1
:105200000346314620460EF0B9F90E2003B0F0BD3A
:10521000214B32689A42CED120486BF0A1FE304635
:1052200001AA022139F0AAFE019B186839F08CFF0F
:10523000061EA38828DB9E4226DA019B586839F0B7
:1052400083FF021EE38803DB9A42B8BF3046C1DB0E
:105250001348013B002240F29C616BF075FE3A4618
:10526000314620460EF04CF9400040F0010003B0FA
:10527000F0BD0B48013B00225C216BF065FE094844
:105280006BF04AFE58F042FC0548013B002240F218
:1052900096616BF059FE00BF6C600B003C880B0000
:1052A0007C940B007C900B00F0B52F4B8DB007ACBD
:1052B000CDE90034052330F07DFD2C49079840F2FC
:1052C0006B3230F00DFF294940F2E452DDE907501E
:1052D00030F006FFDDE90860244940F2E55230F085
:1052E000FFFEDDE9097420463AF090FF10BB012271
:1052F00004A9204636F0C8F940B3059BB3F5805F9A
:1053000024D1049B13B30B980E2811D040F27B429A
:105310001649039330F0E4FE0B9A039B0093284652
:10532000134631463A465DF057FB07980DB0F0BD85
:105330000022F3E721460E4832F0BAFC044601226F
:1053400004A9204636F0A0F90028D6D1204639F02D
:1053500075FFC288009207484FF4087343224FF448
:105360008E616BF069FE00BF44D40B0004E70B00B4
:10537000A0D50B0018940B0030B5174B87B003ACC9
:10538000CDE90034032330F015FD1449039840F2B1
:10539000DF2230F0A5FE124940F2E742DDE903507A
:1053A00030F09EFE049C40F2E742A0684FF480710A
:1053B00030F014FE05980E280CD0084940F27B42CC
:1053C00030F08EFE0599626828465DF03FFC039838
:1053D00007B030BD0021F6E77CD40B0004E70B00DA
:1053E00028EB0B002DE9F04F2DED028B5F4BA9B0A0
:1053F00005ACCDE90034032330F0DCFC5C490598B2
:1054000040F2DF2230F06CFEDDE90530039339F025
:1054100015FFC37B002B40F08E80069D2E462F4645
:1054200028AB0DF12008B3EE0F8A0DF11F040DF12A
:105430003F09C3F1810A0AEB040307EE103AB8EE04
:10544000C77A2846C7EE087A17EE903AF4EE677AE4
:10545000F1EE10FA23F0030B4BF0020B6CBFDFF8F8
:1054600018B1ABF1FF4B594632F022FC39F0FEFD8A
:1054700020EE080A5AF022FAFDEEC07AB54217EE85
:10548000902A594604F8012F30460BD032F010FC18
:1054900039F0ECFD20EE080A5AF010FAFDEEC07A61
:1054A00017EE902A4C4584F86020C4D16FF01E049A
:1054B0009FED308A304D08F15F06A4EB080404EB41
:1054C000090307EE103AB8EEC77A3846C7EE087AF5
:1054D00017EE903AF4EE677A23F00301F1EE10FA3A
:1054E00041F0020174BFA1F1FF41294632F0E0FB17
:1054F00039F0BCFD20EE080A5AF0E0F9FDEEC07A62
:1055000017EE903A09F8013F4E45D8D107980E287A
:105510000FD0174940F27B4230F0E2FD0799039823
:1055200042465DF01BFC059829B0BDEC028BBDE83E
:10553000F08F0021F3E7069839F080FE04460698C4
:1055400039F07CFEC27B0D4B04EB820422699A4247
:105550007FF463AF069C4FF48E626068032130F0E5
:105560003DFDD4E9025726695AE700BF94D40B00E9
:1055700004E70B0000007C4202004000ED2E070013
:105580002DE9F0414F4B92B003ACCDE90034032339
:1055900030F010FC4C49039840F2DF2230F0A0FDBF
:1055A0003022002106A8039F2FF08AFD049E16F0EA
:1055B000030410D0304639F041FEC288434840F21F
:1055C0001313CDE9003240F239214FF4897340F2D0
:1055D0003A226BF045FD33683D4A93423FD03D4A45
:1055E00093424ED03C4A934221D03C4A9342E1D16F
:1055F00006AD44F00101042230463DF027FB39F0AE
:1056000035FD0234182CA5EC010AF2D105980E28BC
:1056100023D02D4940F27B4230F062FD0599384697
:1056200006AA5DF0EDFB039812B0BDE8F0812C4BAB
:10563000610041F0010104223046A3FB04353DF036
:1056400005FB39F013FD04EB550501340DEB850521
:10565000092C85ED060AEAD1D8E70021DFE706AD7F
:1056600044F00101042230463DF0F0FA39F0FEFC2E
:1056700002342B46062C05F1140583ED000AEFD108
:10568000C4E70DF1180845460224A11E41F00101AE
:10569000042230463DF0DAFA39F0E8FC44F001012A
:1056A00088ED000A042230463DF0D0FA39F0DEFCE5
:1056B00004340E2C85ED030A08F1140805F11005D9
:1056C000E3D1A3E7C4D40B0004E70B008C720B00FA
:1056D000F0D60B00A0D60B0044D60B00DCD50B0097
:1056E000ABAAAAAA2DE9F04F2DED028B8FB04F4B3C
:1056F00004AF07F10804CDE90034082330F05AFB69
:105700004B49B86840F2DF2230F0EAFC786ABB68A7
:105710007B600E286ED0464940F27B4230F0E0FCC0
:105720007B6A3B60786939F0A1FCD7F80C80404671
:10573000B0EE408A3AF0BEFE002869D0C30767D5B4
:10574000461007EE906AB8EE670AB5EE400AF1EE31
:1057500010FA58D4F1EEC07AFDEEE77A17EE909A7F
:1057600019F0010F5FD009FB09F39E425BD1B30032
:10577000073323F00703ADEB030D0DF1100A002EE4
:105780003BD00024AAF1040B25466100042241F01D
:10579000010140463DF05AFA39F0D6FC0134A642E8
:1057A0004BF8040F0544F0D138690E2818D039F0B1
:1057B0005DFC97F820203B7FCDE901323B7E0093D2
:1057C000D7E90010F0EE480A53464FEA59025DF05F
:1057D000CBFBB8682C37BD46BDEC028BBDE8F08F23
:1057E00075B107EE905AF8EEE77AB7EE007A87EED9
:1057F000270ADEE700233B6094E738690E28D6D1FC
:10580000B7EE000AD5E75FF059FDF0EE407AA3E766
:10581000404639F013FD40F23F22C388054840F26C
:1058200084616BF01DFC04486BF012FCDCD40B00AF
:1058300004E70B00FC930B00A4720B0000B52DEDE8
:10584000028B184B89B00DF1140CCDE9003C0323F9
:1058500030F0B0FA0698F8B139F008FCB0EE408AA2
:105860001149059840F2DF2230F03AFC0798059B79
:105870000E2814D00C49039340F27B4230F030FCE8
:105880000799039B1846B0EE480A5DF0BDFD0598E8
:1058900009B0BDEC028B00BDB6EE008AE0E7002146
:1058A000F0E700BFACD40B0004E70B002DE9F04F8C
:1058B0002DED028B624B93B008ACCDE900340A2386
:1058C00030F078FA5F4908984FF45B7230F008FCCA
:1058D0005C4940F2D5520546099830F001FC59491F
:1058E000064640F2D6520A9830F0FAFB07460C986A
:1058F0000E2800F0848039F0B9FBB0EE408A0D9894
:105900000E2875D039F0B2FBF0EE408A0B994E4864
:105910004FF44A721BF040FA40F2ED220E99044611
:105920004A481BF039FAAA88B3889342804677D157
:10593000EA88F188914273D1A87BB27B82426FD111
:10594000B88898426CD1FB888B4269D1B97B91426F
:1059500066D1E4B2092C69DC0123A34013F0AA0F3D
:1059600041D1092C62D1082966D10F980E2852D056
:1059700039F0EAFB4FF0000A814610980E2841D01A
:1059800039F0E2FB034611980E284FF0000B40D08F
:105990002C49079340F27B4230F0A2FBAA88818811
:1059A000914240D1C188EA88079B91423BD1827BDA
:1059B000082A3ED1CDE902A35FFA88F3CDE904B00D
:1059C00000932846CDF80490F0EE680AB0EE480A3D
:1059D00023463A46314608F0CBFC0E2013B0BDEC0E
:1059E000028BBDE8F08F1029BFD019486BF030FB57
:1059F000F7EE007A77EEC87AF0EE678A86E7B6EEC1
:105A0000008A7CE711980E284FF0010B4FF000033D
:105A1000BED10020CEE74FF0010A4FF00009ACE7FD
:105A20000C486BF015FB0C486BF012FB0B486BF04D
:105A30000FFB0B486BF00CFB0A486BF009FB00BF37
:105A400010D90B0004E70B0060E80B0038DB0B00FB
:105A5000748D0B0064910B00C48B0B0018850B0038
:105A6000D88B0B00908D0B002DE9F0432E4B97B097
:105A70000FACCDE90034072330F09CF92B490F9887
:105A800040F2DF2230F02CFB054605220CA91098CD
:105A900035F0FAFDEC88264BAA8811A90AA800F077
:105AA000F3FB2246234B12A90DF12A0000F0ECFB78
:105AB000BDF92860BDF92A70BDF92C80BDF92E9082
:105AC0009DF83810A9EB07030022A8EB060440203C
:105AD00003FB04F430F0A4FB15990D9BB3FBF0F32A
:105AE0000E2902461BD0CDE908300846079139F04F
:105AF0002BFBDDE90713099A9C4212D80E3918BF17
:105B00000121049003912846CDE901890C99009761
:105B1000334608F073FF0E2017B0BDE8F083002075
:105B2000EAE705486BF008FA10D80B0004E70B0011
:105B3000D0D90B00C8D90B00387C0B0013460A469D
:105B4000014640F2E1201BF015B900BF70B52B4BA8
:105B500086B002ACCDE90034042330F02BF928499B
:105B6000039840F2D45230F0BBFA254905464FF471
:105B70005B72029830F0B4FA0599044640F2A7220D
:105B800020481BF009F940F2D952049906461E48F4
:105B90001BF002F9AA88A3889A4223D1EA88E388F5
:105BA0009A421FD1A37B102B01D0012B20D1C2B26E
:105BB000092A1ADC0123934013F0AA0F0CD1092AF9
:105BC00013D1AB7B082B16D12046F3B2294609F03E
:105BD00075F90E2006B070BDAB7B102BF4D00B48CE
:105BE0006BF022FA0A486BF01FFA0A486BF01CFAB5
:105BF00009486BF019FA09486BF016FAB8D70B0090
:105C000004E70B008CDA0B0060E80B0010750B004A
:105C100058820B0020730B0020750B0004750B00DD
:105C200013460A46014640F2E1201BF0A3B800BF2C
:105C30002DE9F04F394B97B00CACCDE900340A2375
:105C400030F0B8F836490C984FF45B7230F048FAEF
:105C500040F296638288044600210E9830F0AEF937
:105C600040F29C63E288002182460F9830F0A6F94A
:105C70002B4940F2D45283460D9830F031FAC68851
:105C80008288284B054610A90AA800F0FDFA324682
:105C9000254B11A90DF12A0000F0F6FAA27BAB7B8F
:105CA000BDF92860BDF92A70BDF92C80BDF92E9090
:105CB0009A422FD314980E2822D039F045FA034681
:105CC00015980E284FF0000221D0CDE9083239F0A6
:105CD0003BFADDE908320021CDE90601CDE90432C5
:105CE0002046CDE90289CDE900670FFA8BF30FFA60
:105CF0008AF2294608F0F0FE0E2017B0BDE8F08FBA
:105D000015980E284FF001024FF00003DDD101215C
:105D10000020E1E705486BF09BF900BF40D70B007E
:105D200004E70B00D0D90B00C8D90B0030750B006D
:105D300000B51E4B89B00DF10C0CCDE9003C0523DC
:105D400030F038F84FF45B721949039830F0C8F915
:105D5000837BDDF818C001229A4094451FD2079B2F
:105D60006FF000418B4201D09A421BD9BDF910104F
:105D7000002911DB828891420EDABDF91420002A35
:105D80000ADBB0F806E0724506DA0093634608F0D5
:105D900073FF0E2009B000BD06486BF059F90648A4
:105DA0006BF056F905486BF053F900BFA0D80B0013
:105DB00004E70B00A0760B00C4720B008C820B0072
:105DC0002DE9F0411E4B88B003ACCDE9003405232A
:105DD0002FF0F0FF4FF45B721A49039830F080F90E
:105DE000827B079D012393409D4225D2BDF910601F
:105DF000BDF91470BDF918808288044640F296639C
:105E00000021304630F0DAF8E28840F29C6300214D
:105E1000384630F0D3F840F225520021404630F0A9
:105E2000C1F82046009543463A46314609F0B4F998
:105E30000E2008B0BDE8F08103486BF009F900BFFF
:105E400090D70B0004E70B00A0760B0000B5134BB6
:105E500089B00DF1080CCDE9003C06232FF0AAFF14
:105E60000F4902984FF45B7230F03AF9827B079940
:105E70000123934099420ED2BDF918C0BDF91430E8
:105E8000BDF91020CDE900C1BDF90C1009F046FAAA
:105E90000E2009B000BD03486BF0DAF870D80B0093
:105EA00004E70B00A0760B0030B5264B91B00BAC8D
:105EB000CDE9003405232FF07DFF23490B984FF4E3
:105EC0005B7230F00DF9052205A905460C9835F0F6
:105ED000DBFB052208A90D9835F0D6FB9DF81C10B8
:105EE0000022402030F09CF99DF828100446002242
:105EF000402030F095F984421AD1069B099AB3FBF1
:105F0000F4F3B2FBF4F2934218D1A87B0E9901226C
:105F1000824091420FD29DF83C200292CDE900418F
:105F20002846089A059909F033FA0E2011B030BDC1
:105F300006486BF08DF806486BF08AF805486BF060
:105F400087F800BF48D80B0004E70B006C8F0B00EC
:105F5000A0760B00848F0B0070B51B4B8AB004AC8D
:105F6000CDE9003406232FF025FF4FF45B7217496B
:105F7000049830F0B5F8827B099D012393409D423F
:105F80001FD28288124B0446C08805A9064602A883
:105F900000F07AF9324606A90DF10A000D4B00F027
:105FA00073F9BDF90E10BDF90C30BDF90A20CDE929
:105FB00000152046BDF9081009F07CFA0E200AB041
:105FC00070BD05486BF044F8C8D80B0004E70B001F
:105FD000D0D90B00C8D90B00A0760B0000B5114B2F
:105FE00087B00DF10C0CCDE9003C03232FF0E2FE4D
:105FF0000D49039840F2DF2230F072F8827B049959
:1060000001239340994207D2059A9A4204D209F09B
:10601000DBFC0E2007B000BD044840F223316BF0DA
:106020001FF800BFF8D80B0004E70B00D8930B0053
:106030002DE9F0432DED028B5A4BA1B013ACCDE905
:1060400000340D232FF0B6FE574913984FF45B72BE
:1060500030F046F840F2D45204465349149830F0D8
:106060003FF8A27B837B9A42C0F098800546159842
:106070000E2800F08F8039F067F80FFA80F9169833
:106080000E2800F0838039F05FF80FFA80F8199835
:106090000E2878D039F058F806B21A980E286FD02A
:1060A00039F052F807B2189B00930DF142030293A6
:1060B00010AB179901930FAA0DF13E0320466DF026
:1060C000E9FF1C9B00930DF14A03029312AB01936D
:1060D00028461B990DF1460311AA6DF0DBFF1D98B0
:1060E0000E284AD038F0C2FFB0EE408A1E980E2823
:1060F0003BD038F0BBFFB5EEC00AF1EE10FAF0EE7F
:10610000400A32D41F980E2834D0CDED0D0A39F054
:106110001BF8DDED0D0A0023CDE90A03BDF942307D
:10612000BDF9402005972046BDF94A400994BDF9C4
:1061300048400894CDE90235BDF94640BDF93E30EE
:106140000794BDF944400496CDE90032B0EE480A08
:10615000BDF93C3006944246494609F061FC0E20E8
:1061600021B0BDEC028BBDE8F0831F980E28F7EE3E
:10617000000ACAD101230020CEE79FED0C8AB5E7C3
:10618000EF887F088FE7AE88760886E7E3884FEAD6
:1061900053087CE7A3884FEA530970E704486AF084
:1061A00057FF00BF60D90B0004E70B0000000000A0
:1061B00030750B0000B52E4B8DB00DF1140CCDE9F0
:1061C000003C07232FF0F6FD2A49059840F2DF2214
:1061D0002FF086FFDDF820C00CF1FF33012B20D912
:1061E000BCF1040F40D1079B022B2FDDA3F1040E5D
:1061F000BEF11C0F2CD8204A012101FA0EF10A40F1
:1062000052B39DF82C109DF82820CDE901219DF86E
:10621000242000920699624609F08CF90E200DB0F8
:1062200000BD079B022B11DD1A1F1C2A10D8124932
:106230004FF0010E0EFA02FE0EEA01010029E0D134
:10624000142A05D1BCF1010FDBD008E0002BD8DC0B
:106250000A4819466AF004FFBEF1140FF8D1084845
:10626000182261466AF0FCFE064861466AF0F8FEB4
:10627000D8D70B0004E70B0011100010287B0B008F
:10628000187B0B00047B0B00F8B50F461D46196800
:106290000646144638682FF077FF2B680021224607
:1062A0002FF08CFE3080B8680E2809D069682FF076
:1062B0006BFF22466B68B6F900102FF07FFE044694
:1062C000B480F8BD30B585B004461D4602A8094B20
:1062D0000191FFF7D9FF0199074B0DF10A002A46FA
:1062E0000431FFF7D1FF02AB03CB20602046616091
:1062F00005B030BDD0D90B00C8D90B002DE9F04353
:106300000D4685B0002191464AF0B0FC04460021BC
:1063100028464AF0ABFC2379662B68D00379662BBC
:10632000054664D0002308208DF80F302CF0C6FEFF
:10633000804608202CF0CEFE074608202CF0CAFE2E
:106340004346CDE9007006460DF10F02294620466E
:106350004AF00CFA00284DD0B9F1040F56D8DFE806
:1063600009F01A25303B03002046CDE900769DF860
:106370000F202946434601F0B7F8044640462CF06A
:106380009BFE38462CF098FE30462CF095FE2046B9
:1063900005B0BDE8F0832046CDE900769DF80F20DA
:1063A0002946434600F03CF80446E7E72046CDE99D
:1063B00000769DF80F202946434600F017FA044660
:1063C000DCE72046CDE900769DF80F2029464346BC
:1063D00000F0F2FB0446D1E72046CDE900769DF8B7
:1063E0000F202946434600F0CDFD0446C6E7084885
:1063F0006AF02EFE40462CF05FFE38462CF05CFE24
:1064000030462CF059FE03486AF022FE0024B5E71E
:1064100020780B0050770B000022FFF76FBF00BF02
:106420002DE9F043074610463A7983B08C46622A3C
:1064300019460A9D0B9EFB69DCF81C405ED019D8FA
:10644000422A2CD0482A11D19CF804E0BEF1480F12
:1064500000F00C81BEF1680F00F02D81BEF1620FDB
:1064600055D003D8BEF1420F00F08280002003B067
:10647000BDE8F083682AF9D19CF80420682A00F06E
:106480004081622A43D0F1D89946B046BE46422A9E
:1064900023462E4667464C464546F446D2D19CF8E4
:1064A0000420622A00F095806AD8422A3BD0482A0C
:1064B000DCD101934CF014FF019BD0F81CC04FF0CD
:1064C000000E002127881A783A402CF8022B026926
:1064D000D5F80480776801318A4243443C44F1D8BE
:1064E000296802FB18110B44316802FB1711C268BE
:1064F0000EF1010E72450C44E3D8B8E7A046AE4653
:1065000062461C463546BC464346764617463A79AF
:10651000622A00F01B81482A00F03D81682A7FD062
:10652000622A8DD9A2E701934CF0DAFE019BD0F8E4
:106530001CC04FF0000E002127781A783A400CF862
:10654000012B0269D5F80480776801318A424344FF
:106550003C44F1D8296802FB18110B44316802FB56
:106560001711C2680EF1010E72450C44E3D87EE7A4
:10657000B6461A462E462346BC46754614468EE756
:10658000682A7FF473AF01934CF0AAFE019BD0F808
:106590001CE000270021B4F800C01A7802EA0C02BF
:1065A0002EF8022B0269D5F80480D6F804C0013118
:1065B0008A4243446444EED8296802FB18110B4414
:1065C000316802FB1C11C2680137BA420C44E1D8A1
:1065D0004DE7682201934CF083FE019BD0F81CC06C
:1065E0004FF0000E002194F900701A783A402CF810
:1065F000022B0269D5F80480776801318A4243444E
:106600003C44F0D8296802FB18110B44316802FBA6
:106610001711C2680EF1010E72450C44E2D826E74C
:1066200001934CF05DFE019BD0F81CC04FF0000EB2
:1066300000211F8894F900203A402CF8022B0269AF
:10664000D6F804806F6801318A4244443B44F0D854
:10665000316802FB18110C44296802FB1711C2684B
:106660000EF1010E72450B44E2D800E701934CF0A5
:1066700037FE019BD0F81CC04FF0000E0021278888
:106680001A883A402CF8022B0269D5F80480776802
:1066900001318A4243443C44F1D8296802FB181175
:1066A0000B44316802FB1711C2680EF1010E7245EE
:1066B0000C44E3D8DBE6724601934CF011FE019BDB
:1066C000D0F81CC04FF0000E002127881A883A40ED
:1066D0002CF8022B0269D5F80480776801318A42D0
:1066E00043443C44F1D8296802FB18110B4431683B
:1066F00002FB1711C2680EF1010E72450C44E3D87B
:10670000B5E601934CF0ECFD019BD0F81CC04FF0B6
:10671000000E002127881A883A402CF8022B0269C3
:10672000D5F80480776801318A4243443C44F1D86B
:10673000296802FB18110B44316802FB1711C2686B
:106740000EF1010E72450C44E3D890E601934CF033
:10675000C7FD019BD0F81CC04FF0000E00211F7830
:1067600022783A400CF8012B0269D6F804806F6851
:1067700001318A4244443B44F1D8316802FB18118C
:106780000C44296802FB1711C2680EF1010E724514
:106790000B44E3D86BE601934CF0A2FD019BD0F8CB
:1067A0001CC04FF0000E00211F8894F900203A40D1
:1067B0002CF8022B0269D6F804806F6801318A42F6
:1067C00044443B44F0D8316802FB18110C4429685A
:1067D00002FB1711C2680EF1010E72450B44E2D89C
:1067E00045E600BF0122FFF789BD00BF2DE9F04358
:1067F000074610463A7983B08C46622A19460A9DAC
:106800000B9EFB69DCF81C405ED019D8422A2CD0C4
:10681000482A11D19CF804E0BEF1480F00F00C8129
:10682000BEF1680F00F02D81BEF1620F55D003D884
:10683000BEF1420F00F08280002003B0BDE8F0837B
:10684000682AF9D19CF80420682A00F04081622A65
:1068500043D0F1D89946B046BE46422A23462E463A
:1068600067464C464546F446D2D19CF80420622A3D
:1068700000F095806AD8422A3BD0482ADCD10193A7
:106880004CF02EFD019BD0F81CC04FF0000E0021F3
:1068900027881A783A432CF8022B0269D5F804802D
:1068A000776801318A4243443C44F1D8296802FBAD
:1068B00018110B44316802FB1711C2680EF1010E6A
:1068C00072450C44E3D8B8E7A046AE4662461C4683
:1068D0003546BC464346764617463A79622A00F06A
:1068E0001B81482A00F03D81682A7FD0622A8DD919
:1068F000A2E701934CF0F4FC019BD0F81CC04FF0D0
:10690000000E002127781A783A430CF8012B02690F
:10691000D5F80480776801318A4243443C44F1D879
:10692000296802FB18110B44316802FB1711C26879
:106930000EF1010E72450C44E3D87EE7B6461A46C6
:106940002E462346BC46754614468EE7682A7FF4D9
:1069500073AF01934CF0C4FC019BD0F81CE00027FE
:106960000021B4F800C01A7842EA0C022EF8022B7B
:106970000269D5F80480D6F804C001318A42434444
:106980006444EED8296802FB18110B44316802FBFD
:106990001C11C2680137BA420C44E1D84DE76822A5
:1069A00001934CF09DFC019BD0F81CC04FF0000EF1
:1069B000002194F900701A783A432CF8022B0269EE
:1069C000D5F80480776801318A4243443C44F0D8CA
:1069D000296802FB18110B44316802FB1711C268C9
:1069E0000EF1010E72450C44E2D826E701934CF0FB
:1069F00077FC019BD0F81CC04FF0000E00211F88CF
:106A000094F900203A432CF8022B0269D6F804804E
:106A10006F6801318A4244443B44F0D8316802FB3C
:106A200018110C44296802FB1711C2680EF1010EFF
:106A300072450B44E2D800E701934CF051FC019BF6
:106A4000D0F81CC04FF0000E002127881A883A4366
:106A50002CF8022B0269D5F80480776801318A424C
:106A600043443C44F1D8296802FB18110B443168B7
:106A700002FB1711C2680EF1010E72450C44E3D8F7
:106A8000DBE6724601934CF02BFC019BD0F81CC056
:106A90004FF0000E002127881A883A432CF8022B69
:106AA0000269D5F80480776801318A4243443C4446
:106AB000F1D8296802FB18110B44316802FB171149
:106AC000C2680EF1010E72450C44E3D8B5E601939D
:106AD0004CF006FC019BD0F81CC04FF0000E0021CA
:106AE00027881A883A432CF8022B0269D5F80480CB
:106AF000776801318A4243443C44F1D8296802FB5B
:106B000018110B44316802FB1711C2680EF1010E17
:106B100072450C44E3D890E601934CF0E1FB019BF5
:106B2000D0F81CC04FF0000E00211F7822783A43A5
:106B30000CF8012B0269D6F804806F6801318A4293
:106B400044443B44F1D8316802FB18110C442968D5
:106B500002FB1711C2680EF1010E72450B44E3D817
:106B60006BE601934CF0BCFB019BD0F81CC04FF0CE
:106B7000000E00211F8894F900203A432CF8022BC4
:106B80000269D6F804806F6801318A4244443B446C
:106B9000F0D8316802FB18110C44296802FB171168
:106BA000C2680EF1010E72450B44E2D845E600BF03
:106BB0000222FFF7A3BB00BF2DE9F04307461046B2
:106BC0003A7983B08C46622A19460A9D0B9EFB696E
:106BD000DCF81C405ED019D8422A2CD0482A11D1AA
:106BE0009CF804E0BEF1480F00F00C81BEF1680F84
:106BF00000F02D81BEF1620F55D003D8BEF1420FD7
:106C000000F08280002003B0BDE8F083682AF9D14B
:106C10009CF80420682A00F04081622A43D0F1D811
:106C20009946B046BE46422A23462E4667464C4603
:106C30004546F446D2D19CF80420622A00F09580A3
:106C40006AD8422A3BD0482ADCD101934CF048FB59
:106C5000019BD0F81CC04FF0000E002127881A7845
:106C60007A402CF8022B0269D5F80480776801314C
:106C70008A4243443C44F1D8296802FB18110B4472
:106C8000316802FB1711C2680EF1010E72450C4407
:106C9000E3D8B8E7A046AE4662461C463546BC4639
:106CA0004346764617463A79622A00F01B81482A05
:106CB00000F03D81682A7FD0622A8DD9A2E7019336
:106CC0004CF00EFB019BD0F81CC04FF0000E0021D1
:106CD00027781A787A400CF8012B0269D5F80480DD
:106CE000776801318A4243443C44F1D8296802FB69
:106CF00018110B44316802FB1711C2680EF1010E26
:106D000072450C44E3D87EE7B6461A462E46234623
:106D1000BC46754614468EE7682A7FF473AF01932C
:106D20004CF0DEFA019BD0F81CE000270021B4F8FB
:106D300000C01A7882EA0C022EF8022B0269D5F8FC
:106D40000480D6F804C001318A4243446444EED83A
:106D5000296802FB18110B44316802FB1C11C26840
:106D60000137BA420C44E1D84DE7682201934CF058
:106D7000B7FA019BD0F81CC04FF0000E002194F927
:106D800000701A787A402CF8022B0269D5F804803A
:106D9000776801318A4243443C44F0D8296802FBB9
:106DA00018110B44316802FB1711C2680EF1010E75
:106DB00072450C44E2D826E701934CF091FA019B0E
:106DC000D0F81CC04FF0000E00211F8894F900205D
:106DD0007A402CF8022B0269D6F804806F680131E2
:106DE0008A4244443B44F0D8316802FB18110C44F9
:106DF000296802FB1711C2680EF1010E72450B449F
:106E0000E2D800E701934CF06BFA019BD0F81CC06C
:106E10004FF0000E002127881A887A402CF8022BA8
:106E20000269D5F80480776801318A4243443C44C2
:106E3000F1D8296802FB18110B44316802FB1711C5
:106E4000C2680EF1010E72450C44E3D8DBE67246CF
:106E500001934CF045FA019BD0F81CC04FF0000E96
:106E6000002127881A887A402CF8022B0269D5F86D
:106E70000480776801318A4243443C44F1D8296850
:106E800002FB18110B44316802FB1711C2680EF1A6
:106E9000010E72450C44E3D8B5E601934CF020FA9C
:106EA000019BD0F81CC04FF0000E002127881A88E3
:106EB0007A402CF8022B0269D5F8048077680131FA
:106EC0008A4243443C44F1D8296802FB18110B4420
:106ED000316802FB1711C2680EF1010E72450C44B5
:106EE000E3D890E601934CF0FBF9019BD0F81CC06D
:106EF0004FF0000E00211F7822787A400CF8012B09
:106F00000269D6F804806F6801318A4244443B44E8
:106F1000F1D8316802FB18110C44296802FB1711E3
:106F2000C2680EF1010E72450B44E3D86BE6019383
:106F30004CF0D6F9019BD0F81CC04FF0000E002198
:106F40001F8894F900207A402CF8022B0269D6F8A9
:106F500004806F6801318A4244443B44F0D8316870
:106F600002FB18110C44296802FB1711C2680EF1CC
:106F7000010E72450B44E2D845E600BF0322FFF73D
:106F8000BDB900BF2DE9F04117460279CC6982B046
:106F9000622A9C46089DC369099E6ED038D8422A51
:106FA00000F0A380482A40F09C800979019342298F
:106FB00000F03E81622900F04482482900F083817C
:106FC0006146384668224CF08BF9019BD0F81CC012
:106FD0004FF0000E0021B4F900701A88BA402CF866
:106FE000022B0269D5F80480776801318A42434454
:106FF0003C44F0D8296802FB18110B44316802FBAD
:107000001711C2680EF1010E72450C44E2D869E016
:10701000682A66D109790193422900F09880622993
:1070200000F0C18148293846614600F027814CF0C4
:1070300057F9019BD0F81CE000270021B4F900C0EB
:10704000B3F9002002FA0CF22EF8022B0269D5F8EF
:107050000480D6F804C001318A4243446444EDD828
:10706000296802FB18110B44316802FB1C11C2682D
:107070000137BA420C44E0D834E00A790193422A3D
:107080006146384600F08A80622A00F0B481482ABE
:1070900000F0408168224CF023F9019BD0F81CC01D
:1070A0004FF0000E0021B4F9007093F90020BA40AF
:1070B0002CF8022B0269D5F80480776801318A42E6
:1070C00043443C44EFD8296802FB18110B44316853
:1070D00002FB1711C2680EF1010E72450C44E1D893
:1070E00000E0002002B0BDE8F0810A790193422A55
:1070F0006146384678D0622A00F0CC81482A00F0F8
:107100002E8168224CF0ECF8019BD0F81CC04FF0A7
:10711000000E0021B4F900701A78BA402CF8022B46
:107120000269D5F80480776801318A4243443C44BF
:10713000F0D8296802FB18110B44316802FB1711C3
:10714000C2680EF1010E72450C44E2D8CAE76146EE
:1071500038464CF0C5F8019BD0F81CC04FF0000E2B
:1071600000212778B3F90020BA402CF8022B0269DD
:10717000D5F80480776801318A4243443C44F0D812
:10718000296802FB18110B44316802FB1711C26811
:107190000EF1010E72450C44E2D8A3E768224CF0D0
:1071A0009FF8019BD0F81CC04FF0000E00212778FB
:1071B00093F90020BA402CF8022B0269D5F804801C
:1071C000776801318A4243443C44F0D8296802FB85
:1071D00018110B44316802FB1711C2680EF1010E41
:1071E00072450C44E2D87DE74CF07AF8019BD0F868
:1071F0001CC04FF0000E002127781A78BA400CF816
:10720000012B0269D5F80480776801318A42434432
:107210003C44F1D8296802FB18110B44316802FB89
:107220001711C2680EF1010E72450C44E3D859E7FC
:10723000614638464CF054F8019BD0F81CC04FF022
:10724000000E002127781A88BA402CF8022B026918
:10725000D5F80480776801318A4243443C44F1D830
:10726000296802FB18110B44316802FB1711C26830
:107270000EF1010E72450C44E3D833E74CF030F8C0
:10728000019BD0F81CC04FF0000E0021B4F9007033
:107290001A88BA402CF8022B0269D5F80480776866
:1072A00001318A4243443C44F0D8296802FB18115A
:1072B0000B44316802FB1711C2680EF1010E7245D2
:1072C0000C44E2D80EE70A46384661464CF008F80E
:1072D000019BD0F81CC04FF0000E002127881A88AF
:1072E000BA402CF8022B0269D5F804807768013186
:1072F0008A4243443C44F1D8296802FB18110B44EC
:10730000316802FB1711C2680EF1010E72450C4480
:10731000E3D8E7E64BF0E4FF019BD0F81CC04FF048
:10732000000E0021278893F90020BA402CF8022B88
:107330000269D5F80480776801318A4243443C44AD
:10734000F0D8296802FB18110B44316802FB1711B1
:10735000C2680EF1010E72450C44E2D8C2E64BF051
:10736000BFFF019BD0F81CC04FF0000E0021278802
:107370001A78BA402CF8022B0269D5F80480776895
:1073800001318A4243443C44F1D8296802FB181178
:107390000B44316802FB1711C2680EF1010E7245F1
:1073A0000C44E3D89EE6614638464BF099FF019BBA
:1073B000D0F81CC04FF0000E002194F90070B3F912
:1073C0000020BA402CF8022B0269D5F804807768B7
:1073D00001318A4243443C44EFD8296802FB18112A
:1073E0000B44316802FB1711C2680EF1010E7245A1
:1073F0000C44E1D876E64BF073FF019BD0F81CC03B
:107400004FF0000E002194F9007093F90020BA406B
:107410000CF8012B0269D5F80480776801318A42A3
:1074200043443C44EFD8296802FB18110B443168EF
:1074300002FB1711C2680EF1010E72450C44E1D82F
:1074400050E60A46384661464BF04AFF019BD0F8A9
:107450001CC04FF0000E002194F9007093F9002039
:10746000BA400CF8012B0269D5F804807768013125
:107470008A4243443C44EFD8296802FB18110B446C
:10748000316802FB1711C2680EF1010E72450C44FF
:10749000E1D827E668224BF023FF019BD0F81CC0FF
:1074A0004FF0000E002194F900701A78BA402CF8C1
:1074B000022B0269D5F80480776801318A4243447F
:1074C0003C44F0D8296802FB18110B44316802FBD8
:1074D0001711C2680EF1010E72450C44E2D801E6A4
:1074E0000422FEF70BBF00BF2DE9F04117460279D9
:1074F000CC6982B0622A9C46089DC369099E6ED001
:1075000038D8422A00F0A380482A40F09C800979AC
:107510000193422900F03E81622900F0448248290B
:1075200000F083816146384668224BF0D9FE019B0A
:10753000D0F81CC04FF0000E0021B4F900701A887A
:107540003A412CF8022B0269D5F8048077680131A2
:107550008A4243443C44F0D8296802FB18110B448A
:10756000316802FB1711C2680EF1010E72450C441E
:10757000E2D869E0682A66D109790193422900F0CE
:107580009880622900F0C18148293846614600F0A0
:1075900027814BF0A5FE019BD0F81CE000270021BD
:1075A000B4F900C0B3F9002042FA0CF22EF8022B15
:1075B0000269D5F80480D6F804C001318A424344F8
:1075C0006444EDD8296802FB18110B44316802FBB2
:1075D0001C11C2680137BA420C44E0D834E00A7981
:1075E0000193422A6146384600F08A80622A00F000
:1075F000B481482A00F0408168224BF071FE019B63
:10760000D0F81CC04FF0000E0021B4F9007093F9BF
:1076100000203A412CF8022B0269D5F804807768E3
:1076200001318A4243443C44EFD8296802FB1811D7
:107630000B44316802FB1711C2680EF1010E72454E
:107640000C44E1D800E0002002B0BDE8F0810A79E6
:107650000193422A6146384678D0622A00F0CC81F4
:10766000482A00F02E8168224BF03AFE019BD0F8A8
:107670001CC04FF0000E0021B4F900701A783A4196
:107680002CF8022B0269D5F80480776801318A4210
:1076900043443C44F0D8296802FB18110B4431687C
:1076A00002FB1711C2680EF1010E72450C44E2D8BC
:1076B000CAE7614638464BF013FE019BD0F81CC068
:1076C0004FF0000E00212778B3F900203A412CF842
:1076D000022B0269D5F80480776801318A4243445D
:1076E0003C44F0D8296802FB18110B44316802FBB6
:1076F0001711C2680EF1010E72450C44E2D8A3E7DF
:1077000068224BF0EDFD019BD0F81CC04FF0000E3D
:107710000021277893F900203A412CF8022B0269C6
:10772000D5F80480776801318A4243443C44F0D85C
:10773000296802FB18110B44316802FB1711C2685B
:107740000EF1010E72450C44E2D87DE74BF0C8FD06
:10775000019BD0F81CC04FF0000E002127781A784A
:107760003A410CF8012B0269D5F8048077680131A1
:107770008A4243443C44F1D8296802FB18110B4467
:10778000316802FB1711C2680EF1010E72450C44FC
:10779000E3D859E7614638464BF0A2FD019BD0F88B
:1077A0001CC04FF0000E002127781A883A412CF8AF
:1077B000022B0269D5F80480776801318A4243447C
:1077C0003C44F1D8296802FB18110B44316802FBD4
:1077D0001711C2680EF1010E72450C44E3D833E76D
:1077E0004BF07EFD019BD0F81CC04FF0000E002135
:1077F000B4F900701A883A412CF8022B0269D5F8C6
:107800000480776801318A4243443C44F0D82968B7
:1078100002FB18110B44316802FB1711C2680EF10C
:10782000010E72450C44E2D80EE70A46384661461E
:107830004BF056FD019BD0F81CC04FF0000E00210C
:1078400027881A883A412CF8022B0269D5F804805F
:10785000776801318A4243443C44F1D8296802FBED
:1078600018110B44316802FB1711C2680EF1010EAA
:1078700072450C44E3D8E7E64BF032FD019BD0F8AB
:107880001CC04FF0000E0021278893F900203A41D8
:107890002CF8022B0269D5F80480776801318A42FE
:1078A00043443C44F0D8296802FB18110B4431686A
:1078B00002FB1711C2680EF1010E72450C44E2D8AA
:1078C000C2E64BF00DFD019BD0F81CC04FF0000E3E
:1078D000002127881A783A412CF8022B0269D5F842
:1078E0000480776801318A4243443C44F1D82968D6
:1078F00002FB18110B44316802FB1711C2680EF12C
:10790000010E72450C44E3D89EE6614638464BF0C2
:10791000E7FC019BD0F81CC04FF0000E002194F949
:107920000070B3F900203A412CF8022B0269D5F817
:107930000480776801318A4243443C44EFD8296887
:1079400002FB18110B44316802FB1711C2680EF1DB
:10795000010E72450C44E1D876E64BF0C1FC019B68
:10796000D0F81CC04FF0000E002194F9007093F97C
:1079700000203A410CF8012B0269D5F804807768A1
:1079800001318A4243443C44EFD8296802FB181174
:107990000B44316802FB1711C2680EF1010E7245EB
:1079A0000C44E1D850E60A46384661464BF098FC54
:1079B000019BD0F81CC04FF0000E002194F900701C
:1079C00093F900203A410CF8012B0269D5F80480A4
:1079D000776801318A4243443C44EFD8296802FB6E
:1079E00018110B44316802FB1711C2680EF1010E29
:1079F00072450C44E1D827E668224BF071FC019BEC
:107A0000D0F81CC04FF0000E002194F900701A78D5
:107A10003A412CF8022B0269D5F8048077680131CD
:107A20008A4243443C44F0D8296802FB18110B44B5
:107A3000316802FB1711C2680EF1010E72450C4449
:107A4000E2D801E630B5184CD4F8B43083B013B99D
:107A500009E01B683BB19A688242FAD15A688A42AF
:107A6000F7D103B030BDCDE900010C202BF026FB8F
:107A7000D4F8B4C0DDE90021BCF1000F0CD063469E
:107A800001E01B6843B19D68AA42FAD15D68A94232
:107A9000E7D01B68002BF6D1C0E900C18260C4F8B2
:107AA000B40003B030BD00BF4070012010B5DFF856
:107AB00030E0DEF8B4C0BCF1000F0AD0634601E04C
:107AC0001B6833B19C688C42FAD15C689442F7D150
:107AD00010BDC0E900C28160CEF8B40010BD00BF87
:107AE0004070012010B5054BD3F8B4402CB12046AE
:107AF00024F0AAFD2468002CF9D110BD40700120AB
:107B00000B4AD2F8B4308BB102F1B40C02E09C46BF
:107B10001B685BB19A688242F9D15A688A42F6D1F1
:107B20001968CCF8001000221A607047704700BF37
:107B3000407001202DE9F843144CD4F8B4701FB301
:107B40004FF000093846B8463F6825F06DF820B977
:107B5000D8F8040025F068F8A0B1D4F8B4308BB19F
:107B6000D8E9012104F1B40002E018461B684BB1CA
:107B70009E68B142F9D15E68B242F6D11A680260DD
:107B8000C3F80090002FDDD1BDE8F88340700120DC
:107B90000349044A0023C1F8B4301370704700BF92
:107BA00040700120187B012008B5074B1B780BB9EA
:107BB000002008BD054808F0FBFE0028F8D1BDE80C
:107BC0000840024808F054BFF37A0120E84401203D
:107BD000014809F0C1BB00BF4045012000B50B487A
:107BE00083B008F0E5FE68B9094A127852B103463D
:107BF00001220DF10701054808F0E0FE9DF807009D
:107C000003B000BDFF2003B000BD00BFE844012069
:107C1000F37A01202DE9F041074682B013480E4661
:107C200009F004FCF0B9124B1B78DBB1D6B1044665
:107C300080460CE0AAB239190C48CDF80080002328
:107C400009F01AFD002804440CDBA6420AD90748B3
:107C500009F034FC351B8542ECD3044809F02EFCB6
:107C600082B2E8E702B0BDE8F08100BF40450120E4
:107C7000F37A012008B509F06DFB0348012108F0F3
:107C80006BFA0E2008BD00BF700D012030B585B025
:107C900002AB51F8044B01930C4B009301380223C3
:107CA0002EF088F840F29E22094902982EF018FA28
:107CB00040F2226105469FED070A03982EF0C2F9B3
:107CC0002946204608F0E2F805B030BDFCB40B00B0
:107CD000CCB60B000000000008B508F085F90E20B6
:107CE00008BD00BF08B5152124F0DEFCBDE8084042
:107CF0000148AA2124F0D8BCA00A012008F076B9D6
:107D000008B508F08FF900280CBF1E203E2008BDE2
:107D100008B508F08DF900280CBF1E203E2008BDD4
:107D200008F09AB908B508F0C3F900280CBF1E2066
:107D30003E2008BD30B585B000240546ADF80610DC
:107D400020460DF10E01ADF80E4058F03BFB0DF151
:107D50000601284658F036FB18B9BDF80E0005B0EC
:107D600030BD204605B030BD08B5014869F0F8F8CF
:107D700084900B002DE9F041036905465BB158F092
:107D800035FB286901215BF04FFC27482969FFF783
:107D9000B7FE00232B61EB688BB1244B1878FF28CA
:107DA0000DD058F0FDFA294604462148FFF7A8FEF9
:107DB0000023EB6085F8443034F0080330D11D4CCB
:107DC0000023AB6104F52A7825464FF6FF770E268F
:107DD0002B88BB42284601D009F02CF8EE65883587
:107DE0004545F5D161F030FE4FF6FF7506460F466A
:107DF00000231A4634F813104433A94218BF42F046
:107E00000102B3F5AA7FF5D142B161F01DFE801BDE
:107E100061EB0701802871F10001E9D3BDE8F08131
:107E2000204603F0DDFFCAE7BDFF0800A7060120DA
:107E300005010300A00A012010B58EB004462022DF
:107E40001D4806A959F0D4FE80B31C4B0FCB0DF191
:107E5000080CACE807002046ACF8003008F0C6F883
:107E6000F0B1694608F0A6FC9DF8010014499DF8A0
:107E700000204FEA101C00F00F0011F80CC0085C45
:107E800000236CF3070360F30F23100902F00F02C5
:107E9000085C8A5C60F3174362F31F63CDF811300E
:107EA00002A9204608F09CFA0EB010BD06A9204693
:107EB00008F096FA0EB010BD24180B0038180B000D
:107EC00068630B0008B508F02DF908B10E2008BD55
:107ED00001483CF0B5FD00BF648F0B0010B50446AF
:107EE000084638F0A7FA0146204608F035F90E207A
:107EF00010BD00BF10B5044608463AF0E9FC014643
:107F0000204608F06DFA0E2010BD00BF70B52DEDB3
:107F1000028B51F8043B94B01D460CAB0193394BD6
:107F20000093013808232DF045FF0C98052206A97F
:107F300033F0AAFB0D9800230E28CDE909330B93EB
:107F400003D0052209A933F09FFB1198002847D0E0
:107F500040F239412EF0DEF8DFED2B7AB4EEE70A7D
:107F6000F1EE10FAB0EE408A43D4DFED287AB4EE99
:107F7000E70AF1EE10FA3CDC40F2226210989DF81C
:107F800038409DF83C6000212EF00CF8079A1F2A1B
:107F900003461DD813980E2820D03CB31C490593E6
:107FA00040F27B322EF09CF8059B039009AA0192C7
:107FB000214606AA129C00922846B0EE480A324694
:107FC000029408F021FA0E2014B0BDEC028B70BDB3
:107FD0004CB10A9A92B913980E28DFD10020E4E739
:107FE0000C481190B4E7139A0E2AF7D00A483CF0D7
:107FF00027FD0A4A0A490B4869F032F80A483CF062
:108000001FFD00BF7CB40B000AD7A33C0AD7234155
:10801000CCB60B00CECC4CBEE4890B0014180B0080
:108020001C180B00487B0B0044900B0010B52DED85
:10803000048B51F8043B90B01C4608AB0193444BB1
:108040000093013808232DF0B5FE0B980E2866D05A
:108050009FED400A40F222612DF0F4FF0C98F0EE03
:10806000408A002860D00D9B002B62D040F239413D
:108070002EF050F8DFED387AB4EEE70AF1EE10FAA0
:10808000B0EE408A58D4DFED357AB4EEE70AF1EE6F
:1080900010FA51DCF5EE408AF1EE10FA04D0F4EE5D
:1080A000C08AF1EE10FA4FD40D9840F287612EF09D
:1080B00031F8B4EEC08AF1EE10FAB0EE409A40D436
:1080C00008980023069328B1052205A933F0DCFAAD
:1080D000069BE3B909984FF43F7201212DF062FF2E
:1080E0009DF83C100E9A0090CDE901219DF82830B2
:1080F000DDE90512B0EE491AF0EE480AB0EE680A62
:10810000204608F031FA10B0BDEC048B10BD059884
:1081100024F08AFD0028DDD1114868F099FF0C9801
:10812000DFED0C8A00289ED10D9B0E480C90002B91
:108130009CD10C4B0D9399E70B4A0C490C4868F005
:108140008FFF0C4868F084FF0B4868F081FF00BF88
:10815000BCB40B00000000000AD7233B66D62342C4
:1081600040890B00CECC4CBE00180B000C180B0045
:10817000487B0B0080720B0044780B0008B508F0B8
:10818000D9FA0E2008BD00BF08B508F0F3FA0E209A
:1081900008BD00BF022808D1900708D108B50C4BD4
:1081A0001068984205D01E2008BD002070471E2090
:1081B0007047087913799842F5D1481D511D062260
:1081C0002CF084FD00280CBF3E201E2008BD00BFFF
:1081D000CCB60B0008F0EABA08B508F0F3FA400094
:1081E00040F0010008BD00BF10B508468AB0114636
:1081F0001A46134B0DF1140CCDE9003C02232DF06F
:1082000081FE07A90598052233F03EFA089840F24E
:108210009E2206212DF0E2FE40F2A12303220698C1
:1082200000212DF0CBFE074904460C2038F0ECFA73
:1082300007990390E2B208F0B1FA03980AB010BDB2
:108240007CB60B00CCB60B0000B50A4685B092F8A0
:1082500005C093790649CDE9023C92F807C0137A2C
:10826000CDE9003C537A927A3CF018FB05B000BD92
:1082700048180B00062801D00020704700B50B46B7
:1082800083B00146581D019355F01AFA019B1B79E2
:108290005840400040F0010003B000BD312926D80D
:1082A000102928D91139202914D8DFE801F0171A2C
:1082B00013131313131313131313131313131D1186
:1082C0001313131313131313131313131313140090
:1082D000222303707047312303707047112303700A
:1082E00070471223037070472123037070474129A0
:1082F00004D1017070470029FBD07047704700BF60
:1083000001F0E6B82DE9F04F474B97B00DACCDE941
:1083100000340431092301382DF04CFD43490D98F8
:1083200040F2A4522DF0DCFE4149824640F26962DF
:108330000E982DF0D5FE9DF83C503F2D70D89DF83D
:1083400040608346304608F03FFA9DF84470384656
:1083500008F03AFA129840F2844200212DF022FEF1
:10836000149B9DF84C800E2B044614D00DF1280967
:1083700018460522494633F087F9B8F1000F14D0AA
:108380000B9840F22D4221462DF028FE15980E281C
:1083900014D1002315E0B8F1000F29D10DF12809FF
:1083A00024480522494633F06FF90B9840F22D42DC
:1083B00021462DF01FFE15980E28EAD03AF088FAD3
:1083C00003461D490993282038F01EFA099B0095A1
:1083D000CDE90593CDE90348CDE901675B4600226D
:1083E0005146089008F07CFB089817B0BDE8F08F64
:1083F00068B90DF12809494605220E4833F044F9C1
:108400000B9840F22D4221462DF0E8FDBEE70DF11C
:10841000280938F097FA0522494633F035F9AFE7D5
:1084200040F212502DF0B8FC84B70B007CBD0B005D
:1084300054BE0B00A8600B00DCB70B0008B508F0B9
:10844000A1FA0E2008BD00BFF8B504460D46174638
:108450001E4608F0ADFAA0B9204608F05DFA90B1CA
:10846000032D04D0162333604FF0FF30F8BD17F012
:108470000100FBD0204608F0FBFA003818BF0120AD
:10848000F8BD55F043FB014868F04EFD608A0B00D3
:1084900010B508468AB011461A46164B0DF11C0C51
:1084A000CDE9003C03232DF02DFD40F2123212499C
:1084B00007982DF015FE40F222610446B7EE000A3F
:1084C00008982DF0BFFD4FF43F7209988DED050A15
:1084D00001212DF067FD09490490242038F094F91A
:1084E000049A9DED050A0390214608F021FA0398AD
:1084F0000AB010BD08B90B00DCB70B0020B90B00A7
:1085000010B582B0044608F053FA98B9204608F036
:10851000AFFA034620B1580040F0010002B010BD90
:108520000190204608F0F8F9019B0028F3D1024899
:1085300068F0FAFC55F0EAFA608A0B0010B50446C0
:1085400008F036FA20B9204608F0A4F90E2010BD34
:1085500055F0DCFA2DE9F04105460E4614461F465B
:1085600008F026FA90B9284608F0D6F958B114B99F
:108570002046BDE8F0813B46224631462846BDE80C
:10858000F04108F01BBA024868F0CEFC55F0BEFA84
:10859000608A0B0008B5014868F0E2FCEC8F0B0024
:1085A00008B508F007FB0E2008BD00BF10B5044653
:1085B00008F006FB20B92046BDE8104008F006BBD5
:1085C00055F0A4FA10B5044608F0FAFA30B920467E
:1085D00008F008FB400040F0010010BD55F096FA8D
:1085E00010B5044608F0ECFA30B9204608F0FCFA61
:1085F000002808BF0E2010BD55F088FA10B5ADF563
:10860000007D044608F0DCFA58B94FF40072694660
:10861000204608F0EBFA694638F012F90DF5007DB6
:1086200010BD55F073FA00BF10B58C6882B094B1DC
:1086300000910C49019204463CF030F9DDE900322A
:108640002046996800F066FE0749204602B0BDE862
:1086500010403CF023B9054902B0BDE810403CF0A1
:108660001DB900BF70180B0098110B0080180B008B
:1086700030B50C6887B005462046CDE9022108F0E8
:108680009FFADDE9022190B904AB0193094B0093F5
:10869000681E022304312DF08DFB20469DF8142026
:1086A0009DF8101008F0C6FA0E2007B030BD55F046
:1086B0002DFA00BFCCB70B0030B585B004460D468F
:1086C00008F07EFA58B9052201A9284632F0DCFFED
:1086D000204601A908F0F6FA0E2005B030BD55F08D
:1086E00015FA00BF08B54FF6FF73984200D008BDD9
:1086F000014868F019FC00BF608A0B00014B0022A2
:108700001A707047027B01200023DFF824C01A464C
:108710003CF81310814203F1440304D00132052ACE
:10872000F6D10020704702EB02120CEBC20070473A
:10873000A00A012000234FF6FF724360028080F8F8
:108740005A308370083001F0A5B800BF08B5406802
:1087500008F070FB0E2008BD10B584B003AB51F8D3
:10876000044B0193094B0093013801232DF022FBA8
:10877000204608F0C1FC28B10399204608F05EFBB2
:1087800004B010BD024868F0CFFB00BFC8B90B00B1
:10879000988F0B0008B508F0AFFC00B108BD014888
:1087A00068F0C2FB988F0B0018B143680BB11888B2
:1087B00070474FF6FF70704708B508F09DFC002821
:1087C0000CBF1E203E2008BD10B5044608F094FCE6
:1087D00090B1606808F09AFCB4EE400AF1EE10FA2D
:1087E00008D610EE103A23F0030040F00200A0F18A
:1087F000FF4010BD024810BD024868F095FB00BF65
:1088000002004000988F0B0010B5044608F074FC7D
:1088100030B1606808F094FCBDE8104038F018BA38
:10882000014868F081FB00BF988F0B0008B508F085
:108830008FFC00280CBF1E203E2008BD0346C06DE3
:108840000E2800D0704700B583B0054901930C2075
:1088500037F0DAFF019B4360D86503B000BD00BF6D
:10886000D0B90B0010B584B003AB51F8044B0193A1
:108870000F4B0093013801232DF09CFA9DF80C302A
:108880005BB1204608F038FC70B160689DF80C10B0
:1088900008F068FC0E2004B010BD064840F25112EA
:1088A00040F2F32168F064FB034868F03DFB00BF31
:1088B000C0B90B00A4930B00988F0B0010B50446B1
:1088C00082B0084636F0D2FB20468DED010A08F052
:1088D00013FC9DED010A28B1606808F07DFC0E20B4
:1088E00002B010BD014868F01FFB00BF988F0B005D
:1088F0002DE9F04F3E4B8FB007ACCDE90034043189
:10890000072301382DF056FA3A49079840F21232FF
:108910002DF0E6FB384940F26962064608982DF0D2
:10892000DFFB9DF824708346384607F04DFF9DF825
:108930002880404607F048FF0B9840F2844200210F
:108940002DF030FB0D9B9DF830900E2B044610D07F
:108950000DF1100A18460522514632F095FEB9F184
:10896000000F10D0059840F22D4221462DF036FB25
:108970000FE0B9F1000F22D10DF1100A1F480522B6
:10898000514632F081FE059840F22D4221462DF0ED
:1089900031FB1B49182037F037FF3B4605465A4646
:1089A0003146CDE9029ACDE9008408F039FC304621
:1089B000294607F01BFF28460FB0BDE8F08F68B9C5
:1089C0000DF1100A514605220C4832F05DFE059863
:1089D00040F22D4221462DF001FBDAE70DF1100A9D
:1089E00037F0B0FF0522514632F04EFEBAE700BF25
:1089F000B8BA0B00DCB70B0054BE0B00A8600B002C
:108A0000F0BA0B0008F03ABC08B508F039FC0028B1
:108A100008BF0E2008BD00BF00B5ADF5017D4FF4C5
:108A20000072694608F02EFC694637F009FF0DF523
:108A3000017D00BD10B58C6882B094B100910C49E5
:108A4000019204463BF02AFFDDE900322046996896
:108A500000F060FC0749204602B0BDE810403BF042
:108A60001DBF054902B0BDE810403BF017BF00BF75
:108A7000A8180B0098110B00B4180B0010B584B0A7
:108A800004460522084601A932F0FEFD204601A950
:108A900008F01EFC0E2004B010BD00BF10B5022A65
:108AA00082B004460B4606D01946204602B0BDE807
:108AB000104035F0EDBE4FF42270CDE9001254F0B5
:108AC000A9FF014620463BF047FE064920463BF001
:108AD00043FEDDE900322046194602B0BDE81040F1
:108AE00035F0D6BE68190B0030B50C464FF6FF7155
:108AF0008C4289B03DD00546002004908DF81800C6
:108B000002A92148ADF81440CDE90223FEF79AFFEF
